:020000040000FA
:2000000080FF0010590100001D0100001F01000021010000230100002501000082F9FEEFE5
:200020000000000000000000000000002701000029010000000000002B010000492A0000CF
:200040002D0100002D0100002D0100002D0100002D0100002D0100002D0100002D01000030
:200060002D0100002D0100002D0100002D0100002D0100002D0100002D0100002D01000010
:200080002D0100002D0100002D0100002D0100002D0100002D0100002D0100002D010000F0
:2000A000D10300002D010000592A00002D0100002D010000912A00002D0100002D01000048
:2000C0002D0100002D0100002D0100002D0100002D0100002D0100002D0100002D010000B0
:2000E0002D010000946A00000000001088040000946A000000080020000000008804001076
:20010000F0C9000000080020000000008760ACD42D90F644472466B49B2C178CFEE7FEE7E7
:20012000FEE7FEE7FEE7FEE7FEE7FEE7FEE70B4610B5401A5C1AA24200D810BDC45843F8B6
:20014000044BF7E710B5034600241A1A914200D810BD43F8044BF8E738B50D4C0D4DAC429D
:2001600007D30D4DAC420CD302F0C2FF06F0E8F8FEE794E803000C3454F8042CFFF7D7FF09
:20018000EDE754F8080B54F8041CFFF7DBFFE9E7E4000000FC0000000C0100005F64667595
:2001A0000D0A00586D6F64656D20746F6F206D616E79207265747279206572726F7200587F
:2001C0006D6F64656D2073796E63206572726F7200586D6F64656D2063616E63656C65642D
:2001E0002062792072656D6F7465007374617274696E67206170706C69636174696F6E2E0A
:200200002E2E0D0A00444655206D6F64650D0A006170706C69636174696F6E20636F727246
:2002200075707465640D0A0073656C6675706461746520666F756E640D0A0073656C6675E6
:2002400070646174652066696E616C697A65640D0A006170702075706461746520666F7555
:200260006E640D0A0062616420636865636B73756D0D0A00636865636B73756D206F6B0D8A
:200280000A00636865636B696E67207570646174652E2E2E0D0A0061707020757064617455
:2002A00065206E6F7420666F756E640D0A006261642066696C652073697A650D0A00626179
:2002C00064207570646174650D0A005F70645F6C64722E62696E007570645F6C64722E624B
:2002E000696E005F70645F6170702E62696E007570645F6170702E62696E00FF214365874E
:2003000091000000951000008D100000291400004514000049160000511600003114000069
:20032000EF2830B50ED8084B084D13442C6803EBC020074B14441A68064B2C601A6008608F
:20034000002030BD082030BD00000080BC070010E8B800108804001070B505460A4CD0F84E
:20036000A80166882146324605F0E6FF32462146D5F8AC0105F0E0FFBDE870400122034B3A
:2003800003485A6002F056BB386400008C040010FB6700000122024B02489A6002F04ABB0C
:2003A0008C0400101B68000008B5024802F042FB072008BD0868000003780BB91846704734
:2003C0004278042A02D142798A42F8D01844F3E7034B044A1B6810681B68DB68184700BF62
:2003E00080040010B8070010F0B516461D46194B8BB0186007460C462422002101A805F07B
:200400009DFF336801932B6802934FF40063ADF80C30E4B16379FE2B19D1A379012B16D1AF
:200420000D4B049405930D4B022206930C4B01A907930C4B384608930B4B1B68DB685B6835
:200440009847019B3360029B2B600BB0F0BD4FF0FF30FAE78C04001021030000A90300003F
:200460009503000059030000800400102DE9F04F0025BFB00DF10C0810222E49074640467D
:2004800005F05AFF022003F09BFC23A800F0CCFF23A800F0D7FF2C46DFF8A090264EDFF887
:2004A000A0A0BC4203D100203FB0BDE8F08FCDF800804FF4E043102207A909EB041007F16A
:2004C000FF3B02F099FC5C4512D0079BB360089BB360099BB3600A9BB3607B1F9C421BD299
:2004E000102207A923A801F0AFF800250134D8E70BA923A801F0ACF823A800F099FFB3681C
:20050000079A9A42E9D113A90BA800F073FF70B9504602F08FFAE0E75C45E7D013AB58194B
:20052000102207A9103505F007FFEDB2DEE70120BAE700BF0C0100000000092000000080FE
:20054000306800002DE9F04F824699B0022003F095FA4422002107A805F0F0FE514B524DA5
:20056000079303238DF828304FF0005308934FF4006309934D4B4E4E02934E4B4E4F0393DA
:20058000002306932B6033684C4C1B68059704975B6807AA02A92046984798B9FE213846D5
:2005A000FFF70AFF0146002859D13022444B012183F818234FF080721A60336820681B6899
:2005C0009B6898473F4B404F98463A68DFF80C91DFF80CB11A603B68D8F800209B1A53453E
:2005E00047D8D9F80430C3B1336800211B6820689B689847002340F2DC502B60019302F028
:20060000C1F9584602F016FA326801211268206892689047019BC9F80430D9F80830012B2B
:20062000D9D1336800211B6820689B6898472B68B3F5E04F24D0B3F5F02F30D1234802F0E4
:20064000F9F928680009FFF711FFA8B1204802F0F1F903F059F960B102F08AFB09E08379BA
:20066000012BA2D109AB08AA2068FFF7BDFE00289BD019B0BDE8F08F164802F0DBF9F8E7B9
:20068000124802F0D7F928680009FFF7EFFE0028F2D00F4802F0CEF905F0C2FEE9E70E48ED
:2006A000EBE700BF00C20820BC07001054640000800400108464000068640000B80700101D
:2006C00000E100E088040010E8B80010820200007402000065020000AE0200008C0400105C
:2006E0002368000070B50446002020C940CA40087541404120C4013BF7D170BD70B501240F
:2007000020C940CA6408B541644120C0013BF7D1B4FA84F0400970BD2DE9F0410024013BBC
:200720009B0025462646A6465FF0000C03E05FEA0E0CBCEB030CBEEB0C0752F8078051F82E
:200740000C70A7FB0878E41955EB080556F100061CF1040C9C4501DCF445ECDD40F80E4001
:200760002C46354600261EF1040E9E45DCDDBEEB430FDCDD40F80E40BDE8F081002310B571
:200780001C465AB2914200DC10BD40F823400133F7E700231A4610B55CB2A14203DCB2FAFE
:2007A00082F0400910BD50F8234001332243F3E701234A1150F8220001F01F0103FA01F1AA
:2007C00008407047013949B2002904DA013149B231B90846704750F82130002BF2D0F5E760
:2007E00001F18043013B50F82330002023B9013900EB411108B270475B080130F6E70023F5
:2008000010B55CB2A24200DC10BD51F8234040F823400133F5E710B5013A52B2002A01DA18
:20082000002010BD50F8224051F822309C4203D8F2D24FF0FF3010BD012010BD002300EBD2
:200840008101884200D3704751F8042C43EA520341F8043DD307F4E770B59DF910401E4629
:2008600023460546FFF73EFF30B9224629463046FFF7D1FF012807D02346324629462846D7
:20088000BDE87040FFF73ABF70BD70B59DF910401E4623460546FFF731FF38B123463246D4
:2008A00029462846BDE87040FFF71CBF70BD2DE9F04F1F46B5B09DF9F84004AD234681463A
:2008C0002846FFF729FF24AB2146384602930395FFF778FF2026C0EB841005B295FBF6F686
:2008E0006B4276B203F01F0305F01F0814A858BFC3F100083146FFF741FFB8F1000F4FEAC5
:2009000086002ADD002214AB18441346C8F1200EA34217D30126630001934FEA840814AB5C
:2009200003EB080A671E34AB03EB8707002D52DB002334AAC6F101009E4602EB860C02EB74
:2009400080002BE057F8236006FA08F10A4340F8232026FA0EF20133DAE714AB22463946BE
:200960001844FFF74CFFD5E75CF8C82C0DF1D00B0BEB810B52F821205BF880BCA2EB0B0BBE
:20098000ABEB0E0B5A4504D034BF4FF0010E4FF0000E50F8C82C013342F821B0019A59B286
:2009A0009142E1DBA6EB0E035E42214614A85E41FFF744FF34AB434453F8802C57F8803C03
:2009C000214643EAC2735046013D47F8803C2DB2FFF734FFAAE734AB03EB8606224656F8D7
:2009E000C81C4846FFF70BFF35B0BDE8F08F30B505461C4691B0684693F90030FFF78CFEBF
:200A0000D4F8AC3069462846984711B030BD13460A46FFF7ECBF2DE9F04793F9006092B0BF
:200A2000044689461046314615469846FFF7B1FE002840F093804246494602A8FFF7E7FFEA
:200A4000434602AA21460AA8FFF7D1FF02A908464246FFF7DCFF43462A4649464846FFF724
:200A6000C6FF08F10407424629462846FFF7CFFF3B462A46214620460096FFF7EDFE3B46CE
:200A80002A46294628460096FFF7E6FE3B462A46214628460096FFF7F8FE43462A462146F1
:200AA0002046FFF7A4FF3B462246214628460096FFF7D2FE3B4600962A4621462046FFF7D3
:200AC000CBFE2368DB074CD533463A4621462046FFF708FE824631462046FFF7AFFE06F1BE
:200AE0008043013B54F8230040EACA7044F82300424621462846FFF78AFF3B460AAA294645
:200B000028460096FFF7C1FE3B460AAA294628460096FFF7BAFE0AA908463B462A4600963E
:200B2000FFF7B3FE43460AAA21462046FFF75FFF02AA3B46104621460096FFF7A6FE32461E
:200B400029462046FFF75BFE324649462846FFF756FE324602A94846FFF751FE12B0BDE855
:200B6000F08731462046FFF769FEC1E72DE9F04115468AB0044688462022002102A805F026
:200B8000DDFB032395F900702A46414620462E1D0293FFF73CFF334602AA21462046009762
:200BA000FFF773FE2B46424621462046FFF71FFF0097334605F1840221462046FFF74CFE5B
:200BC0000AB0BDE8F081FFFFF0B5082289B00C460646FFF714FE0027CB6A6A4603930B6B81
:200BE000684604934B6B029705938B6B01970693CB6B6946079308230097FFF773FD0823D0
:200C000005466A4631463046FFF76CFD236B05440393636B6A460493A36B69460593E36B68
:200C20006846069308230797FFF75CFD082305446A4631463046FFF755FD236A0544009393
:200C4000636A6A460193A36A31460293A36B30460693E36B05970793082304970397FFF773
:200C600041FD636AA26B0093A36A04920193E36AE26B0293636B054403930693236A0592F9
:200C800007936A46082331463046FFF72BFDE36A05440093236B6A460193636B31460293FF
:200CA000236A30460693A36A05970793082304970397FFF723FD236B2D1A0093636B6A46F9
:200CC0000193A36B31460293E36B30460393636A05970693E36A049707930823FFF70EFD5C
:200CE000636B2D1A0093A36B6A460193E36B31460293236A30460393636A06970493A36AF9
:200D00000593236B07930823FFF7F8FCA36B2D1A0093E36B6A460193636A31460393A36A9D
:200D200030460493E36A02970593636B069707930823FFF7E3FC2D1A0D4C0FD435B9082288
:200D400031462046FFF767FD01280FD00823224631463046FFF7D2FC2D1AEFE70823224660
:200D600031463046FFF7BEFC2D18F7D409B0F0BD30650000F0B515461C4607460E4689B08F
:200D80001A4629466846FFF742FE23466A4639463846FFF72CFE23462A4669466846FFF73E
:200DA00026FE23466A4631463046FFF720FE09B0F0BD2DE9F043144680461F4689468BB0B7
:200DC000129D024615F9046B21462B4602A80096FFF75BFD02A9129A0846FFF718FE129BDB
:200DE00002AA41464046FFF702FE129B02AA21462046FFF7FCFD2B464A463946384600969B
:200E0000FFF743FD129A394602A8FFF700FE02A92B46424608460096FFF737FD02A92B4605
:200E2000224608460096FFF730FD2B464246214620460096FFF729FD129B22464946484699
:200E4000FFF7D5FD2B4602AA414620460096FFF71CFD129B224639463846FFF7C8FD2B46DD
:200E60004A46394638460096FFF70FFD324602A92046FFF7C4FC0BB0BDE8F083F8B5042367
:200E80000E46D11C91FBF3F1144649B20546FFF775FC0022671E51B28C4202F1010200DC50
:200EA000F8BD7B1A23F00300715C03F00303DB0001FA03F3295819432950ECE72DE9F047CA
:200EC000B3F902401E462023884604F11F0191FBF3F70823073494FBF3F4944228BF144631
:200EE0004FFA87F949460546FFF748FC22464146FFF7C4FFB6F90230E4009C4221D90022AE
:200F0000E41A05EB8701C4F120078D420FD324364A4629463046FFF77EFC012811D04B46F4
:200F2000324629462846BDE8F047FFF7E7BB51F8040C20FA04F3134341F8043D00FA07F2BB
:200F4000E3E7BDE8F087036870B513F001050646144605D013460A460146FFF7C3FB0546A8
:200F600021463046FFF76AFC45B104F18042013A56F8223043F0004346F8223070BDF0B5D8
:200F80000F46A1B006461946384615461C46FFF700FC28B121463046FFF7F0FB21B0F0BDBE
:200FA000224639466846FFF72AFC2246294608A8FFF725FC214610A8FFF7E0FB0123214667
:200FC00018A81093FFF7DAFB224608A96846FFF722FC28B9224610A93046FFF710FCDDE7CA
:200FE000009BDA0709D421466846FFF727FC2246294610A8FFF7A7FFE6E7089BDB0707D412
:20100000214608A8FFF71AFC2246294618A8F1E7002823461CDD08AA69466846FFF76EFB46
:2010200021466846FFF70AFC224618A910A8FFF7F2FB002805DA10A923462A460846FFF7FE
:2010400051FB10A9234618AA0846FFF757FBCEE708A96A460846FFF751FB214608A8FFF717
:20106000EDFB224610A918A8FFF7D5FB002805DA18A923462A460846FFF734FB18A92346A3
:2010800010AA0846FFF73AFBBEE7FFFF004870472C6500002DE9F04F1D462023FDB0869E1E
:2010A0004FF0000BB6F9027080461F3797FBF3F77FB207F1FF3924AB43F829B07CAB96F933
:2010C0000040059203EB890242F8C0BC42F8A0BC8A4696F9012001466CA8FFF7CFFEA30033
:2010E0000793A2006CAB134496F90120184608EB02010493FFF7C2FE294696F901204CA8E2
:20110000FFF7BCFE96F9012054A8A918FFF7B6FE21464CA8FFF73DFB0546002840F03D811E
:20112000214654A8FFF735FB8346002840F0338106F124033A464CA918460393FFF76BFB6E
:20114000012840F02A813A4654A90398FFF763FB0128069040F021811CAD0DF130083B460E
:20116000039A54A92846FFF70AFF514640463346059A48F829B0FFF7A1FE41464046039BDA
:201180002A460097FFF793FB0DF5B879039B2A464CA914A80097FFF78AFB484622466CA9B5
:2011A000FFF72DFBA30009EB030A504622460499FFF725FB06F144031946224634A8049344
:2011C000FFF71DFB049BA100591822463CA8FFF716FB331D494634AA284600940593FFF7B0
:2011E00054FB53464A463CA934A80096FFF7E1FD2346321D29462846FFF7C1FE2A465146FB
:2012000048463346FFF7B6FD049B3946099340466CAB0A93CDF82C90CDF820B0FFF7D2FA52
:201220003946814614A8FFF7CDFA8145B8BF81461FFA89F909F1FF331BB2194640460493DB
:20124000FFF7B6FA049B10F10008194614A818BF4FF00108FFF7ACFA002814BF0223002327
:201260000DF1200A43EA08085AF828802246414624A8FFF7C4FA0DF1B00AA30008EB03014E
:2012800022465046FFF7BBFA21462846FFF776FA069BA9F102082B600FFA88F80DF190097A
:2012A0000495B8F1000F22DA049923460846059AFFF765FE3346049A51464846FFF75AFD0C
:2012C0003A4649460398FFF7A6FA012805D03B46039A49464846FFF711FA013C64B2002C15
:2012E0004EDABBFA8BF040097DB0BDE8F08F3346049A51464846D6F8A450A84741460CA8D4
:20130000FFF756FA031C18BF0123414614A80693FFF74EFA002814BF02200020069B18431A
:2013200008AB53F8203033B31946224634A80693FFF765FA069B0799224659183CA8FFF7F4
:201340005EFA3346049A3CA934A8FFF713FD059B34AA494644A80094FFF797FA53464A461A
:201360003CA934A80096FFF724FD0499334644AA0846FFF73CFB08F1FF380FFA88F890E750
:201380007CAB03EB840252F8C02C59F8243053404BEA030BA1E72846A6E75846A4E7FFFF57
:2013A00000B5C1B004224FF4FC41684604F0C4FF009B01331AD14FF480724FF4FC416846DF
:2013C00004F0BAFF40220A49684604F0B5FF0721084605F019F84FF4807269464FF4FC4076
:2013E00005F026F8012041B05DF804FB0020FAE7DC65000030B504460D4693B040220849BA
:2014000002A804F099FF074B2022009321462B4602A8FFF73FFE003018BF012013B030BDE2
:20142000DC6500002C6500006C22002104F086BF20B1002200F16C03984200D170470270CB
:201440000130F9E700230C4A036082600B4A4360C2600B4A836602610A4A42610A4A8261D4
:201460000A4AC2610A4A026202F17452A2F52302A2F692424262704767E6096A85AE67BBEC
:2014800072F36E3C3AF54FA57F520E518C68059BABD9831F2DE9F04F00F10803CBB00093D1
:2014A0001A46002352F8044B02A840F823400133082BF7D14FF0000E059BDDF824B0069D63
:2014C000089FDDF81CC002AC0193ADF1180294E85004BEF10F0F61D84B7891F800901B04E9
:2014E00043EA0968CB7848EA030391F8028043EA08231364354B4FEAF52853F82E3088EA08
:20150000B5181846136C88EA756818448CEA07032B4080447B409844019BD8444344184693
:2015200046EA04094FEA743306EA040B83EAB40309EA0A0949EA0B0983EAB4530EF1010E9C
:201540004B44BEF1400F434401F1040102F10402BB46CDF804A01AD1029300230997069044
:20156000CDF820C0079503940496CDF814A0009A02A951F82310126801330A440099082BF7
:2015800041F8042B0091F2D14BB0BDE8F08FB24667462646AC461C4605469AE7936BD2F877
:2015A00004904FEAF34888EA734888EA9328536A1846136818444FEAB94383EAF913804465
:2015C00083EAD90908EB090393E700BF1C6600002DE9F041054603680E4603F03F00134428
:2015E0009A422B6088BF6B68144684BF01336B6078B1C0F14007974216D805F128083A4640
:20160000404404F099FE41462846FFF743FF3E44E41B2746E11B3F2F31440ED8002024F0A7
:201620003F031E4404F03F0464B12835224631462844BDE8F04104F07FBE2846FFF72AFF7E
:20164000403FE7E7BDE8F0810AB1FFF7C1BF7047F7B502680D464168530F43EAC103044690
:20166000180ED1008DF80000180C02F03F023B4F8DF801008DF80330180A0B0E372A8DF8AE
:2016800004304FEA114394BFC2F13806C2F178068DF802008DF805308DF807100B0A4022C0
:2016A000002138468DF8063004F048FE80233246394620463B70FFF7C7FF082269462046F0
:2016C000FFF786FFE37A2B7063896B70A3681B0AAB70A368EB70E37B2B71E3896B71E36892
:2016E0001B0AAB71E368EB71E37C2B72638A6B7223691B0AAB722369EB72E37D2B73E38A1A
:201700006B7363691B0AAB736369EB73E37E2B74638B6B74A3691B0AAB74A369EB74E37FC8
:201720002B75E38B6B75E3691B0AAB75E369EB7594F823302B76638C6B76236A1B0AAB765B
:20174000236AEB7694F827302B77E38C6B77636A1B0AAB77636AEB7703B0F0BD9804001076
:2017600030B504460D469DB001A8FFF75DFE01A8FFF768FE2146074C2A4601A8FFF764FF6F
:20178000214601A8FFF764FF01A8FFF751FE20461DB030BDC007001010B5A8B90B4C2378E3
:2017A000DBB2012B02D02078C0B210BD0849094A09481160237003F05DF80028F3D0237800
:2017C00003F0FE032370EEE7012010BD840400101CBB0010D804001000000C4070B50028BB
:2017E0005AD12E4B1B78D80754D40E2954D8DFE801F0081D23295353535353532C323D533F
:201800004700274B274E1D6801F05AF900F1320401F056F9A04201D3012070BD2946304681
:2018200002F09CFFC305F3D5002070BD1C4B1B68D3F844321360F7E7194B1B68D3F83C32A2
:201840001380F1E74FF48053F4E7154B1B68D3F830321370E8E7124B1B68196A1160596A33
:201860005160996A9160DB6AD360DDE70C4B1B68196911605969516099699160DB69F3E736
:20188000074B0848196802F073FF0028CCBF0020012070BD032070BD042070BD8404001067
:2018A000D804001000000C4007B590B98BB10B480078C0070FD4009313460A46084909485C
:2018C000096803F06BF9B0FA80F0400903B05DF804FB0420FAE70320F8E700BF8404001078
:2018E000D804001000000C4018B9034B1878C0B270470120704700BF8404001007B590B9A4
:201900008BB10B480078C0070FD4009313460A4608490948096803F0FDF9B0FA80F040097B
:2019200003B05DF804FB0420FAE70320F8E700BF84040010D804001000000C4001380A4483
:20194000914200D1704711F8013B00F8013FF7E7026810B552B111460B4611F8014B202C56
:201960000CD93A2CF8D1511C8B4202D04FF0FF3010BD1278302AF9D101330360002010BDDA
:2019800008B568B103685BB11A784AB1D9888288914205D15878FFF7A7FF10F0010000D01C
:2019A000092008BDCA7E8B7E032843EA022301BF487D0A7D42EA002243EA0243184670478A
:2019C000F8B5C56A00F13007044601232A4639464078FFF793FFA0B9236AA269EB1A93429B
:2019E000207101D30020F8BDE678012EFAD9A36939461D442A4601236078FFF77FFF013E42
:201A0000F3E70120F8BD03790BB1FFF7D9BF18467047C36A70B58B4206460D4612D0FFF7A5
:201A2000F2FF044660B92A46012306F130017078FFF73AFF00281CBF4FF0FF350124F5628D
:201A4000204670BD0024FBE7002310B503714FF0FF33C3620446FFF7DCFFC0B994F82F228A
:201A600094F82E3243EA02234AF65522934210D1D4F86630084A23F07F4393420AD0D4F8B7
:201A8000820020F07F40801A18BF012010BD032010BD022010BD00BF464154000023F0B555
:201AA000036085B0074608461546FFF751FF061EC0F20781864B53F82640002C00F00381D2
:201AC0003C6023786BB16078FFF70EFFC70708D4002D00F0D38010F0040000D00A2005B00B
:201AE000F0BD0023F0B223706070FFF755FEC10700F1EB800DB14207F0D400212046FFF75C
:201B0000A3FF012840F0C580002204F5FB7111F8043C03B10B684DF822300132042A01F1A4
:201B20001001F4D100265DF82650002D00F0A88029462046FFF788FF002840F0A28094F841
:201B40003C2094F83B3043EA0223B3F5007F40F0A38094F8473094F8461094F8400051EA7A
:201B6000032108BF616D431E012BA161E07000F2938094F83D60A670002E00F08D80731ECD
:201B8000334240F0898094F8423094F8417047EA03273B0727817FD194F8442094F84330D8
:201BA00094F83FE053EA022394F83E2008BF236D52EA0E2270D001FB00FE02EB1710704469
:201BC000834269D31B1AB3FBF6F3002B64D040F6F576B34264D94FF6F576B34294BF0226E6
:201BE000032602332A442844032E6361E5612262A06257D1002F4FD1E26D9B00626203F2D2
:201C0000FF13B1EB532F47D34FF0FF332361E3608023032E63712AD194F8612094F8603076
:201C200043EA0223012B22D1691C2046FFF7F1FEE8B994F82F2294F82E32607143EA0223D6
:201C40004AF65522934212D1226B224B9A420ED103F1FF53D4F8142203F5005320339A429E
:201C600001BFD4F818322361D4F81C32E3601A4A2670138801339BB21380E38000202EE76C
:201C800002200136042E7FF44EAF032804D1012025E70328FBD008B10D2020E705464EE7B9
:201CA00001269EE7002FF7D07244022E62624FEA43021BBFD21803F00103134603EB520303
:201CC0009DE70B200BE70C2009E7032007E700BFDC04001052526141E004001010B504463E
:201CE000FFF791FE002851D12378032B46D16379012B43D104F130010B4604F50C72934256
:201D000045D1552384F82E32AA2384F82F32522384F8303084F8313061234122722084F88C
:201D2000323084F81732236984F8332084F81622C3F3072284F8183284F819221A0C1B0EC2
:201D400084F81B32E36884F81A22C3F3072284F81D221A0C84F81E22E26984F81C320132F3
:201D60001B0E84F8140284F8150284F81F32E26201236078FFF7C2FD002363710022607862
:201D80001146FFF72BFD003018BF012010BD03F8010BB4E743690239023B99423DBF837841
:201DA000806A01FB0300002070470129F8B506460D465DD9436999425AD20378022B29D063
:201DC000032B39D0012B53D101EB5104016A01EB5421FFF71EFE10B14FF0FF30F8BD316ADE
:201DE000671CC4F30804344401EB5721304694F83040FFF70EFE0028EED1C7F308073E441B
:201E000096F83000EB0744EA00204CBF0009C0F30B00F8BD016A01EB1521FFF7FAFD00289B
:201E2000DAD16D0005F4FF75354495F8313095F8300040EA0320F8BD016A01EBD511FFF7C4
:201E4000E8FD0028C8D1AD0005F4FE7505F1300333449878DA783544000440EA026095F82B
:201E600030205B78104340EA032020F07040F8BD0120F8BD70B5044682680D46012AE1801C
:201E800001D1022070BD036859698A42F9D2BAB91978032901D1596A99B919898D42F0D213
:201EA000586AE2600028ECD0236800EB1510303305F00F0503EB451520616561002070BD57
:201EC00011460A469E783601B5421146206802D2FFF760FFE5E7FFF768FF431C024607D068
:201EE0000128CED923685B699842CAD2AD1BEBE7012070BD10B5C1880446FFF7BBFF80B924
:201F000021692068FFF785FD58B90146636903F120029A4206D1E52263691A70012223683F
:201F20001A7110BD03F8011BF3E701292DE9F04105460C46164672D9436999426FD2037860
:201F4000022B3ED0032B4DD0012B68D101EB5107016A01EB5721FFF75CFD002860D107F1E3
:201F60000108C7F3080714F001042F4417BF97F83030F3B203F00F0233011CBF03F0F003B0
:201F8000134387F830300123296A2B7101EB58212846FFF73EFD002842D1C8F308032B4445
:201FA0003CB1C6F3071283F8302001232B71BDE8F08193F83020C6F3032622F00F0232436C
:201FC000F1E7016A01EB1421FFF723FD40BB640004F4FF742C44C6F3072284F8306084F8E3
:201FE0003120E2E7016A01EBD411FFF712FDB8B9A40004F4FE7404F130012944CB782C44C1
:202000001B0603F0704343EA0602C2F3072384F830204B70130C120E8B70CA70C5E702201C
:20202000BDE8F081F8B505460F4671B9C668E6B143699E4228BF012634466B6901349C4253
:2020400016D3012E13D8002408E0FFF7AEFE0128044635D9013003D14FF0FF342046F8BDBC
:202060006B699C42FAD33E46E6E70126E4E7022421462846FFF799FE30B1411CECD00128F3
:202080001ED0B442D9D1DEE76FF0704221462846FFF74BFF90B957B92B69EC605A1CDDD06B
:2020A000013B2B616B7943F001036B71D6E7224639462846FFF739FF0028EDD00128CBD078
:2020C0000124CBE72DE9F843C68804460136B3B2894613B90420BDE8F8830369002BF9D065
:2020E00016F00F0807D1C16801330361006859B903899E42EED22368E680303303EB4813E7
:2021000063610020BDE8F8838778013F17EA1617F1D1FFF74AFE0128054602D80220BDE839
:20212000F883421C02D10120BDE8F883206843699D4226D3B9F1000FCCD0E168FFF772FFA1
:202140000546002833D00128E8D0431CEBD02068FFF759FC0028E6D1236803F50C723033F8
:20216000934215D1226829461046FFF713FE4FF00109D062206883789F420CD3C36ADF1B69
:20218000C762E56029462068FFF704FE2061B2E703F8010BE4E780F80490FFF711FC0028BF
:2021A000C1D122680137D36A0133D362E2E70720BDE8F8832DE9F8430B7804462F2B0D464A
:2021C00001D05C2B00D101350026A6602B781F2B2FD920262B78AC462F2B05F10105F9D085
:2021E0005C2BF7D0A7693B4607F10B02934227D14FF000084FF0080E454643460CF1FF3949
:2022000019F8012F0135202A24D92F2A22D05C2A20D02E2A78D0C64508D9100606D4464835
:2022200010F8011F002978D08A42F9D10620BDE8F88331462046FFF71DFE6661BDE8F88354
:2022400003F8016BD2E743F0020307F8082008F10108D5E7212A654434BF04220022B8F169
:20226000000FE3D039782046E52904BF05213970BEF1080F04BF9B00DBB203F00301012913
:2022800003F00C0308BF42F01002042B08BF42F00802FA720021FFF7EDFDD8B921692068EF
:2022A000FFF7B7FBB0B96269137893B1D37A19070AD4A36903F10B0E9E450BD012F8017BCB
:2022C00013F8011B8F42F7D000212046FFF7FAFEE3E70420A369DB7A38B104282AD113F068
:2022E000040F08BF0520BDE8F8835A0722D46169CB7ADB0605D523681878FFF753FBA0603F
:2023000068E70520BDE8F883BEF1080F8ED19B00F046DBB24FF00B0E72E7A2F141011929DE
:2023200091D9A2F1610119299EBF203A43F00103D2B28AE7BDE8F8831B67000010B5044668
:202340000420216909B9A0B11BE02068FFF761FBB8B962691378BBB1E52B0CD02E2B0AD095
:20236000D37A03F03F030F2B05D023F02003082B01D0002010BD00212046FFF7A3FE00285F
:20238000DFD00023236110BD0420FAE738B500210546FFF76FFD044648BB29692868FFF7F5
:2023A00038FB044618BB6B691B78E52B15D129692868FFF72EFB044668B901466B6903F1B5
:2023C00020029A4210D10B22A9696869FFF7B6FA01222B681A71204638BD002BE7D00121C8
:2023E0002846FFF76FFED6E703F8011BE9E7042C08BF0724EFE7012970B504460D4601D8AB
:20240000022070BD43699942FAD263699D4205D229462046FFF7C9FC064608B9002070BDAE
:202420000128EDD0411C10D0002229462046FFF77CFD58B923695A1C05D001332361637997
:2024400043F0010363713546DFE7012070BDFFFF1FB5019004A840F8041D00911446FFF799
:2024600077FA011E15DB0D4B53F8210008B100220270019808B10022027043F8210030B1A8
:20248000012C08D10022694601A8FFF707FB04B010BD0B20FBE70020F9E700BFDC04001087
:2024A0002DE9F0438DB0019114460646002800F08280002302F01E02036001A905A8FFF75F
:2024C000EDFA002845D102AB019905A80B93FFF771FE0A9D10B9002D08BF062014F01C0F27
:2024E00004F01F0740D0B8B3042832D105A8FFF74DFF70BB0A9D47F008073C073DD5262373
:2025000000242B744B23DDF81480AC73EC736B74EC722C776C77AC77EC7798F8000029465B
:20252000FFF740FA0123AC76EC762C756C7588F80430044608B301464046D8F82C90FFF739
:202540005AFF30B90598013CC4604946FFF761FA98B10DB0BDE8F083EB7A13F0110F2ED1B6
:202560006307CAD50820F4E70028F2D1EB7AD80623D4A10701D5DA0721D40024DDF8148049
:202580003B07D8F82C3048BF47F02007F3613562B771F47198F800002946FFF703FA30616D
:2025A000EB692046F360B8F80630B460B461C6F80080B380CDE70920CBE70420C9E7072004
:2025C000C7E72DE9F74F9B460023CBF80030044689461546FFF7D4F9064620BBE379002B15
:2025E00040F09480A379D80740F19280E368A768DF1BAF4228BF2F4604F12403009397B1C1
:20260000A268C2F30803002B71D120688378013B03EA522313F0FF0314D142B920690128CB
:202620000BD80226E671304603B0BDE8F08F61690193FFF7BAFB019BF1E7411C01D1012618
:20264000F0E76061D4F800A0616950460193FFF7A1FB0028E5D0019B7D0A00EB030829D001
:202660009AF802205919914288BFD51A2B46424649469AF80100FFF717F90028DFD1A37916
:202680005A060BD5A069A0EB0800854206D94FF40072009909EB4020FFF750F96D02A3685D
:2026A000A9442B44A360DBF800307F1B2B44CBF80030A4E7A269904517D0A3795B060BD50D
:2026C000012300999AF80100FFF718F90028B6D1A37923F04003A3712068012342460099A1
:2026E0004078FFF7E1F80028A9D1C4F81880A1684846C1F30801C1F50075BD4228BF3D4675
:2027000024312A462144FFF719F9C8E71E468AE7072688E710B50446FFF732F9002842D1FC
:20272000A3799A063FD55B060CD520680123A26904F124014078FFF7E1F898BBA37923F0AD
:202740004003A371E1692068FFF763F9014650BB236ADA7A42F02002DA72E2681A77A28925
:20276000120A5A77E2899A77E27BDA77226999759A76C2F30720120C1A75120A5A752622DD
:202780001A764B22D876D9755A769974D974A379206823F02003A37101230371BDE81040FB
:2027A000FFF79CBA012010BD10B50446FFF7B2FF20B92046FFF7E4F800B9206010BDF8B565
:2027C00004460D46FFF7DCF8064600286CD1E379002B40F08D80E368AB4204D2A27912F0F2
:2027E000020F08BF1D460022A368A260002D2FD1A368E268934257D9E360A37943F0200333
:20280000A37151E00025A368C3F30803002BEFD0A2699542ECD0A37904F1240713F0400F6C
:202820000BD02068012339464078FFF767F800283ED1A37923F04003A371206801232A46AC
:2028400039464078FFF730F8002831D1A561CFE7206887787F02F3B1013B6A1EB2FBF7F237
:20286000B3FBF7F18A4216D37A4213406169A360ED1A0029C6D0BD421FD8A3682B44A360F8
:20288000C5F30803002BBDD02068FFF783FA48B100EB5525B7E7216969B9FFF7C3FB01283D
:2028A000014603D10226E6713046F8BD013001D10126F8E721616161DBE7A37920689A07FF
:2028C00005D5FFF7AFFB014620B93D46D5E7FFF76CFA01464B1CEBD00129E3D923685B6925
:2028E0009942DFD2A36861613B44A360ED1BC2E71E46D9E730B595B014A941F84C0D01228C
:2029000006A8FFF7CBF860B903AB019906A80C93FFF750FC28B90B9961B1CD7AEA070BD5B1
:20292000072015B030BD21460698FFF764FD0028F7D123E00620F4E7069B1878FFF732F81D
:202940000446A0B1EB0612D506A90DA81C22FEF7F5FF02210DA80F94FFF78CFA0028E0D1A9
:202960000DA8FFF7EBFC0028DAD00428D9D106A8FFF7C0FA0028D4D1002CD4D10698FFF78D
:20298000ADF9CEE7034B19681A68521A8242FBD3704700BFE8B800104FF08062054B0649A7
:2029A000C3F880210860002104480160044801701A60704700E100E0E4040010EC040010DE
:2029C000E8040010044A1368002BFCD0034B1878B0FA80F040097047EC040010E804001047
:2029E000FFF7D0BF7047FFFF01220A4B10B59A601122094CDA60204602F0BCFA20464FF4ED
:202A0000E13102F00DFB03232046E360BDE8104002F09CBA00C0024000C00040044B1A46ED
:202A200059698906FCD5186053699B06FCD5704700C0004010B5441E14F8010F00B910BD4E
:202A4000FFF7ECFFF8E7FFFF024A136801331360704700BFE8B8001008B5084B08481B6841
:202A6000197801F02DFB0122064B1870064B1A604FF08062054BC3F8802008BDE40400105C
:202A800000000820E8040010EC04001000E100E013B500240748009423462246214601F059
:202AA00003FEA04204DA0122034B1C70034B1A6002B010BD00000C40E8040010EC040010C9
:202AC000014B1868704700BFE8B8001008B505494FF4004001F08AF9034B1B681B1A584262
:202AE000584108BDFCDF0100F0FF070030B51D4DADF50B7D2A78012A05D0022A0DD01A4820
:202B0000FFF798FF04E0194901A8FFF7C9FC38B1002420460DF50B7D30BD01221449F3E73A
:202B2000002101A8FFF74BFE0028F1D16B46049A104901A8FFF745FD0028E9D1049A009BFE
:202B40009A42E5D100F0E0FE04460028E0D001A8FFF72AFE2B78012BDBD10448FFF7CAFEA7
:202B6000D7E700BF85040010BE020000EF020000E30200000000008000B51A4BADF50B7DE5
:202B80001A78012A05D0022A0DD01748FFF752FF04E0164901A8FFF783FC38B100200DF588
:202BA0000B7D5DF804FB01221149F3E7049BB3F5E04F01D00F48E9E7002101A8FFF7FFFDB8
:202BC0000028EBD16B46049A0B4901A8FFF7F9FC0028E3D1049A009B9A42DFD103F020FC2A
:202BE000DDE700BF85040010BE020000D7020000CB020000AE0200000000008030B5012419
:202C0000ADF50B7D2A4D22462A4901A82C70FFF747FC78B12246284901A8FFF741FC38B1F3
:202C20002648FFF707FF002420460DF50B7D30BD02232B70049BB3F5F02F09D02048FFF7CC
:202C4000F9FE01A8FFF7B0FD1A48FFF753FEEAE7002101A8FFF7B3FD0028E4D16B46049A1B
:202C6000184901A8FFF7ADFC0028DCD1049A009B9A42D8D11448FFF7DDFE04980009FDF752
:202C8000F5FB044648B11148FFF7D4FE01A8FFF78BFD0F48FFF7CEFEC6E70E48FFF7CAFEDF
:202CA00001A8FFF781FD0348FFF724FEBCE700BF85040010EF020000E3020000970200002A
:202CC000AE020000000000808202000074020000520200006502000070B50125ADF50A7D9B
:202CE0001B4E2A461B4901A83570FFF7D9FB1A4C70B12A46194901A8FFF7D2FB30B14FF09A
:202D0000FF33236000200DF50A7D70BD022333702268134B01A89A4212D14FF0FF32114B44
:202D20002260D3F88011C3F88021CB0608D5FFF73BFD0848FFF7DEFD0B48FFF77BFEE1E7D2
:202D4000FFF732FD0948FFF775FE0120DBE700BF85040010D702000000D00010CB020000D3
:202D600081EC9C4A00C00F403B0200002802000048F2040310B51C68FFF7A8FEA0B91648AD
:202D8000FFF758FE1548FFF755FE1548FDF7DAFBBFF34F8F1349144BCA6802F4E062134310
:202DA000CB60BFF34F8FFEE71048FFF743FE104802F014F94FF0FF320E4B0721C3F8CC21F4
:202DC0000022C3F8CC21C3F8D011C3F8D02172B6BFF34F8FA047FEE7100200000502000044
:202DE000E093040000ED00E00400FA05EB01000000C0004000C00F4070B505460C46164673
:202E000086B01946102202A803F096FA0A9B32460093294602AB204600F080FB10220021CE
:202E200002A803F08BFA00F0D9FB06B070BDFFFF10B586B00DF107024FF4F021234800F01A
:202E40001DFC04460A2202A903F07CFA2048FFF7F1FD002C11DA611C03D11E48FFF7EAFDD8
:202E60002FE0A21C01D11C48F8E7E31C01D11B48F4E7043425D11A48F0E71A48FFF7DAFDCB
:202E800002A8FFF7D7FD1848FFF7D4FD9DF807300BB91648E2E71648FFF7CCFDB4F5F02FFB
:202EA0000AD14FF4F040FDF7E1FA0028F1D000F02BFD30B1FFF75CFFB4F5E04F03D103F023
:202EC000AFFA06B010BD0B48C8E700BF0000008053680000D1010000BF010000A301000094
:202EE0002D6700003C6700005A6700006502000082020000AE020000F0B5A1B000F05CFEFF
:202F000000F09CFDFFF770FD4FF47A725D4B1B68B3FBF2F3013BB3F1807F80F0A380F8214D
:202F2000594A5360594B83F823100023936007231360FEF735FA28B15548FFF77BFD554891
:202F4000FFF778FD544C00F08FFA544821684569013169406368216081699A1C4A40A368BE
:202F60006260C269033353404FF480512046A360FEF7F6FB202103F04FFA224604F50071E9
:202F8000402003F051FA46F6B0710020FEF7E8FB46F6B071FEF72EFA10B94148FFF74AFD35
:202FA000FFF746FF0A226946912003F0CBF93D48FFF740FD3C48FFF73DFD6846FFF73AFD4C
:202FC0003A48FFF737FD3A4B3A4A1968914208D1002239481A60FFF72DFD47F23050FDF725
:202FE000B1FA364B5B695B0509D43548FFF722FD3148FFF71FFD47F23050FDF7A3FA314CC0
:20300000314801F021F84FF416720021204603F095F92E4B2E4EC4F84C322E4B2E4FC4F879
:2030200050322E4B2E4DC4F8543200F013FD2D4801F0A8F94FF000520A242B4B1A600122FF
:2030400031463846FFF704FA03280CD12846013CFFF7F0FC14F0FF04F1D12448FFF7EAFCE1
:20306000FFF786FEFEE70028F7D1FFF735FE08B1FFF782FDFFF7C2FD0028F1D0FFF736FDE3
:20308000EEE700BF74CE001010E000E000ED00E0306800001B68000004D00010004002402C
:2030A0006502000053680000636700009C010000F07F0020EFCDABAB0502000040800920F6
:2030C000786700001CBB0010000008209929000065680000C5290000ECB800108529000023
:2030E0002B67000000000C4000E100E08E670000024A034B1A6000F04FBD00BF000000006D
:2031000008ED00E02DE9F047334B344A1B6882B003F1100019780433117013F8031C04322F
:2031200002F8031C13F8021C02F8021C13F8011C834202F8011CEDD10425294A294FDFF888
:20314000A8E002AE114601AB11F8010B03F8010BB342F9D1AB0723D09DF804409DF8050041
:203160009DF806109DF8073012F80CAC12F80B9C12F80A8C12F809CC013584EA0A0480EACA
:20318000090081EA080183EA0C032C2D147150719171D37102F10402D4D102B0BDE8F087E5
:2031A0009DF805409DF804309DF807109DF806004FEA950C3C5D1EF80CC0FB5C795C385C10
:2031C00084EA0C048DF804408DF807308DF806108DF80500C8E700BFF4040010F804001045
:2031E00004050010A806001058680000F0B40E4B1B68587B5E7A5C7859799A7A9F789D7926
:203200005E7358709E7BD8785C715972DC79D97B9A70DA7A9F729E719D73DC70D873D972FB
:20322000DA71F0BC704700BFA80700102DE9F04F874B87B01B68874C0293059303F1100578
:203240001A4621461E1D11F8013B1078434002F8013BB242F7D1AA4204F104041346EFD128
:203260007D4BDFF800920393029B7C4C043301920493FFF7BBFF029D0499002315F8232062
:2032800019F8022005F823200133042BF6D10135A942F2D1039F0299DDF804E038460E1D0E
:2032A00010F8013B0A78534001F8013B8E42F7D1B64507F10407F1D1029E777896F800E02B
:2032C000B178F07814F80E8087EA010314F807C0625C434014F808A088EA0303A25C14F804
:2032E0000C808CEA030314F800C08AEA030314F80AA014F8088014F80CC0534083EA0A0351
:20330000A25C14F80CC083EA0803534083EA0C03337014F8078014F80EA08EEA010314F8D8
:2033200001C0225C434014F80AA088EA030314F80880A25C8CEA030314F80AA014F80CC001
:2033400088EA0303534014F8088014F80CC083EA0A03A25C83EA080383EA0C035340737014
:2033600014F80E208EEA070314F802A014F801C083EA000214F8008014F807B08CEA0202DE
:2033800014F80BB014F80CC088EA02028AEA020214F80AA014F8088014F80BB08CEA020215
:2033A00082EA0A0214F80CC014F8088082EA0B0B8BEA0C0B8BEA080B86F802B014F80EE069
:2033C000E75D225C4B40E05D615C14F80E708EEA03035340A25C4340E75D615C5340205C7A
:2033E000615C7B40A25C43404B405340F370019B0436B3427FF461AF039B194A103B9A42DD
:2034000003937FF436AFFFF7F1FE029A002312F8231019F8011002F823100133042BF6D164
:2034200001329542F2D1059B019E039D29461C1D11F8012B1878424003F8012B9C42F7D124
:20344000A64205F104052346F0D107B0BDE8F08FA8070010980500108805001074CD001026
:20346000F8040010A80500100022F0B5284CD1B2CB095800034403EBC30383EA4103A354F6
:203480000132B2F5807FF2D1012302261946214873405BB2DAB283EA82035BB2DAB283EA38
:2034A00002134CB2002C5BB2ACBF00251B25002BACBF002209225340DBB25E0083F06307B2
:2034C00046EAD3124FEA931E7A4084EA41014EEA830E5F0982EA0E0247EAC3071C09C9B23B
:2034E00069407A4044EA0314624001294254CFD1632500232A460749074C057001E011F805
:20350000012FA3540133B3F5807FF8D1F0BD00BF74CD0010A8060010A80500102DE9F84F4B
:20352000174606461C46DFF8AC8010220D46DDF8289007F00F0A02F0FFFEC8F800601CB17F
:20354000234B1C60FFF7DEFDDFF88CB0B9F1000F01D0CBF800903446F7B129461022204697
:2035600002F0EAFEC8F80040FFF760FEDBF80010631E013904F10F0E5A7811F8010F424000
:2035800003F8012F7345F7D11034A31B9F42CBF8005005F11005E0D8BAF1000F0FD02946BF
:2035A0001022204602F0C8FECAF1100204EB0A00002102F0C3FEC8F80040FFF737FEDBF823
:2035C00000104846BDE8F84F102202F0B5BE00BFF4040010A8070010F0040010B02200214D
:2035E000014802F0ABBE00BFF804001037B504460B4D6B690193019BDB0709D4013C0120AD
:20360000A4B2FFF7BFF9002CF3D16FF0010005E0044A1368013313602868C0B203B030BD5F
:2036200000C00040AC07001013B5074C226801921E20FFF7DBFF002804DB2368019A9B1A9F
:203640001E2BF5D902B010BDE8B8001010B5002341F221040144884201D1184610BD10F8D0
:20366000012B83EA0223082213F4004F4FEA430318BF6340013A9BB2F6D1ECE72DE9F04F9C
:2036800000269C4BADF6440D1B68059006910492994910220AA8039302F04EFE022000F038
:2036A0008FFB4FF0190B34464FF001084FF043093546DFF850A20227B9F1000F02D048464A
:2036C000FFF7ACF9C820FFF791FF02282ED00FDC012800F0C180874B1A68039BD21AB2F5EF
:2036E000FA6F10D96FF00300AAE04FF01509E2E7042800F09F801828EDD16420FFF776FF3E
:20370000182800F0A180013FD6D1B9F1430FECD0FFF78AFF1820FFF781F91820FFF77EF9ED
:203720001820FFF77BF96FF0010089E04FF48067704A039B1268D21AB2F5FA6FD2D8B9F1D2
:20374000430F0DF5876989F8000008BF012500204946FA1C002D0CBF964602F1010E704567
:2037600000F101037AD399F8022099F80130D243D2B2934240F0B980984504D008F1FF32E0
:20378000934240F0B280B946002D73D00DF23B423946104608930792FFF758FF079A089B6D
:2037A000D15D0DF23C42D25D02EB012292B2904240F09B804F4A98451268039227D1069BA0
:2037C0001B1B9F4201D39946DBB1059B4A460DF23B41181902F0B0FD0AAB00934A464FF4FD
:2037E000E0430EA90DF23B40FFF706FB41F6FC3B41F6FB3C002706EBA90E0EAB764549D145
:203800004C444FF01A0B08F101085FFA88F80BF1FF3BBBF1000F62DCFFF706FF1820FFF781
:20382000FDF81820FFF7FAF81820FFF7F7F86FF0020005E0FFF7F8FE0620FFF7EFF82046BB
:203840000DF6440DBDE8F08FFFF7EEFE0620FFF7E5F84FF0FF30F3E7802769E70A20099112
:2038600008920793FFF7C2FE079B0999089AC85418466FE729462A460DF587601044C07854
:20388000013201449742C9B2F6DC0DF23B42D25D8A428DE7664501D81A680BE05E450ED12C
:2038A000DAF808501A68AA420CBF01213946084604990870CAF80820043301369EE70F4A6B
:2038C0009642E9D90E4A9642F6D11A68DAF808500499AA420CBF01223A460A70ECE7062041
:2038E000FFF79CF84FF00009E5E6FFF79DFE1520F6E700BFE8B800100C010000FBDF010031
:20390000FCDF010000000920F0B5294887B0FFF791F872B61D21082002F076FD1D2108207D
:2039200002F076FD62B602AE10222249304602F003FD4FF40044204F204D2148FFF77AF821
:2039400020494FF480522144384602F0F5FC294600964FF4E0434FF480523846FFF74CFAE9
:203960004FF6FE739C4285BFA4F58031C90B210B103172B6084602F047FD4FF480522946B4
:20398000204602F055FD62B604F58054B4F5002FD3D10D48FFF74EF84FF4F02200210B48C2
:2039A00002F0CCFC0A48FFF745F8012007B0F0BD9E6700000C010000E8180010E8A8001081
:2039C0002B6700000080FF7F6368000000000080BF67000070B5104B104D114CAB61114847
:2039E0004FF04063A36110494FF40073836100238B610E4E0E4B4FF4C002DA612E600D4D02
:203A000025600D4C04604FF4706008601A600F229A631A6270BD00BF400863000080092085
:203A200020800920408009206080092061086300808009200000FC3FF0FBFF0708B50F20BE
:203A400000F016F90F2000F013F9BDE80840FFF7C1BFFFFF084B0222C3F88820C3F88C209A
:203A6000C3F89420C3F89820C3F89C20C3F8AC20C3F8B020704700BF00C002400128104AE0
:203A8000104B0BD1506790671222C3F8F42FD3F8F82F02F01202122AF9D170470121D16720
:203AA000032191631A22C3F8F42FD3F8F82F02F01A021A2AF9D1034B0322C3F810217047B0
:203AC00000C0024000C008200A4A08B50323C2F8B0311368C3F30B0343F48043136001F08D
:203AE000FBF9022000F050F9BDE80840012000F03FB900BF00C00F4008B50B2000F0B8F82B
:203B0000202001F0D5F9104B3122C3F880210021C3F88421C3F88821C3F88C21C3F89021E3
:203B2000C3F89421C3F89821C3F89C2101F180000131132943F82020F8D124220349024829
:203B4000BDE8084000F072BB00C002408C68000010B50E4C4FF00733C4F8DC310B2001F0E8
:203B6000A7F900220120114600F0B0F9D4F80031DB0754BF0648074800F094F9D4F8A031C9
:203B800043F00103C4F8A03110BD00BF00C00F406C6800001C69000008B5FFF7ADFFFFF718
:203BA00093FFFFF7D5FFFFF749FF00F005F8BDE8084000F009B8FFFF08B500F0CBF8014B26
:203BC000186008BD74CE001010B50B4C0122C4F808210321104600F036F8D4F8A8305B0596
:203BE000FBD540F20122044B1F20C3F80821BDE8104000F03DB800BF00C00F40400100F154
:203C0000804303F57C231846D3F880201143C3F88010AA23C0F88C305523C0F88C307047FE
:203C2000400100F1804303F57C231846D3F8802022EA0101C3F88010AA23C0F88C3055231D
:203C4000C0F88C307047400100F1804303F57C23184641EA4212C3F884200122C3F88020F3
:203C6000AA23C0F88C305523C0F88C307047FFFF04490122D1F8C43002FA00F00343C1F84A
:203C8000C430704700C00F4005490122D1F8C43002FA00F023EA0003C1F8C430704700BF1D
:203CA00000C00F40054B0128D3F804210CBF42F4807222F48072C3F80421704700C00F40EB
:203CC000024BD3F80401C0F30020704700C00F40044AD2F8043103F480731843C2F80401DD
:203CE000704700BF00C00F40064BD3F80C3113F0030305D0012B0ABF034B0020186870476E
:203D00000248704700C00F4068680000001BB70008B5074BD3F8880010F4807007D0D3F8F9
:203D20008420FFF7E1FF02F01F0202FB000008BD00C00F4008B5FFF7C3FF28B1012807D1D6
:203D4000BDE80840FFF7E4BFBDE80840FFF7CCBF002008BD08B5FFF7EDFF044BD3F804319C
:203D600003F01F03B0FBF3F008BD00BF00C00F40044AD2F8B43123F4407343EA0020C2F83F
:203D8000B401704700C00F40044AD2F8B43123F01F031843C2F8B401704700BF00C00F4027
:203DA00008B5064BD3F8A81111F01F0104D0FFF7C1FFB0FBF1F008BD084608BD00C00F4053
:203DC0000128094B06D0022808D136221A604FF0FF3207E015221A60002203E000221A6012
:203DE0004FF6FF725A6070470000092010B504460220FFF7E5FF054B21B154F8042B013991
:203E00009A60F9E7014B986810BD00BF00000920002902DA484200127047074BB0FBF3F08F
:203E200041434FF47A70B1FBF0F1FF31090A91428CBF881A0020704740420F0070B5164658
:203E40000C784B6800EB4414C4F800320D46012289683046FFF7DCFFC4F80402E968002217
:203E60003046FFF7D5FFC4F80802296901223046FFF7CEFFC4F80C02696901223046FFF723
:203E8000C7FFC4F81002A96902223046FFF7C0FFC4F81402E96901223046FFF7B9FFC4F806
:203EA000180270BD10B50446FFF754FF054B2146BDE81040D3F800210132B0FBF2F20248BF
:203EC000FFF7BCBF00C00F4000C00920002914BF4FF480730023002A0CBF1A4643F0010299
:203EE000034B003018BF01209A601860704700BF00C00920084A0F284FF00103D2F8C41110
:203F000085BF1038834083400B4398BF21EA0303C2F8C431C0B2704700C00F4030B545695F
:203F2000039C072D54D8DFE805F00415273D3D15273D42688368C2F30B02980442F00C4220
:203F400042F4103200F4E0105B05104303F46003184330BD4068A304C0F30B0003F4E013B9
:203F600040F004406405184304F460041303204303F4E043184326E040689A04C0F30B00B5
:203F800002F4E01240F008405B05104303F460030A03184302F4E042C903104301F460318F
:203FA000084330BD40689B04C0F30B0040F0004003F4E0130903184301F4E0416405084339
:203FC00004F460042043D20302F46032104330BD002030BDF0B5C7690C68012606FA04F50F
:203FE000FFB22F422DD1EDB285600D68640106FA05F5EDB205610519C5F808310663036B59
:20400000DB07FCD5CB682044C0F800310B69C0F8043149699DF81830C90201F460519B0170
:2040200003F4F86341F4404119439DF814305B0003F03E030B43C0F81031C0F80C21012067
:20404000F0BD0020F0BDFFFF10B504461D20FFF70FFE00231946FF22C4F8F031C4F8D0315C
:20406000C4F8B031C4F89031C4F87031C4F85031C4F83031C4F81031A2602261024A9954B4
:204080000133082BFBD110BDB007001000EB4112D2F8103123F00103C2F810310123426830
:2040A0008B40DBB2134218BF8360C268134218BF0361024B00225A54704700BFB007001085
:2040C00010B50124036804FA01F1C9B20B4002460BD0436811EA030002D09160204610BD13
:2040E000D3680B4001D0116110BD184610BDFFFF30B5049C9DF8145003980A604D614C6024
:20410000072D24D8DFE805F0040C131A1A0C131ACB600223DC4008618B604C60032030BDA7
:20412000CB600C4B53F8203001200B6130BD094A086152F823300220CB6030BD054A52F8BC
:204140002330CB6052F8203000200B6130BD4FF0FF3030BD3C6900002DE9F0431C468BB0E8
:204160009DF8483088460293139B16460193009413460A4604A90546FFF7BAFFB0F10009A3
:2041800001DA002030E019F0010F04D13046FFF7B1FE074601E000273E4619F0020F04D143
:2041A0002046FFF7A7FE814601E00024A14610481049835D005D0A5D0090895D04A8FFF7DE
:2041C000ADFE8DE880020246002304A92846FFF701FF0028D5D005EB4815D5F81031012078
:2041E00043F00103C5F810310BB0BDE8F08300BFBC690000DC69000070B50B4D00230124C9
:20420000C16904FA03F6314011F0FF0FDAB206D1595D21B904490120C854104670BD0133C9
:20422000082BEDD1002070BDB007001030B501EB820291420CD00B6811F8045BC3F31724A9
:2042400005F007035B0103EBD50340F82340F0E730BD82B000238DF807309DF807300F2BC7
:2042600004D89DF807300133DBB2F4E702B0704701F003010A430260FFF7EBBF436823F08F
:20428000FF0319434160FFF7E4BF01231AB142688B40134303E042688B4022EA03034360BF
:2042A000FFF7D7BF40F2FF7341F4806183638260C160FFF7CEBF40F2FF7383634FF0FF3351
:2042C00083600023C360FFF7C4BF036903F03F030B7043694B6083698B60C369CB60036A2E
:2042E0000B6170478B6843628A780B8893408362CA780B7913438A781201D2B213434A79E8
:2043000012B943F0010301E043F00903C362FFF7A0BF30B5002A15BF07220F220023082376
:20432000934208D851F8045B03F12004013340F82450DBB2F4E730BD10B5002A15BF0722E7
:204340000F2200230823934208D803F1200450F82440013341F8044BDBB2F4E710BD38B587
:204360000C460546FFF71CFD61004B1E1844B0FBF1F101B101392846BDE83840C9B2FFF7F6
:204380007DBFFFFF10B504461C20FFF771FC1C2000F08EFD636823F480736360FFF759FF98
:2043A00000222260FFF755FFFFF753FF6FF06043E2636362E260FFF74CFFE262FFF749FFB6
:2043C00040F2FF73A36302232360FFF742FF20460749FFF7C4FF636843F480736360FFF737
:2043E00038FF03232360BDE81040FFF732BF00BF801A060010F4807304D16FF005020A6006
:204400001846704720F4FF5020F01F0018B16FF006030B6000E00860012070472DE9F041F2
:204420000D4606461F4605F0C008FFF73BFF4FF48032736BB8F1000F03D1180601D5002414
:2044400019E05906FBD440F20521194061B1DB070FD505F03F04012CF1D0292CEFD00C3C2A
:2044600018BF4FF0FF3406E0013AE2D16FF0030401E04FF0FF343046FFF71DFFCCB9B8F1B0
:20448000000F02D10020BDE8F08130463946FFF71CFF05F03F00431E012BF3D905F01F0558
:2044A000092DEFD03B78181A18BF4FF0FF30BDE8F0812046BDE8F081F0B5074615466FF09F
:2044C000060387B000934FF0FF3313600E04142401AB32464D213846FFF7A0FF009038B9B5
:2044E00069460298FFF786FF029B00982B6001E0013CEDD107B0F0BD2DE9F04188B008ADC4
:20450000002345F81C3D2A4606460F46FFF7D4FF60BB019BC3F34323032B03D0042B08BF3E
:2045200000241FE06FF0060302934FEA0748142403AB424647213046FFF770FF029020B9B7
:2045400002A90498FFF756FF08B9013CF0D1029C6CB92A4639463046FFF7AEFF019BC3F3ED
:204560004323042B18BF6FF0040400E00446204608B0BDE8F08170B5064686B06FF00603FB
:2045800000930D04142401AB2A4677213046FFF745FF009060B969460298FFF72BFF38B1E0
:2045A000009848B9029B9B0606D46FF006030093013CE8D16FF0060006B070BD70B58DB2AD
:2045C00088B06FF0060301AA294606460293FFF773FF029028BB019BC3F34323042B01D1AA
:2045E000002024E0053B012B1BD8142403AB00224C213046FFF712FF0290A8B902A904980C
:20460000FFF7F8FE80B1029888B901AA29463046FFF752FF019BC3F34323042BE0D0072B02
:20462000DED06FF0040002E0013CDFD1029808B070BDFFFF2DE9F0411E46194F194B8046E0
:204640001546002908BF1F4686B04FF4005400214046FFF790FF00BB01AB3A4669214046BA
:20466000FFF7DCFE90B9029B002B0FDA2A6822B923F07F432B6010460FE022F07F41194033
:204680008A4208D1C3F38073337006E0013CDED16FF0060001E06FF0010006B0BDE8F081E5
:2046A0000080FF400080FF002DE9F0411F4640F23A23456B04462B409046069E33B140F28C
:2046C0003A2383634FF0FF30BDE8F081EA0506D54FF480728263C3631846BDE8F08115F48C
:2046E000806202D04FF4806326E0154B2B4023B3456B79B16B040DD5D8F8003013F03F0FBD
:20470000194408BF0122FFF704FED8F800302033C8F800307FB12B040DD53168204611F0D6
:204720003F0F18BF0022394408BF0122FFF704FE336820333360024BA3630120BDE8F081C8
:2047400000C40F0007B501AAB1F83412FFF7B4FE0198C0F3432003B05DF804FB07B501AA6B
:20476000B1F83412FFF7A8FE019803B05DF804FB2DE9F0430D468DB0B1F834120446914625
:20478000FFF7BAFE074600286BD140F22A730121E3633648FFF730FD0CAE40234FF0060878
:2047A00006F8280D014601220193CDF800804B462E48FFF7D1FC3046D5F84C3298470123F5
:2047C000ADF810308DF81530294B022204A920468DF8147006938DF812808DF81320FFF718
:2047E00081FD6FF00603B5F834720393202639462046FFF7C0FE0246039070B907AB4D21E7
:204800002046FFF70BFE039038B903A90898FFF7F1FD10B1039B4BB904E0013E16F0FF06EE
:20482000E5D103E0D5F85032984708B1002600E040269DF808100D48FFF728FC294620469B
:20484000FFF780FF052804D1B5F834122046FFF7B5FE29462046FFF775FF0428F9D1304634
:2048600000E000200DB0BDE8F08300BF00000820404B4C002DE9F0430546AF4B0026C1F838
:20488000383289B0C1F830620C46AC49FFF767FD324603212846FFF7EBFC334632464FF46E
:2048A00080712846FFF7BAFD0646002840F07181D4F8543264209847142703AB4FF4D5722E
:2048C00048212846FFF7AAFD30B9049BC3F30803B3F5D57F06D05AE1013FEED1831C00F080
:2048E0005681B0B9964B03AA0393D4F83032012143F00103C4F83032284602ABFFF79AFE06
:204900009DF80830002B3AD0D4F8303243F080430DE08B4B02AA029339460DF10703284678
:20492000FFF788FE30B9D4F8303243F00103C4F8303224E0871C20D0402203212846FFF70E
:2049400097FCD4F85432642098474FF40077DFF8F08103AB424641212846FFF75FFD38B9C4
:20496000049A002A04DA43461340434507D00EE1013FECD16FF006060BE1064609E11427A2
:2049800003AB0022C2212846FFF748FD40B9049BE361059BA361069B6361079B236101E0CF
:2049A000013FEDD1D4F83032D80719D50023A4F83432142703AB002243212846FFF72EFDDB
:2049C00058B9049BC3F30C02D10506D5520A032A03D11B0CA4F8343224E0013FEAD121E02C
:2049E0000123A4F8343208AF6FF0060347F8183D4FF0140803AB4FF4803243212846FFF718
:204A00000DFD029018B1B8F10108F3D105E039460498FFF7EFFC0028F5D000220321284639
:204A2000FFF726FCB4F8348214274FEA084803AB4246C9212846FFF7F1FC40B9049BE362EA
:204A4000059BA362069B6362079B236201E0013FEDD1236923B92669003618BF012698E0A2
:204A6000D4F83032374FD4F828E01F40354BCEF30341012202FA01F19F42C4F83C12636A01
:204A800003D11B0C13449B0210E0980FC3F3C23340EA8E000233C0F30B0002FA03F300FB4D
:204AA0000333B1F5007FC4BF490A4B43C4F84432D4F84432B4F834125B02C4F840322846D8
:204AC000FFF71AFD002864D121462846FFF73AFE04285ED118492846FFF741FCD4F83022EE
:204AE00012F0010230D001220B212846FFF7CDFB0DF120086FF00603B4F8349248F8183DA1
:204B0000202749462846FFF736FD029078B903AB022246212846FFF781FC029038B9414641
:204B20000498FFF767FC10B1029B8BB131E0013F17F0FF07E5D12CE0002D3101801A0600C7
:204B40000080FF00010000400B212846FFF79DFB0DF120086FF0060348F8183D202703AB55
:204B60004FF4007250212846FFF758FC029048B941460498FFF73EFC20B1029B002B3FF4A5
:204B80006AAF06E0013F17F0FF07E8D101E06FF00106304609B0BDE8F08300BF2DE9F04F6E
:204BA000B3F100088FB005460C46174601DA0020A9E0189B08EB0302D1F844329A42F6D8F8
:204BC000B1F83412FFF798FC0028F0D109238DF81A3002238DF81B3001238DF81D304B4BF7
:204BE000DDF860A08DF81C000893BAF1000F6CDD564640F22A737F2EEB634FF0010144486E
:204C0000A8BF7F26FFF7F8FA0DF13809730209F8280D0293019306230146012200933C48E3
:204C20003B46FFF799FAD4F84C32484698470EA921F8206D2846FFF755FBD4F830326FF015
:204C40000602012E05920CBF512252225B00C346039258BF4FEA482B4FF0200909AB5A465C
:204C600003992846FFF7DAFB059020B905A90A98FFF7C0FB20B909F1FF3919F0FF09EDD116
:204C8000059B2BBBD4F85032984708BB9DF810101F48FFF7FBF9012E05D0B4F83412284634
:204CA000FFF78CFC05E021462846FFF74BFD0528F3D021462846FFF745FD0428F9D1029BEE
:204CC000C6EB0A0A1F44B0448FE7189B58021AD19DF810100E48FFF7D9F9189B012B05DDB6
:204CE000B4F834122846FFF769FC05E021462846FFF728FD0528F3D021462846FFF722FD4A
:204D00000428F9D153E70FB0BDE8F08F404B4C00000008202DE9F04FB3F100088FB00546F6
:204D20000C46174601DA0020BBE0189B08EB0302D1F844329A42F6D8B1F83412FFF7DCFBDE
:204D40000028F0D109238DF81A3001238DF81D30554BDDF860A08DF81B008DF81C00089328
:204D6000BAF1000F40F3878056467F2EA8BF7F26D4F830326FF00602012E05920CBF58224A
:204D800059225B00C346039258BF4FEA482B4FF0200909AB5A4603992846FFF73FFB059051
:204DA00020B905A90A98FFF725FB20B909F1FF3919F0FF09EDD1059B002BB4D121462846B5
:204DC000FFF7C0FC0628F9D140F21A730121EB633648FFF711FA0DF1380905234FEA462B6A
:204DE00009F8280D01463A460093CDF804B001232E48FFF7B1F9D4F84C32484698470EA902
:204E000021F8206D2846FFF76DFAD4F85032984740B19DF810102548FFF738F9189B012BDB
:204E200033DC2CE09DF810102048FFF72FF9012E05D121462846FFF785FC062810D1B4F810
:204E400034122846FFF7BAFB21462846FFF77AFC062805D10120FDF7C3FDFDF7C3FDEEE750
:204E600021462846FFF76EFC0428F3D1C6EB0A0A5F44B04474E7189B580212D1C9E721464F
:204E80002846FFF75FFC062804D1B4F834122846FFF794FB21462846FFF754FC0428F9D15A
:204EA00041E70FB0BDE8F08F002D31010000082000F01F0240098000012300F180409340DE
:204EC00000F57C20C0F8CC31D0F8CC2122EA0303C0F8CC317047FFFF38B51B4BD3F8A0217C
:204EE00050065EBFD3F8A02142F02002C3F8A021D3F8A0215106FBD50020FEF7D3FE124BED
:204F0000D3F88830DA0503D501210020FEF788FE0D4C0125002210460921C4F80C51FEF76B
:204F200092FE00202946FEF769FE2846FEF7D0FED4F888305B05FBD50120FEF7B3FE024BFD
:204F40000222C3F8A82138BD00C00F40034B98420BBF01238023C3650363704700400A401D
:204F6000034B98424FF000030CBFC3650363704700400A40174B10B5984204460DD003F50D
:204F8000082398420BD003F58043984209D0124884420CBF0820032004E0042002E018206B
:204FA00000E01920FEF764FE0723A3602046FFF7D7FF084A002394426360E3602362E36405
:204FC0006365236504BF2361A3690323E3601023A36210BD0000014000400A4008B50246F0
:204FE000FFF7BEFF0C4B98420DD003F5082398420BD003F58043984209D0084882420CBFCB
:205000000820032004E0042002E0182000E01920BDE80840FEF738BE0000014000400A4067
:2050200038B50C460546FEF7BBFE2101B0FBF1F1EB68B0FBF1F043F08003EB60CBB22B60A1
:20504000C1F307236B60EB6823F08003EB6038BD034600F00F0040001B0648BF01307047E6
:20506000436810229A6019611A68D206FCD5704738B504461546FFF7F3FF20462946BDE809
:205080003840FFF7EDBF38B5044608461546FFF7DFFF010441F4A0612046FFF7E1FF204665
:2050A0002946BDE83840FFF7DBBF436830229A6019611A689206FCD5586970474FF40C7041
:2050C0007047FFFF044A0029D0F8C801034908BF4FF48072FFF7CCBF000101000005FE0045
:2050E000D0F8C83100225B689A64D0F8A021D179D96401219964D279DA641A68D205FCD52A
:205100004FF0FF329A635A639A600C225A6070470346B3F89E31D0F8C8019B0703D50249B3
:20512000024AFFF7A5BF70470005FE00000101007047FFFF70B50904D0F8C861084D41F4AB
:20514000000444F48074304629462246FFF790FF304629462246BDE87040FFF789BF00BFAE
:205160000005D00093682DE9F041B3F50C7F8046144633D3566806F110026260A3F1100290
:20518000A2606568AA0702D001356560F9E705F50772A3F50B736260A360636813F00307BC
:2051A00002D001336360F8E72846224600F05AFE39461022304601F0C1F82368B56028464A
:2051C000C5F8C8617360FFF78BFF28463946FFF7B1FFC8F800503846BDE8F0810148BDE871
:2051E000F08100BF0A00040010B50A4AD0F8C841002908BF4FF4807220460749FFF738FF7F
:20520000636803225A641A68D205FCD54FF480729A6010BD000101000005D80038B50546A3
:2052200088780C46FFF714FF012102469140D5F8C8315B68586C014359649A64A288DA6424
:205240001A68D205FCD54FF480729A6038BD704710B504460846FFF7FBFE010441F4800142
:20526000D4F8C80141F4A0614FF48072BDE81040FFF7FEBE10B504460846FFF7E9FE010448
:2052800041F48001D4F8C80141F4A061024ABDE81040FFF7EDBE00BF0001200010B50446BC
:2052A0000846FFF7D5FE010441F48001D4F8C80141F4A0614FF48072BDE81040FFF7D8BE9B
:2052C00010B504460846FFF7C3FE010441F48001D4F8C80141F4A061024ABDE81040FFF7FD
:2052E000C7BE00BF0001010010B504460846FFF7AFFE010441F48001D4F8C80141F4A061E2
:205300004FF48072BDE81040FFF7B2BE043A38B51D46D0F8C8410D2A48D8DFE802F00E0E72
:20532000474747474747474744074A0A0122002041E04FF4007200203DE00846FFF788FE76
:20534000012303FA00F0236815B11843206002E023EA00002060226823682168DB071B4BBB
:2053600002F0020201EA030348BF42F004020BB142F020022168164B0B400BB142F0400292
:2053800023681449194009B142F0080223681249194009B142F01002120420460F4942F48F
:2053A0008072FFF765FE0022104604E000220C4801E00822002061684B6815B11A434A605C
:2053C00038BD23EA02024A6038BD00BF200882A01004415008822008044110040005F30077
:2053E00001000400D0F8C80101F00F032DE9F0419B00456843F00103AB622C6A2605FCD5AF
:2054000014F480681DD0C4F309085FEA980C25D016460023AF690133634546F8047BF9D10B
:2054200002EB830204F003045CB1AE691444002326FA03F502F8015BA24203F10803F7D147
:20544000456841F248230B410022DB07AA6202D4034AFFF718FE4046BDE8F0814446E3E786
:205460000005F20070470020704700207047FFF7B9BFFFFFD0F8C8012DE9F04101F00F0488
:205480004668A400DF1C44F00204BF08B4629846736206D0002452F8045B0134BC42F561C9
:2054A000F9D10023B362034AFFF7EDFD4046BDE8F08100BF0005FA002DE9F047D0F8C891F5
:2054C0008246D9F80420136823F004019160516801EA030818F0080461D118F0040F2BD080
:2054E000166B3EB3274605460121A140314219D00F43916313689806FCD5E30750693DD43F
:20550000002C00F09080AB6D63B1D9F80020114201D0C1066DD402225046D5F8D8109847C8
:20552000D9F804201F2C05D0B74204F1010405F10405D9D10423936018F4007F0FD0DAF864
:205540003C3063B148464049FFF78AFD3F494846FFF7ABFDDAF83C3001465046984718F081
:20556000010F09D0DAF834300BB150469847D9F80C300133C9F80C30BDE8F087AB6D002B3E
:20558000D0D0D9F80020114201D0C20629D403225046D5F8D8109847D9F80420C2E7484616
:2055A0002B49FFF75DFD48462A49FFF77EFDC606044626D4A50706D5DAF838301BB1504682
:2055C00004F00101984704F00903092BD4D1640724D5DAF82C30002BCED050469847BDE8A8
:2055E000F08705225046D5F8D8109847D9F8042098E704225046D5F8D8109847D9F804202A
:2056000090E75046FFF76CFD504600F015FBDAF82830002BCED050469847CBE7DAF830303C
:20562000002BDAD1A8E743077FF56DAFDAF85830002B3FF479AF01225046DAF8D8109847F9
:20564000D9F8042070E700BF0005FB000002FB000005FE000002FE0090F8143213F01F034C
:2056600005D100F29D12C0F8CC21184670470148704700BF010004007047704790F81432F9
:2056800003F01F03012B06D0022B15D0002B37D100F5CF720DE090F89D318BB390F8182235
:2056A00090F89B319A422BD20023A0F8D43100F5EA72C0F8CC2121E090F818321A064BBF0A
:2056C0004FF48031012103F00F0203F08F0201FA02F290F89D1109B91B0711D1D0F8B43194
:2056E0001A420DD0D0F8B8311A420CBF00230123A0F8D43100F5EA73C0F8CC3100207047D7
:20570000004870470100040010B590F8142212F01F0237D190F81732022B09D0032B19D0E9
:20572000012B2FD1D0F8A031C0F8CC31122321E0D0F8AC3190F816128A4205D01C780CB172
:205740005C8823440132F7E71A78DAB1C0F8CC315B880FE0D0F8A43190F81642A24204D014
:20576000197801B10B440132F8E71A7852B1C0F8CC311B78B0F8D0219A4288BFA0F8D03153
:20578000002010BD004810BD0100040090F8143203F01F03012B0FD190F89D3163B190F821
:2057A000183290F89B219A4206D903F5E0730344C0F8CC310020704700487047010004007E
:2057C000F8B590F81432044613F01F030D4602D0022B1BD04AE0B0F81632012B0ED1036C0E
:2057E00003B19847B4F89E312DB143F00203A4F89E310020F8BD23F00203F8E7022B35D11B
:2058000090F81912BDE8F840FFF72DBE90F818321A0603F08F0105D503F00F024FF48036CB
:20582000964001E001268E4094F89D21F2B11B071CD0D4F8B4311E4218D0B4F81672AFB92C
:2058400035B12046FFF73CFDD4F8B8311E430AE0D4F8BC311E42CCD12046FFF745FDD4F8AD
:20586000B83123EA0606C4F8B861C2E70048F8BD01000400F8B590F81472044617F01F0774
:2058800040F0BE8090F81632002B00F08480D0F8A851D0F8AC3190F89A21012A08BF1D46AD
:2058A0002B78002B00F0A2806B78042B4ED0052B4ED0022B6CD16A7994F81632934243D180
:2058C00084F89D312B7984F89B310023E21801330021082B82F8C011F8D1012694F899315C
:2058E0009E4217D20122B240D4F8B4311A4203D020463146FFF7BEFC4FF48032B240D4F8AA
:20590000B4311A4204D0204646F08001FFF7B2FC0136E3E74FF00113C4F8B4310023C4F8DD
:20592000B831C4F8BC3120460121FFF75DFCEB7913F0400FB4F89E3114BF43F0010323F0B0
:205940000103A4F89E3123E06B8822E0EF781FE0F7B9AB781A0603F08F0606D503F00F031F
:205960004FF4803202FA03F301E00123B340D4F8B42120461343C4F8B4312946FFF74EFC9B
:2059800020463146FFF764FC20463146FFF786FC2B781D4484E780F89D31012594F899314E
:2059A0009D4217D20122AA40D4F8B4311A4203D020462946FFF75EFC4FF48032AA40D4F862
:2059C000B4311A4204D0204645F08001FFF752FC0135E3E700214FF00113C4F8B431C4F881
:2059E000B811C4F8BC112046FFF7FEFB94F89D0194F81622034B904214BF18460020F8BDEC
:205A00000048F8BD010004002DE9F74F90F81432044603F01F03012B40F0918090F89D3138
:205A2000002B00F08C80D0F8AC31D0F8A85190F89A210026012A08BF1D46434BB246374618
:205A4000B1462A78002A78D06A78042A0AD0052A1CD0022A6ED1697994F89D21914269D093
:205A60006A8868E095F8029094F81822EF7891455DD194F81622974259D104EB090393F84F
:205A8000C0A183F8C07100231E4653E094F8182291454FD195F8028018F0800F08F08F0B4B
:205AA00006D008F00F084FF4803202FA08F803E04FF0010808FA0BF894F8162297421BD157
:205AC000D4F8B421204642EA0802C4F8B421D4F8B821294622EA0802C4F8B8210193FFF7AF
:205AE0009DFB20465946FFF7B3FB20465946FFF7D5FB46EA080618E057451BD118EA060FC5
:205B000017D1D4F8B4216FEA080802EA0802C4F8B421D4F8B821204602EA0802C4F8B82176
:205B200059460193FFF7A6FBBA46019B02E0002600E0BA462A78154483E7184600E002482A
:205B400003B0BDE8F08F00BF01000400002100F50572FFF78CBCB0F8D03110B5402B28BF1F
:205B600040238021D0F8CC210446FFF783FCD4F8CC310344C4F8CC31B4F8D031181AA4F869
:205B8000D00110BD10B50021D0F8CC210446FFF729FCD4F8CC310344C4F8CC31B4F8D031F1
:205BA000181AA4F8D00110BD002280211346FFF761BC002100F5EA72FFF714BC10B58021AC
:205BC0000446FFF77DFB0023A4F8D03110BDFFFF90F8143213F01F0307D190F8162262F0A5
:205BE0007F0280F89C21184670470148704700BF01000400F8B504460F460546002694F8CD
:205C000098319E4213D2D5F858316BB12046D5F878113A469847074B984205D0054638B134
:205C20002046FFF7CBFF03E001360435E7E7014D2846F8BD0200040001224FF00111A0F89A
:205C40009E210022C0F8B41180F89C2180F89D21C0F8B821C0F8BC210E21FFF7CBBFFFFFA8
:205C600010B50446FFF772FF94F814122046C909FFF7EDFAB4F81A322046A4F8D0310121CA
:205C8000FFF7B8FF374B98426AD194F81432C3F3411313B1022B50D05EE094F815320B2B8C
:205CA0005AD8DFE803F0060F5913591E272931333C3EE3682046984700284DD12046FFF7A0
:205CC0004AFF4CE0636A2046002102E0636A20460121984700283FD12046FFF765FFE36C9E
:205CE00027E02046FFF774FF002835D12046FFF75BFF34E02369DDE720460021FFF7E0FA2F
:205D00000023A4F8D0312AE06369D3E7A3692046984708BB2046FFF747FF636C09E0E36979
:205D2000C8E7236A20469847B0B92046FFF73CFFA36CA3B12046984711E0A36863B12046C4
:205D40000121984740B9B4F81A32002BCED094F81432DB0903D0B1E72046FFF72FFF0020BD
:205D600010BD00BF0200040038B590F814320446DB0923D1B0F8D03113B3FFF703FFB4F8A1
:205D8000D031EBB920460221FFF734FF0F4B984218D194F81432C3F34113022B0AD1A368A0
:205DA00043B1204601219847054618B92046FFF7FBFE08E02046FFF701FF01E0FFF7F9FE05
:205DC000002500E00546284638BD00BF02000400013A10B50446062A40D8DFE802F0041DDF
:205DE00021063F3A3C00036817E00421FFF702FF1B4B984232D194F814122046C90904D147
:205E0000D4F8CC21B4F8D03103E00021D4F8CC210B46FFF72AFB21E04368204698471DE005
:205E200090F81432DB0909D00321FFF7E3FE0C4B984213D12046FFF78EFE0FE090F89C11BB
:205E40000B060BD501F07F0180F89C11FFF772F904E0002100E08021FFF746FA002010BDB1
:205E60000200040070B515460E464FF407720021044600F063FA2A7B254B84F89921A36581
:205E8000C4F8D84012B1E365C4F8DC40214B224A2360224B6360224BE360224B6362224B71
:205EA0002361224B6361224BA361224BE361224B2362EB6B002B08BF134623651F4A2B6CF0
:205EC000002B08BF134663656B6A2364AB6AA3632B69A3626B69E362AB6923632B6A636391
:205EE000EB6AE3632B6B63646B6BA364AB6BE3643368C4F8A0317368C4F8A431B368C4F805
:205F0000A831F368C4F8AC313369C4F8B03170BDD15D0000615C000079560000695D0000CE
:205F20007D560000C15700000957000059560000755800008D570000095A00007B56000082
:205F400010B590F89831072B0AD800EB83040133C4F85811C4F8782180F89831002010BDC9
:205F6000004810BD0B00040010B590F89941B1EB440F06D800EB81008265C0F8D8300020D6
:205F800010BD014810BD00BF030001000378012B04D007D3082B03D100207047002300E025
:205FA0000A230370004870470300040073B54569044695F81532B5F81A62062B00F2A880D3
:205FC000DFE803F02D466A0432223A00037A062B08D103699B785B074CBF02230823037260
:205FE00001238372237A0020033B012B9CBF05232372637A60712370237A23710623C5F8F1
:20600000CC41A5F8D03184E0037A042B7BD000F108040123C5F8CC41A5F8D03171E0007A26
:20602000002870D1012356E0037A0A2B6BD102230372002060726CE0037A023BDBB2072B5E
:2060400061D8012202FA03F313F09B0F5BD056E0037A022B02D0052B02D054E0002E52D0E2
:206060002369B3F80530B34225D336B9062328462372FFF799FD30464BE0032323720022A2
:20608000631CA669B5F8160204F10C01B0476269E368C2F8CC3134E0037A022B02D0092B23
:2060A00002D030E0092303722369B5F81602B3F80530B34204D20A2323720823637211E0AE
:2060C000E36802A941F8043D3246E369984720B9A5F8D001022323721BE00F2804DC0A236D
:2060E000237260720C4814E0019B80B2C5F8CC312369A5F8D001B3F80530834201D90223CB
:206100002372002005E004F10800FFF73FFF00E0024802B070BD00BF0300040002000400DF
:20612000037A13B10023C37202230372002343728372704770B50C46E37A90F818120546D7
:20614000994202D00E2A63D15FE0022A43D00E2A5BD0012A5CD190F8143203F07F03212B5E
:2061600026D12046FFF722FF0646002855D195F81532052B03D09A1ED2B2012A0AD8606928
:20618000FFF7E9FCA37A002B47D0236A98470023A37242E0012B40D02846FFF705FD237AC0
:2061A000012B3AD1636A002B37D02846984734E0D0F814321A4A23F47F0323F09F039342B3
:2061C00026D123690026C0F8CC310923A0F8D031FFF7C1FC21E090F8143203F07F03212B59
:2061E00016D190F81532012B12D1A669B0F8160204F10C01B5F81A22631CB047064660728C
:2062000040B10A232372074E07E02046FFF788FF054E02E02846FFF7C7FC304670BD00BFEE
:2062200000060021030004000200040000892C3020F003007047FFFF2DE9F0410D68074674
:2062400015F0030F0C469046CE684B6801D0272B5CD905F128022260283B6360236813F068
:20626000030104D0013323606368013BF5E72822284600F063F822682389EA601A446F61FB
:20628000226062682169D31A6360002941D0A369002B3ED06269002A3BD02B62E369A96116
:2062A0006B62EA617278E368042A35D17279FE2A32D1B279012A2FD1B278EA72327813446A
:2062C0005A78212A2BD1B3F805102289914226D19A78120701D5E2690AB3216A2B613846D2
:2062E00021B910492A46FFF72BFE04E02A46FFF727FE0C4B23620023B8F1020F14BF1A4681
:2063000002222A726B72AB72BDE8F0810648BDE8F0810648BDE8F0810548BDE8F081054835
:20632000BDE8F081356100000A00040003000100080004000600040000F032B800F04AB8BD
:20634000FCF7DABD0A2AF0B5034601D1002821DB00200D46114F1E46B3FBF2F32C4602FB62
:206360001366BE5D04F8016B5BB910B12D232370AC1C002323700B46621E9A4203D8084615
:20638000F0BD2546E7E710781C7802F8014903F8010BF2E743420120DBE700BF806A0000C6
:2063A00040EA0103DB0703460CD40346043A22BF51F804CB43F804CBB2F10402F7D2043272
:2063C00008BF7047013A24BF11F801CB03F801CBF8D87047034613F0030F0ED101F0FF01D0
:2063E00041EA012141EA0141043A24BF43F8041BB2F10402F9D202F10402013A24BF03F8E2
:20640000011BFAE77047FFFF5FF800F0CD0000105FF800F0290100105FF800F029000010A5
:206420005FF800F05D0100105FF800F07D0000105FF800F0F100001009021B00010100C0A3
:20644000320904000000FE010204092105001000080001001201000200000040C91F8900EA
:20646000000101020301FFFF09021B00010100C0320904000000FE010204092105001000AB
:20648000080001000403090426034E00580050002000530065006D00690063006F006E00D2
:2064A00064007500630074006F00720073001C034C0050004300200043006F006D0070002B
:2064C0006F0073006900740065001C0341004200430044003100320033003400350036003A
:2064E000370038003900080344004600550008034300440043000E034D0065006D006F0096
:20650000720079000803480049004400FC690000586A000000000000786A000000000000A7
:2065200000000000000000000111220208200001FFFFFFFFFFFFFFFFFFFFFFFF0000000008
:20654000000000000000000001000000FFFFFFFF512563FCC2CAB9F3849E17A7ADFAE6BC08
:20656000FFFFFFFFFFFFFFFF00000000FFFFFFFF96C298D84539A1F4A033EB2D817D0377E9
:20658000F240A463E5E6BCF847422CE1F2D1176BF551BF376840B6CBCE5E316B5733CE2BB8
:2065A000169E0F7C4AEBE78E9B7F1AFEE242E34F4B60D2273E3CCE3BF6B053CCB0061D6546
:2065C000BC86987655BDEBB3E7933AAAD835C65A170A00006D0B0000C90B0000F03DFB4655
:2065E00058918CEB4B43CC7CCB19764322EFB9932C488AFF88DC2BA0480CBF660CF54E1C5B
:20660000B0FC5E21A22FBD07EAB521B7E5485193E8BF628237AEC2A6D6DBED79982F8A42B0
:2066200091443771CFFBC0B5A5DBB5E95BC25639F111F159A4823F92D55E1CAB98AA07D876
:20664000015B8312BE853124C37D0C55745DBE72FEB1DE80A706DC9B74F19BC1C1699BE474
:206660008647BEEFC69DC10FCCA10C246F2CE92DAA84744ADCA9B05CDA88F97652513E9858
:206680006DC631A8C82703B0C77F59BFF30BE0C64791A7D55163CA0667292914850AB72738
:2066A00038211B2EFC6D2C4D130D385354730A65BB0A6A762EC9C281852C7292A1E8BFA2F7
:2066C0004B661AA8708B4BC2A3516CC719E892D1240699D685350EF470A06A1016C1A41941
:2066E000086C371E4C774827B5BCB034B30C1C394AAAD84E4FCA9C5BF36F2E68EE828F74A1
:206700006F63A5781478C8840802C78CFAFFBE90EB6C50A4F7A3F9BEF27871C6222A2B2C2E
:206720003A3B3C3D3E3F5B5D7C7F002A00586D6F64656D2074696D656F757400586D6F64E8
:20674000656D207375636365737366756C6C79207265636569766564200020627974657354
:206760000D0A0073656375726520626F6F746C6F6164657220562E004A756D706572206990
:206780007320696E7374616C6C65640D0A005344206D6F756E74206661696C0D0A007374EB
:2067A000617274696E67206170706C69636174696F6E207570646174652E2E2E0D0A0066F6
:2067C000696E616C697A696E67206170706C69636174696F6E207570646174652E2E2E0D06
:2067E0000A007374617274696E672073656C667570646174652E2E2E0D0A00757362206467
:2068000065746163680D0A0072656164206E6F7420616C6C6F7765640D0A00646F6E652169
:206820000D0A00757362206174746163680D0A004453413A20006C647220646F776E2D676B
:2068400072616465206E6F7420616C6C6F7765640D0A000D0A00FFFF8D01020408102040EB
:20686000801B360D0A00FFFF001BB70000000000800000000000000000FFFFFF00F9FFFFEC
:2068800000FFFFFF00FBFFFF00FFFFFFB8010000C0010000C80100006003000068030000F4
:2068A000D0010000A4130000BC130000AC100000B4100000D8010000E001000098030400A8
:2068C000A00304003000000038000000F20000006908000010110000181100007812000072
:2068E00090120000E8010000F0010000F801000001010000090100002101000041010000B3
:2069000049010000510100007101000079010000C4310000CC310000F431000000000000D8
:2069200080000000000000000000000000FEFFFF0000000000FEFFFF0000000000000000DF
:2069400080000C400880084008800840080003400800034008C00A4008C00A40044003408A
:2069600000C0084000C0004000C00040000001400000014000800940008009401840004063
:206980001C400040188000401C800040180009401C00094008800A400C800A400000000039
:2069A0000000000000C0094000C0094000400A4000400A40184009401C4009400002000069
:2069C00000000000020100000000000002020202020202020000000000000202000201019C
:2069E00001010101000000000000000000000000000004040000000000000000BD5000007E
:206A000065510000C5500000B9540000E1500000655400003151000035510000E951000072
:206A20001D5200004F52000051520000755200009D520000C1520000E952000067540000E4
:206A4000E55300006B5400006F54000075540000115100000D530000415F0000695F000089
:206A60004D5B0000575B0000855B0000A95B0000B35B0000BD5B00002D6200003962000088
:206A80003031323334353637383961626364656600FFFFFF00231946054A1360054A136091
:206AA000054A99540133B3F5807FFAD1704700BFE0080010E4080010E00700100023104A16
:206AC000F0B513600F4A13600F4A16469B540133B3F5807FFAD100231A460C4C04F5807EB6
:206AE000994298BF00236778C55C3A442A44D2B2B55C013304F8015FA645B754F0D1F0BDCC
:206B0000E0080010E4080010E0070010DF070010F0B5104C0026A4460F4B25681B680F4FBB
:206B2000864203D1CCF800300020F0BD0135EDB2EC5D2344DBB213F807E005F807E0DC55DF
:206B40007444E4B211F806E0E45D84EA0E0494550136E5E7E0080010E4080010E007001060
:206B6000322300B58BB005930690079105A801A9034B98479DF804000BB05DF804FB00BF1F
:206B8000F11FFF1F00B533238BB008924FF47A720593084B06901B680791B3FBF2F305A8DC
:206BA000099301A9044B98479DF804000BB05DF804FB00BF74CE0010F11FFF1F34234FF4E0
:206BC0007A7200B58BB00593074B06901B680791B3FBF2F305A8089301A9044B98479DF8F6
:206BE00004000BB05DF804FB74CE0010F11FFF1F2DE9F047A14C8AB004F11801102206A8A0
:206C00002669D4F814A000F06DF91022002104F1180000F063F902AC4FF40042FF21984830
:206C200000F05CF910229749204600F05BF94FF4E04300941A4692499348914C00F05EF91F
:206C4000022000F053F92546002341F6FC308F4A54F82310013383429160F9D1936846F6A2
:206C6000F072A2589A4207D04FF40042FF21844800F034F9864810E0864800F03BF94FF484
:206C80004073D4F800231B689A420CD24FF40042FF217B4800F022F97F4800F02BF90020A7
:206CA0000AB0BDE8F08746F6B071754800F012F97A4900F027F948B94FF40042FF217048B8
:206CC00000F00CF9764800F015F9D3E7754800F011F9102106A8FFF7F1FE4FF480524FF476
:206CE000E041714800F0FEF8704A6F494FF48050FFF70EFFFFF7CEFE00226B4913460C4609
:206D000041F822300132B2F5806FF9D14FF49672B6FBF2F002FB106006AE96E8C00306937C
:206D200007930893099308B100F0F0F8604ABAFBF2F302FB13AA72B607210120FFF710FF7D
:206D400007210120FFF73AFFBAF1000F04D0002300BF01339A45FBD100210846FFF700FF08
:206D600000210846FFF72AFF0021524B0846C5F8FC32FFF7F5FE4FF4805241490020FFF7F0
:206D800001FF4D4B5A699206FCD52E2210211A6006A806960797CDF82080CDF82490FFF778
:206DA0008DFE414A41494FF48050FFF7B1FEFFF771FE07210846FFF7D3FE3F4B5A699706EF
:206DC000FCD52E221A6000233C48E218195C0133402B82F8001EF8D14FF4805232494FF42F
:206DE000E040FFF7CFFE344B5A699606FCD52E221A6000231A4644F823200133B3F5806F6A
:206E0000F9D12D4B5A699006FCD52E224FF480544FF02A08284E1A60210B0846FFF7A0FE30
:206E2000291920464FF48052FFF7ACFE04F5805473699906FCD5B4F5E04FC6F80080EBD10A
:206E400000234FF0FF3245F823200133B3F5005FF9D11B4B1B4A1A60174B5A699206FCD547
:206E60002E221A60BFF34F8F1749184BCA6802F4E0621343CB60BFF34F8FFEE704D00010B1
:206E8000E82800100C01000000000080000009206502000074020000366800009898001061
:206EA00030680000E2670000E808001074BD001020A107002143658700C00040DC65000057
:206EC00000D0001081EC9C4A00ED00E00400FA05FFFFFFFF5FF800F0611700005FF800F0AD
:206EE0003D6300005FF800F0396300005FF800F0C13D00005FF800F0352A00005FF800F0DD
:206F0000F92D00005FF800F0F51300005FF800F0852900000C6500000101FFFFFFFFFFFF9A
:206F2000FFFFFFFFFFFFFFFFFFFFFFFFFFFFFFFFFFFFFFFFFFFFFFFFFFFFFFFFFFFFFFFF71
:206F4000FFFFFFFFFFFFFFFFFFFFFFFFFFFFFFFFFFFFFFFFFFFFFFFFFFFFFFFFFFFFFFFF51
:206F6000FFFFFFFFFFFFFFFFFFFFFFFFFFFFFFFFFFFFFFFFFFFFFFFFFFFFFFFFFFFFFFFF31
:206F8000FFFFFFFFFFFFFFFFFFFFFFFFFFFFFFFFFFFFFFFFFFFFFFFFFFFFFFFFFFFFFFFF11
:206FA000FFFFFFFFFFFFFFFFFFFFFFFFFFFFFFFF4A0F507B68229174CCD84E1A8BBBC373A6
:206FC0006CFD7716A707B13A143BB239AA3D86333C1E413C84348BFD0F090B65FCD58B3518
:206FE0002B48F29A9BBF575F43785755F10012BA11607884FFFFFFFFFFFFFFFFFFFFFFFFFD
:20700000FFFFFFFFFFFFFFFFFFFFFFFFFFFFFFFFFFFFFFFFFFFFFFFFFFFFFFFFFFFFFFFF90
:20702000FFFFFFFFFFFFFFFFFFFFFFFFFFFFFFFFFFFFFFFFFFFFFFFFFFFFFFFFFFFFFFFF70
:20704000FFFFFFFFFFFFFFFFFFFFFFFFFFFFFFFFFFFFFFFFFFFFFFFFFFFFFFFFFFFFFFFF50
:20706000FFFFFFFFFFFFFFFFFFFFFFFFFFFFFFFFFFFFFFFFFFFFFFFFFFFFFFFFFFFFFFFF30
:2080000080FF0010758100004D810000158100002F810000358100003B8100000000000055
:208020000000000000000000000000009108050041810000000000001D0905006109050046
:208040004781000069210200011D0300F9350200CD1C0300853B030069CE0100BDCE010008
:2080600099CE01004781000047810000B598030047810000478100004781000085BF01001B
:208080004781000047810000478100004781000047810000478100004781000047810000A0
:2080A000211D050047810000F174040047810000B1DF0500397504004781000047810000AD
:2080C000478100004781000047810000478100004781000047810000478100004781000060
:2080E0004781000064F0070000000010C807000064F007000008002000000000C80700101C
:20810000B072000000080020A077000000000080FC2801001EF0040F0CBFEFF30880EFF321
:2081200009808169004A1047E1090100FEE708B508F086FC08B508F083FC08B508F080FCBF
:2081400008B508F07DFC08B508F07AFC08B508F077FC002310B5934200D310BD1C585C5021
:208160000433F8E700231A468B4200D370471A500433F9E738B50D4C0D4DAC4207D30D4DCC
:20818000AC420CD32CF0C0FF5CF074FDFEE7D4E900010C3454F8042CFFF7DBFFEDE754F82B
:2081A000080B54F8041CFFF7DDFFE9E7E4800000FC80000014810000FFFFFFFFFFFFFFFF31
:2081C000FFFFFFFFFFFFFFFFFFFFFFFFFFFFFFFFFFFFFFFFFFFFFFFFFFFFFFFFFFFFFFFFBF
:2081E000FFFFFFFFFFFFFFFFFFFFFFFFFFFFFFFFFFFFFFFFFFFFFFFFFFFFFFFFFFFFFFFF9F
:2082000012EFCDABE3FDE15FFFFFFFFFFFFFFFFF70B50446002020C940CA400875414041CC
:2082200020C4013BF7D170BD70B5012420C940CA6408B541644120C0013BF7D1B4FA84F0DF
:20824000400970BD2DE9F0410024013B9B0025462646A4465FF0000E03E05FEA0C0EBEEB59
:20826000030EBCEB0E0752F8078051F80E70A7FB0878E41955EB080556F100061EF1040EBF
:208280009E4501DCE645ECDD40F80C402C46354600261CF1040C9C45DCDDBCEB430FDCDD2A
:2082A00040F80C40BDE8F081002310B51C465AB2914200DC10BD40F823400133F7E7002382
:2082C0001A4610B55CB2A14203DCB2FA82F0400910BD50F8234001332243F3E701234A11D8
:2082E00050F8220001F01F0103FA01F108407047013910B549B2041D0A06CBB204D401395B
:2083000054F82120002AF7D001335BB273B103F18042013A50F82220002022B9013B00EBDD
:20832000431318B210BD52080130F6E71846F9E7002310B55CB2A24200DC10BD51F823407B
:2083400040F823400133F5E710B5013A52B2130601D5002010BD50F8224051F822309C426F
:2083600005D802F1FF32F2D24FF0FF30F2E70120F0E7002300EB8101884200D3704751F8CC
:20838000042D43EA52030B60D307F5E770B59DF910401E4623460546FFF73AFF30B9224666
:2083A00029463046FFF7D0FF012807D02346324629462846BDE87040FFF736BF70BD70B5C3
:2083C0009DF910401E4623460546FFF72DFF38B12346324629462846BDE87040FFF718BFB4
:2083E00070BD2DE9F04F1F46B5B09DF9F85004AC2B4681462046FFF725FF24AB294638462F
:20840000CDE90234FFF774FFC0EB851004B22646002CB8BF04F11F06634246F3471603F0BA
:208420001F0304F01F0814A858BFC3F100083146FFF73AFFB8F1000F4FEA86002CDD002228
:2084400014AB18441346C8F1200CAB4219D301266B0000934FEA850814AB434401936F1E98
:2084600034AB03EB8707002C53DA34AB03EB86062A4656F8C81C4846FFF75AFF35B0BDE8E6
:20848000F08F57F82360013306FA08F10A4340F8042B26FA0CF2D8E714AB2A4639461844C3
:2084A000FFF746FFD3E75AF8C83C0CF1010C53F8202034AB03EB800353F8803C0B44D31A49
:2084C00034BF4FF0010B4FF0000B9A4218BF59465EF8C82C42F82030009B4FFA8CF09842B4
:2084E000E1DB731A5E42294614A85E41FFF741FF34AB434453F8802C57F8803C294643EA8F
:20850000C2730198013C47F8803C24B2FFF731FFA9E74FF0000C34ABC6F1010E614603EB44
:20852000860A03EB8E0ED7E730B505461C4691B0684693F90030FFF785FED4F8AC30694656
:208540002846984711B030BD13460A46FFF7ECBF2DE9F04793F9006092B0044689461046EC
:20856000314615469846FFF7AAFE002840F091804246494602A8FFF7E7FF434602AA21460B
:208580000AA8FFF7D1FF02A908464246FFF7DCFF43462A4649464846FFF7C6FF08F104073C
:2085A000424629462846FFF7CFFF3B462A46214620460096FFF7EAFE3B462A462946284692
:2085C0000096FFF7E3FE3B462A46214628460096FFF7F5FE43462A4621462046FFF7A4FF8A
:2085E0003B462246214628460096FFF7CFFE3B4600962A4621462046FFF7C8FE2368DB07E7
:208600004AD533463A4621462046FFF701FE824631462046FFF7ADFE06F18043013B54F8F8
:20862000230040EACA7044F82300424621462846FFF78AFF3B460AAA294628460096FFF7DA
:20864000BEFE3B460AAA294628460096FFF7B7FE0AA908463B462A460096FFF7B0FE434656
:208660000AAA21462046FFF75FFF02AA3B46104621460096FFF7A3FE324629462046FFF7CB
:2086800057FE49462846FFF753FE02A94846FFF74FFE12B0BDE8F08731462046FFF769FEAD
:2086A000C3E72DE9F04115468AB0044688461C22002103A85CF0E9FA032395F900702A464F
:2086C000414620462E1D0293FFF73EFF334602AA214620460097FFF772FE2B46424621464B
:2086E0002046FFF721FF0097334605F1840221462046FFF74BFE0AB0BDE8F081F0B50822C7
:2087000089B00C460646FFF713FE0027CB6A6A4603930B6B684604934B6BCDE901770593A2
:208720008B6B00970693CB6B694607930823FFF76FFD082305466A4631463046FFF768FD99
:20874000236B05440393636B6A460493A36B69460593E36B6846CDE906370823FFF758FDDD
:20876000082305446A4631463046FFF751FD236A05440093636A6A460193A36A3146029311
:20878000A36B30460693E36BCDE90477079308230397FFF73DFD636AA26B0093A36A04929E
:2087A0000193E36AE26B0293636B0544CDE905230393236A6A460793314608233046FFF786
:2087C00027FDE36A05440093236B6A460193636B31460293236A30460693A36ACDE90477C6
:2087E000079308230397FFF71FFD236B2D1A0093636B6A460193A36B31460293E36B3046B0
:208800000393636ACDE904770693E36A07930823FFF70AFD636B2D1A0093A36B6A46019322
:20882000E36B31460293236A30460393636A0493A36ACDE90537236B07930823FFF7F4FCA9
:20884000A36B2D1A0093E36B6A46CDE90137636A31460393A36A30460493E36ACDE9053711
:20886000636B104C07930823FFF7DEFC2D1A0FD435B9082231462046FFF766FD01280FD0B9
:208880000823224631463046FFF7CEFC2D1AEFE70823224631463046FFF7BAFC2D18F7D43F
:2088A00009B0F0BD40870600F0B515461C4607460E4689B01A4629466846FFF745FE23462A
:2088C0006A4639463846FFF72FFE23462A4669466846FFF729FE23466A4631463046FFF779
:2088E00023FE09B0F0BD2DE9F043144680461F4689468BB0129D024615F9046B21462B46CD
:2089000002A80096FFF75BFD02A9129A0846FFF71BFE129B02AA41464046FFF705FE129B09
:2089200002AA21462046FFF7FFFD2B464A46394638460096FFF743FD129A394602A8FFF737
:2089400003FE02A92B46424608460096FFF737FD02A92B46224608460096FFF730FD2B4668
:208960004246214620460096FFF729FD129B224649464846FFF7D8FD2B4602AA41462046E9
:208980000096FFF71CFD129B224639463846FFF7CBFD2B464A46394638460096FFF70FFDCC
:2089A000324602A92046FFF7C3FC0BB0BDE8F083F8B50E46D11C48BF911D144641F38701ED
:2089C0000546FFF771FC0021671E4AB2A24201F1010100DBF8BDBB1A23F00300B25C03F0F3
:2089E0000303DB0002FA03F32A581A432A50ECE72DE9F0471F46B3F90230894613F11F01F5
:208A000048BF03F13E014D11D91D48BF03F10E01CC10944228BF14464FFA85F84146064632
:208A2000FFF742FC22464946FFF7C2FFB7F90220E40094421FD9A41A002206EB8501C4F1C4
:208A400020058E420ED32437424631463846FFF77BFC01280FD043463A463046BDE8F04798
:208A6000FFF7E2BB51F8040D20FA04F313430B6000FA05F2E5E7BDE8F08770B50368054683
:208A800013F00106144605D013460A460146FFF7BFFB064621462846FFF76BFC46B104F193
:208AA0008042013A55F8223043F0004345F8223070BDF0B50F46A1B0064619463846154619
:208AC0001C46FFF7FCFB20B13046FFF7EDFB21B0F0BD224639466846FFF72AFC294608A8D4
:208AE000FFF726FC10A82146FFF7DEFB012318A81093FFF7D9FB224608A96846FFF724FC42
:208B000028B9224610A93046FFF712FCDFE7009BDA0709D421466846FFF72BFC22462946B1
:208B200010A8FFF7AAFFE6E7089BDB0707D4214608A8FFF71EFC2246294618A8F1E70028F3
:208B400023461CDD08AA69466846FFF76DFB21466846FFF70EFC224618A910A8FFF7F4FB6B
:208B6000002805DA10A923462A460846FFF750FB10A9234618AA0846FFF756FBCEE708A9EE
:208B80006A460846FFF750FB214608A8FFF7F1FB224610A918A8FFF7D7FB002805DA18A92C
:208BA00023462A460846FFF733FB18A9234610AA0846FFF739FBBEE72DE9F04F4FF0000BCA
:208BC00080461D46FDB0869E0592B6F9023096F9004013F11F0748BF03F13E0747F3471752
:208BE00007F1FF3924AB43F829B07CAB03EB890242F8C0BC42F8A0BC8A4696F901200146AF
:208C00006CA8FFF7D5FEA3000793A2006CAB134496F90120184608EB02010493FFF7C8FED3
:208C2000294696F901204CA8FFF7C2FE96F9012054A8A918FFF7BCFE21464CA8FFF73FFBC3
:208C40000546002840F0348154A8FFF738FB8346002840F02B8106F124033A464CA91846D9
:208C60000393FFF771FB012840F022813A4654A90398FFF769FB0128069040F019811CAD3C
:208C80000DF130083B46039A54A92846FFF711FF514640463346059A48F829B0FFF7A8FE25
:208CA00041464046039B2A460097FFF79AFB0DF5B879039B2A464CA914A80097FFF791FB6C
:208CC000224648466CA9FFF733FBA30009EB030A50460499FFF72CFB06F14403194634A8F8
:208CE0000493FFF725FB049BA10059183CA8FFF71FFB331D494634AA284600940593FFF7D5
:208D00005EFB53464A463CA934A80096FFF7EBFD2346321D29462846FFF7CBFE2A46514641
:208D200048463346FFF7C0FD049B3946099340466CABCDE90A39CDF820B0FFF7D9FA39464C
:208D4000814614A8FFF7D4FA8145B8BF81461FFA89F909F1FF331BB2194640460493FFF7C2
:208D6000BDFA049B10F10008194614A818BF4FF00108FFF7B3FA002814BF022300230DF176
:208D8000200A48EA03085AF828802246414624A8FFF7CEFA0DF1B00AA30008EB0301504611
:208DA000FFF7C6FA21462846FFF77EFA069BA9F102082B600FFA88F80DF190090495B8F188
:208DC000000F22DADDE9041223460846FFF771FE3346049A51464846FFF766FD3A464946EC
:208DE0000398FFF7B1FA012804D03B46039A4846FFF71AFA013C64B24CAA23064DD5BBFA3B
:208E00008BF040097DB0BDE8F08F049A334651464846D6F8A450A84741460CA8FFF75EFAC7
:208E2000031C18BF0123414614A80693FFF756FA002814BF02220022069B134308AA52F8C2
:208E400023302BB32246194634A80693FFF770FADDE906313CA85918FFF76AFA3346049A82
:208E60003CA934A8FFF720FD059B34AA494644A80094FFF7A4FA53464A463CA934A800967D
:208E8000FFF731FD0499334644AA0846FFF74CFB08F1FF380FFA88F891E759F8243052F8FF
:208EA0002410013C4B404BEA030BA6E72846A9E75846A7E730B504460D4693B04022084944
:208EC00002A85BF0DEFE074B2022009321462B4602A8FFF771FE003018BF012013B030BDDB
:208EE000EC8706003C8706006C2200215BF0CDBE20B1002200F16C03984200D1704700F8FE
:208F0000012BF9E700230D490D4ADFF848C0C0E902120C4A0C49C0E904C20C4AC0E900338D
:208F2000C0E906120A4A8366026202F17452A2F52302A2F692424262704700BF67E6096A14
:208F400085AE67BB3AF54FA57F520E518C68059BABD9831F72F36E3C2DE9F04FD1B000F1D9
:208F6000080308AA019300F1280310460693019B53F8044B40F8044B069CA342F8D1D2E9CD
:208F8000004C4FF00009D36915690493D2E9053E0293936810AE0393D3680593424B079310
:208FA000B9F10F0F67D84B7891F800A01B0443EA0A6391F803A091F8028043EA0A0343EA67
:208FC0000823029F4FEAF52A8AEAB51A8AEA75608EEA070A0AEA050A079F8AEA0E0A82445D
:208FE00057F8040B46F8043B8244049853440344059807971844039F824644EA0C084FEADA
:20900000743080EAB40008EA070804EA0C0B80EAB45048EA0B0809F101098044B9F1400F14
:20902000434401F10401CDF810E005971AD10299CDE90834CDE90D51CDF83CE0CDF830A05F
:20904000CDF828C00B97019B52F8041B1B680B44019941F8043B069B01918B42F3D151B013
:20906000BDE8F08FCDF80CC0DDF808E0A44602951C46554694E756F8083C56F83C0C4FEA24
:20908000F34888EA734888EA932856F8407C56F81C3C4FEAB04B3B448BEAF01B98448BEA07
:2090A000D00343448DE700BF2C8806002DE9F8430368054603F03F079B18036028BF436881
:2090C0000E4628BF0133144628BF436097B1C7F1400991450ED800F128084A4608EB07008D
:2090E0005BF0CFFD403C414628463C44FFF734FF00274E44A04606EB040904E02846FFF75A
:209100002BFFA8F14008B8F13F0FA9EB0801F5D86FF03F03A20906EB821103FB024232B1EE
:2091200005F128003844BDE8F8435BF0AABDBDE8F8830AB1FFF7BABF7047FFFFF7B50D4605
:20914000D0E90021530F43EAC1031BBA354F0093D30002F03F02372A044694BFC2F1380601
:20916000C2F178061BBA40220021384601935BF08CFD80233246394620463B70FFF7D9FF07
:20918000082269462046FFF791FFE37A2B7063896B70A3681B0AAB70A368EB70E37B2B71A0
:2091A000E3896B71E3681B0AAB71E368EB71E37C2B72638A6B7223691B0AAB722369EB72B7
:2091C000E37D2B73E38A6B7363691B0AAB736369EB73E37E2B74638B6B74A3691B0AAB74F0
:2091E000A369EB74E37F2B75E38B6B75E3691B0AAB75E369EB7594F823302B76638C6B7627
:20920000236A1B0AAB76236AEB7694F827302B77E38C6B77636A1B0AAB77636AEB7703B0C1
:20922000F0BD00BFC807001030B504460D469DB001A8FFF759FE01A8FFF764FE2146074C63
:209240002A4601A8FFF775FF214601A8FFF776FF01A8FFF74DFE20461DB030BD08080010E6
:20926000F7B5884D48F016F82C46874E0190874B01A819684FF47A73B3FBF1F30A21B1FBBA
:20928000F3F148F005F9AA8F0021063205EB420230464AF0F5FEAA8F01210A3205EB420280
:2092A00030464AF0EDFEAA8F02210E3205EB420230464AF0E5FEAA8F0621123205EB4202D8
:2092C00030464AF0DDFEAA8F0721163205EB420230464AF0D5FEAA8F03211A3205EB4202C6
:2092E00030464AF0CDFEAB8FB4F80EC001339BB2A289032B88BF00236245114628BF61466F
:209300006245174638BF6746AB87238A608A994228BF19469F4238BF1F466244134403443A
:20932000B4F816C0B842A28A2CBF1B1ADB1B884294BF1B1A5B1A6245114628BF6146624575
:20934000174638BF6746C3F34E032380238B608B994228BF19469F4238BF1F46624413446E
:209360000344B4F81EC0B842A28B2CBF1B1ADB1B884294BF1B1A5B1A6245114628BF61468C
:209380006245174638BF6746C3F34E036380238C608C994228BF19469F4238BF1F4662449C
:2093A00013440344B4F826C0B842A28C2CBF1B1ADB1B884294BF1B1A5B1A6245114628BF93
:2093C00061466245174638BF6746C3F34E03A380238D608D994228BF19469F4238BF1F4619
:2093E000624413440344B4F82EC0B842A28D2CBF1B1ADB1B884294BF1B1A5B1A624511468B
:2094000028BF61466245174638BF6746C3F34E03E380238E608E994228BF19469F4238BF14
:209420001F46624413440344B842A28EB4F836C02CBF1B1ADB1B884294BF1B1A5B1A624533
:20944000114628BF61466245174638BF6746C3F34E032381238F608F994228BF19469F4231
:2094600038BF1F46624413440344B8422CBF1B1ADB1B884294BF1B1A5B1AC3F34E0363818A
:20948000F5E600BF2808001000400340CC20001073B506460124184D694628464AF0CCFD55
:2094A0003246694628468DF805404AF0F4FD2246284600214AF006FE2246214628464AF076
:2094C00001FE2246284602214AF0FCFD2246284606214AF0F7FD2246284607214AF0F2FD0F
:2094E0002246284603214AF0EDFD284621464AF0F9FD204602B070BD004003400C2809D86C
:20950000012303FA00F041F2AA53184208D110F4256F07D111F0030F14BF1C201D20704751
:209520001F2070471E207047F8B504460125027847788678013AAF4211D80023D9B2B14236
:2095400015D33C202179E37848434FF4616101FB0303607903440A4800FB0230F8BD28467E
:209560003146FFF7CBFF01350244EDB2E3E7890714BF02F26D1202F5B7720133DEE700BF21
:20958000805101002DE9F041C8B080461D210DF105002BF0B9FE002800F0858018F08AF8BA
:2095A00030B919F0FFF80446204648B0BDE8F0813F4B9A781F4612B119F0F6F8F3E71B78DC
:2095C000B8F1110FA3F1020362D1022B6DD811F0DBF8384B9DF80500187119F0FFFD19F0FC
:2095E00055F8012006F00EFFB8F1110F14BF4123402304A8ADF8103006F058FF0446002847
:209600004ED10DF10601404608F0B0F80446002846D14FF48C7697F826059DF8052070430B
:20962000254BBDF80610254D1A7259812B181A710322B8F1120F5A7027D1214B93F8A230CF
:20964000012B22D1053004221E4928445BF019FB97F82605042206FB00501B4909305BF045
:2096600010FB1A4902A815F005FF97F82605052206FB005002A90D305BF003FB97F826357C
:2096800006FB03556B780D336B7019F0E3FD8BE7012B0AD819F0FAFD002898D1D52483E716
:2096A00019F020F880E74F247EE773247CE700BF509A0380F8860380C01F001040B40080C0
:2096C0005E5206809C890380A0890380888703804FF48C722DE9F041384D394C95F82635F4
:2096E00088B002FB03435B78012B65D16A46354B16461F683B4607F1180E944618685968ED
:209700000833ACE8030073456246F6D11868CCF800009B88ACF804302B4B1A7A9C46012AFA
:209720001BD12A4A0020114697F804E092F800801346F04537D143239CF8062043433ABBA4
:20974000CA1852788DF804203A78FAB90233102219440DF106005DF081FE0DF106005DF06A
:209760002CFE3146C21D1A485BF08BFA0DF106005DF023FE4FF48C7295F82635083002FB67
:2097800003446070002008B0BDE8F0811233DEE7CA1892F822208DF804203A780AB9233398
:2097A000D5E73333D3E71028D7D093F8433001304332002BBAD1D0E77E20E4E7509A038007
:2097C00040B40080D83000100953068074A20600C81F00104FF48C712DE9F041874F884AD9
:2097E00097F82635A8B001FB03235B789046052B40F0008117F0B0FD014620B117F07AFD31
:2098000028B0BDE8F0810DF107002BF07DFD002800F0F28043F243137A4C7B4D638118F031
:209820000DFFA08118F08AFEA07318F06FFEE07318F096FE754B20741B780EA8A374744B81
:209840000EAEB3F83031A382724BDB88E382BB78637697F82635A3762AF02EFA0FCE0FC594
:2098600096E80F0085E80F003B78103D022B1ED116A90EA82AF078FA1FA905F160002AF08A
:2098800073FA16A85DF040FE06461FA85DF03CFE614B301ADA796FF03B03534303F5A83329
:2098A00003F5C073984202D9032018F0DFFE002384F82A303B78082B23767ED1574BDB7804
:2098C000022B76D0032B76D0012B01D11823237644F24E13E36140F201132384102384F858
:2098E0002230159B84F82630149B84F82530119B84F82430109B84F827300F9B84F828309C
:209900000E9B84F8293095F8B230FF2B65D1002395F88020E362B5F884300AB1013B9BB2C0
:2099200000260022238600233146CDE90423CDE9062308A809226686A6865BF0A6F90922D8
:2099400031460BA85BF0A1F995F89A30082213F0DF0F49D1324908A85BF093F902223149CC
:209960000BA85BF08EF904AA2F4908A85DF0EEFB06AA2D490BA85DF0E9FB2C49069A079898
:20998000A2FB015601FB00660499059A691846EB0202C4E90E124FF48C729DF80730002085
:2099A000237297F8263502FB0388302388F8013026E728238BE7382389E70D2B88D1174B14
:2099C000DB78022B05D0032B05D0012B80D11D237DE72D237BE73D2379E702AA1249144839
:2099E0005DF0B4FB029B93E7124908A85BF049F90422B4E77E2003E74F2001E7509A0380AF
:209A000040B40080C01F001068870380C3580680E02506806C1A00105E520680F886038078
:209A2000FA870380F88703802C89060000E1F50524880380FC870380F7B54FF48C76194FFC
:209A4000194D97F8263506FB03535B78062B23D117F0A2FC044618B117F04CFC03B0F0BD00
:209A60001E210DF107002BF04FFCB8B10F4B1B7C022B15D80E491B01CA18CB5C83B10D4BC0
:209A80005178526819725A72042297F82635204606FB03535A70E1E77E20DFE74F20DDE7F6
:209AA0003620DBE7509A038040B40080A81E0010209A0380C01F00104FF48C7273B52F4DC6
:209AC0002F4E95F8263502FB03635B78052B51D117F042FC014618B117F00CFC02B070BD56
:209AE0000DF107002BF010FC002845D0254B264CDB882A786381AB78082A63732273234B04
:209B000029D1DA78022A22D0032A22D0012A01D1182222731B8BA37317F030FCE07327F097
:209B2000F9FF4FF48C721A4B20749B8800201B0923756B78E07463759DF80730A07523726F
:209B400095F8263502FB036610237370C6E72822DFE73822DDE70D2ADCD1DA78022A05D08F
:209B6000032A05D0012AD5D11D22D2E72D22D0E73D22CEE77E20B1E74F20AFE7509A038058
:209B800040B400806C1A0010C01F0010F886038028080010074B5A689C2A9CBF9D225A60DD
:209BA000054AD269072A04BFDC225A600122034BDA727047209A03806C1A0010509A0380BB
:209BC000F7B54FF48C761A4F1A4D97F8263506FB03535B78082B24D117F0DEFB044618B195
:209BE00017F088FB03B0F0BD1E210DF107002BF08BFBC0B1104A137C022B16D80F481B01AE
:209C0000C118C35C8BB1537C4B70937C4B60FFF7C1FF022297F82635204606FB03535A7081
:209C2000E0E77E20DEE74F20DCE73620DAE700BF509A038040B40080A81E0010209A0380FE
:209C40004FF48C71F8B5244D244F95F8262501FB02725278012A3AD12B78092B39D1204C9E
:209C6000637813BB0026E37833B108221D491E485BF007F80023E37094F8733013B100230A
:209C800084F87330002018F06DFF184B93F864310BB114F023FC4FF48C7295F8263502FB89
:209CA000037302225A703046F8BD08220D490E485AF0E7FF0E4B0F4A1A60002363700E4B94
:209CC0001B78552BCED129F03FFB0646CBE77E26E9E77326E7E700BF509A038040B4008006
:209CE0006C1A0010A001001004290180688703800029018021436587C8370680F7B54FF48F
:209D00008C723C4C3C4F94F82635064602FB03735B782546082B67D117F03EFB28B117F0C3
:209D2000E9FA0446204603B0F0BD1E210DF107002BF0EAFA002859D017F0BCFC10B918F00C
:209D400031FDEEE7A47814B118F02EFDE9E72A78002E36D0062A4BD1284E336923F07F4214
:209D6000EB6823F07F439A420ED06B7963B906F1100018F0E9FC08B97D24D3E733697C24B5
:209D8000AB811B0CAB73CDE7306929F077FFB27C717C307C18F0EEFC00236B716B78023B9E
:209DA000012B03D9042018F061FC01E018F068FC4FF48C7295F8263502FB037702237B7015
:209DC000B0E7092A14D80123934013F4247F0FD00B4E304618F0B8FC0028CDD0336806203C
:209DE000AB811B0CAB73DEE77E249BE74F2499E7732497E7509A038040B40080A81E00104A
:209E0000B81E0010F7B54FF48C771E4D1E4E95F8263507FB03635B78082B2AD117F0BCFA85
:209E2000044618B117F066FA03B0F0BD1E210DF107002BF069FAF0B12A78092A1DD80123F7
:209E4000934013F4247F18D0104B1A7C172A16D85A7C3B2A13D89A7C3B2A10D8186929F05A
:209E6000F1FE022295F82635204607FB03635A70DAE77E20D8E74F20D6E77320D4E7332064
:209E8000D2E700BF509A038040B40080A81E00102DE9F047C54D90B02B7A2C46EC2B00F0D6
:209EA0001A8277D8082B00F09F8422D8042B00F0538407D8022B00F0E083032B00F01D8463
:209EC00036243CE1062BBA4EBA4C00F076844FF48C7340F2518494F8260503FB00635A78AF
:209EE000062A40F0038202225A701EF0D1FB044625E1E72B00F072811BD8E42B00F02381DA
:209F0000E62B00F03681E32BDAD14FF48C71A94DA74A95F8263501FB03235B78062B40F06B
:209F2000E581D4F80F20A44B9A4200F0EB80332405E1E92B00F08E81C0F06C81EB2BBFD107
:209F40004FF48C729B4D9A4C95F8260502FB00425278062A40F0CA81984BDB69072BAFD1AD
:209F60004FF48C7606FB004004302EF06BFE95F82605704323181A790430914B20441A7267
:209F80005DF01BFA95F82635023006FB034358700024D4E0F32B00F0248267D8EF2B00F061
:209FA000D98137D8ED2B00F0B781EE2B88D14FF48C70804D7E4E95F8262500FB02625278AD
:209FC0000B2A40F0938117F013FF002800F0318104227C4903A8E47B5AF053FE04227A49AC
:209FE00008A85AF04EFE4FF47A7018F083FA2046089A039917F02EFF0446002897D14FF474
:20A000008C726F4B187295F8263502FB036302225A7094E0F12B664E664F00F0E1824FF436
:20A020008C7840F2BA8197F8263508FB03635B785A1F3D2A00F25A8100242B4408A905F1A2
:20A040000F005C7325F042F95D4B0422187297F8260508A908FB006005305AF012FE97F88E
:20A06000263508FB03660723737068E0F72B00F0DD8225D8F52B4E4E4E4F00F098824FF4B0
:20A080008C7040F2BE8197F8263500FB03604378062B40F02B81D5F80F00431E0D2B3FF699
:20A0A00046AF17F035FD0446002840F0D18201464FF4807245485AF0E8FDC7F83445AEE27D
:20A0C000FB2B00F00F82FC2B00F03782F82B7FF4F7AE4FF48C703749354A91F8263500FBB1
:20A0E00003204078062840F001813948D5F80F40844204BF3748C1F838054FF48C7101FBCE
:20A10000032334E017F0E6F808B117F099F80024D5F84425D5F850352F49D5F84005134442
:20A12000C5F85035D1E90023161843F10007C1E90067C5F84445C5F8404518F0DDF82046BB
:20A1400010B0BDE8F0874FF48C761A4F184C97F8262506FB02425378082B40F0C78005F187
:20A160000F0018F09FF897F8263506FB034302224EE04FF48C700F4E0D4C96F8261500FBF5
:20A1800001414978822940F0B18005F14F0105F10F0018F02DF800283FF4C9AE4FF48C7225
:20A1A00096F8263502FB0343E1E700BFA81E001040B40080509A0380010203046C1A001095
:20A1C000C01F0010B81E0010BC1E0010680800106D7C8B9A78563412989F03804FF48C7520
:20A1E000AD4EAE4C96F82605684323185B78062B7CD1AB49AB4B11F87C2F04301A722044B8
:20A2000040225AF03EFD422296F8263505FB03435A70BDE64FF48C709F4EA04D96F8261575
:20A2200000FB01514978062960D19F4B5B69580501D55E2483E7D4F80F209C4B9A427FF4B2
:20A2400076AE17F009FF4FF48C7296F8263502FB03538CE74FF48C708F4E904C96F826250A
:20A2600000FB02425278222A40D118F0E3FF28B34FF47A7018F03EF91022002103A85AF0FF
:20A2800004FD202305F10F02009303A96B44884811F053FF002308AA12F8011BFF2915D05A
:20A2A000844BD3E92201DDE90C238B4208BF82427FF43DAE08A817F0A3FE6FE7202205F15F
:20A2C0000F010DEB02005AF0DCFCE3E70133DBB2102BE1D12BE64FF48C756F4E6F4C96F87F
:20A2E000262505FB02425778062F01D07E2426E717F092FC04226B4B0890187296F82605FF
:20A3000008A905FB004010445AF0BBFC96F8263505FB03435F703BE64FF48C765E4C5F4D3D
:20A3200094F8263506FB03535B78062BDED117F073FC80287FF6C4AD5F4813F057FB5F4B82
:20A340005F4A1A60012384F83E3594F8263506FB03530CE74FF48C754F4E504C96F8262540
:20A3600005FB02425378062BC0D117F041FD00283FF45FAF96F82605494905FB004051F88A
:20A38000302F484B04301A723C225AF07AFC96F826353E2205FB03433AE797F8263508FB50
:20A3A00003635B78062BA1D146F09CFA3A2308A903A80393434B984746F0A6FA97F82605A9
:20A3C000384B08FB0060099A09A91A72043010225AF057FC97F8263508FB03661223737045
:20A3E000D6E54FF48C762C4C2C4D94F8262506FB02525378062B7FF479AF334813F0F6FA3B
:20A40000A0E797F82635584333185B78062B7FF46DAFE97B043001393044224B254A042903
:20A4200034D8DFE801F00312181E2400D2F8282526491A7280225AF024FC4FF48C7297F8FB
:20A44000263502FB03668223C9E7D2F8A82520491A728022EFE7D2F828261E491A72802235
:20A46000E9E7D2F8A8261C491A728022E3E7D2F828291A491A7220225AF003FC4FF48C7241
:20A4800097F8263502FB03662223A8E7D2F8002213491A722022EFE7509A038040B40080CB
:20A4A0006C1A0010C01F00104080092001020304D09003806887038030890600F07F002081
:20A4C000EFCDABABF11FFF1F3E890600908C0380108D0380908D0380108E0380909003804C
:20A4E000688903804FF48C71C94BCA4A93F8263501FB03235B78062B7FF4F8AEC64B93F8BF
:20A500002120022A17D0032A12D0012A04D1C3494FF4E13011F070FF012011F0DDFE4FF0CC
:20A520008044AA26552512F0CDF8A660A560FAE70322BB49ECE7BB49EAE74FF48C71B44B4A
:20A54000B44A93F8263501FB03235B78062B7FF4CDAEB54C636959053FF51AAD0A2017F0AC
:20A56000C9FF63695A053FF513AD27F021FD63695B05FAD54FF40032AC4BAD48C3F8802008
:20A580004AF0C5FC4FF080404BF009FD4FF080431A6842F002021A60FF225A601A6842F0BD
:20A5A00001021A60AA229A6055229A60FEE74FF48C7897F8263508FB03635B78122B7FF4E5
:20A5C00095AE002105F10F0017F036F9044600287FF4B5AD97F8263508FB0366022343E5F2
:20A5E0004FF48C7297F8263502FB03635B781A2B7FF47CAE05F11F0017F030FA04464FF445
:20A60000FA6017F077FF002C7FF499AD012105F10F0017F011F9044600287FF490AD4FF4E1
:20A620008C7297F8263502FB0366D7E74FF48C71774E784F96F8262501FB02725278062AFF
:20A640007FF454AED5F80F0017F03CFA044608B1392474E5704BC6F8340593F8203013B95A
:20A66000012386F83E3572484AF051FC4FF48C7296F8263502FB0373C9E44FF48C71644F47
:20A68000644E97F8262501FB02625378062B7FF42DAED5F80F30B3F5007FBFF448AC6548FD
:20A6A0004FF00108B0F8684041201C44624B4FF0420A187203230D46DFF88091C4F308045B
:20A6C000537097F826050AFB049105FB008004304122083130445AF0D4FA97F8263508F1A4
:20A6E000410805FB03635A7801344132B8F1C40FC4F308045A70E4D14AE44FF48C73444D72
:20A70000444C95F826657343E2185778072F7FF6EDAD621DD15AE21D11F0070018BF012024
:20A72000D25A00EBD100504380B2073087427FF4DDAD4FF48C7707FB0640093323440079C5
:20A740003AF028FC00283FF4F2AB95F8263507FB0344022363701BE44FF48C702C4A2D4960
:20A7600092F8263500FB03135B78062B7FF4BEAD012382F866350BE494F8260503FB0063C1
:20A780005B78062B7FF4B2AD1DF0DCFE00287FF4CEAB94F826051DF0ADFE00283FF4C7ABAC
:20A7A0004FF48C730222102094F8261503FB01635A701DF0E7FFFFF7EBBB4FF48C7594F8B1
:20A7C000260505FB00635B78062B7FF48FAD1DF0B9FE00283FF4ABAB022394F826151120A6
:20A7E00005FB01656B70E4E7094B0A4A93F826054FF48C7303FB00235A78062A7FF476ADF4
:20A80000022201215A701DF067FFFFF770BB00BF509A038040B400806C1A0010000001401D
:20A8200000C00940008009404080092000E100E000400240F8860380C01F0010E88F05802E
:20A840004FF48C7230B5194B194C93F8260502FB004252780E2A25D1164AD3F814159568CB
:20A860008D4221D1157C03F21D515DB1D568C3F81455557C83F81C5532F8125F9278A3F8B7
:20A880001D558A700C4A93F81C350D88D3728B78158193724FF48C73062203FB00430020D7
:20A8A0005A7030BD7E20FCE74F20FAE7509A038040B40080A81E0010C01F001073B54FF4FF
:20A8C0008C701A4C1A4E94F8261500FB01614978052927D116F060FD054618B116F00AFD1F
:20A8E00002B070BD01460DF107002AF00DFDD8B1104818F0D3FE104A0020D369142B01BF9A
:20A900000E4BA3F89E50012382F87B304FF48C7294F8263502FB03639DF807201A71032215
:20A920005A70DDE77E20DBE74F20D9E7509A038040B400806C9A06006C1A0010801D0010CA
:20A940004FF48C722DE9F04F434C444E94F8263593B002FB03635B782746062B71D116F0FA
:20A960001BFD014630B116F0C5FC0446204613B0BDE8F08F0DF103002AF0C6FC002862D002
:20A98000374B1A7C9846012A5FD816F093FE10B917F008FFE9E7A47814B117F005FFE4E76A
:20A9A0003B780E2B53D00B3B012B50D92D4B5A7D1AB92D4A5278002A4BD11A7D42B3BA7A84
:20A9C00032B32A4A1B7F15780F33B5FBF3F54FF000094FF0130A0135DFF89CB0EDB20A2255
:20A9E00020210DF105008DF804A05AF04EF900230222594601A88DF80F3025F0CFFC08B965
:20AA00004B24B3E709F101095FFA89F39D42E6D898F81030022193B9154825F0FFFD0028E2
:20AA2000EED000234FF48C72BB7297F8263502FB03669DF8033033710323737096E70D4830
:20AA4000EBE77E2492E74F2490E733248EE773248CE74A248AE700BF509A038040B40080CA
:20AA6000A81E0010C3580680F88603800953068024E5060027E50600A2D506002DE9F04395
:20AA8000C7B0804616F088FC014618B116F032FC044617E04FF48C79584C594E94F82635F0
:20AAA000274609FB03635B78462B00F2A1800DF107002AF029FC002800F09C8023780E2B1C
:20AAC00004D17324204647B0BDE8F0834D4D2B7C23F07C0299072A7400F08E8016F0EAFD9A
:20AAE00010B917F05FFED3E7A47814B117F05CFECEE73B780B3B012BE3D917F0C7FD97F83D
:20AB0000263509FB03635B78063BDBB203F111022A443F2B31D941463B4809F0FBFE0446A0
:20AB2000002863D1394B9B7C63BB01234FF48C72BB7297F8263502FB03669DF807303371AE
:20AB40000323737024F0BCFFB0F5F97F02D3642017F0D0FC24F0B4FFB0F5FB7F03D94FF4CF
:20AB6000FA7017F0C7FC24F0ABFFB0F5FE7FA9D340F2DC5017F0BEFCA4E7013302F8014B21
:20AB8000DBB2C6E7224B5B78002BCED02B7C1A0615D4B8F1000F14BF1223172341221A4902
:20ABA00004A8ADF808305AF06CF802A805F07EFC05460028B9D017F095FD2C4682E7B8F12C
:20ABC000000F4FF02F028DF8103014BF02230123ADF808200F493F220DF112008DF81130B9
:20ABE0005AF04FF802A805F09FFEE1E70546E2E77E2467E74F2465E7332463E7509A0380EF
:20AC000040B40080A81E0010B81E0010C3580680F8860380B91E0010F0B5C7B03AF0AAF992
:20AC2000002814BF0925082516F0B6FB014618B116F060FB044619E04FF48C72524C534ED3
:20AC400094F82635274602FB03635B78472B00F296800DF107002AF057FB002800F0918056
:20AC60004B4B5A7CAA421D4603D93324204647B0F0BD002AF9D022780E2A01D17324F5E7D2
:20AC80001A7C22F07C0119749307EED016F012FD10B917F087FDCDE7A37813B117F084FD26
:20ACA000C8E723780B3B012BE8D917F0EFFC4FF48C72002194F8263502FB03635B78063B65
:20ACC000DBB203F111022A443F2B30D9314809F083FE0446002850D12F4B9B7C63BB0123A6
:20ACE0004FF48C72BB7297F8263502FB03669DF8073033710323737024F0E2FEB0F5F97F0C
:20AD000002D3642017F0F6FB24F0DAFEB0F5FB7F03D94FF4FA7017F0EDFB24F0D1FEB0F5D7
:20AD2000FE7FA3D340F2DC5017F0E4FB9EE7013302F8011BDBB2C7E7184B5B78002BCED0D3
:20AD400095F910304122002B4FF02F031149ADF8083004A80BDB59F094FF02A805F0A6FB41
:20AD600005460028BBD017F0BDFC2C467EE759F088FF02A805F0D8FDF2E70546F3E77E245A
:20AD800074E74F2472E700BF509A038040B40080A81E0010B81E0010C3580680F88603808E
:20ADA0002DE9F0418046C6B068B11E2305268DF8073016F0F1FAF0B116F09CFA04462046F1
:20ADC00046B0BDE8F0814FF48C71374B374A93F8263501FB03235B78062B5ED101460DF1A4
:20ADE00007002AF091FA002859D0314B1E7C002EDFD13324E3E716F05DFC10B917F0D2FC44
:20AE0000DCE7294DAB7813B117F0CEFCD6E72B78092B46D8012707FA03F313F4277F40D0B3
:20AE20000FF0B2FC15F062FF224B9DF80700187118F0D4F917F02AFC384605F0E3FA1923DF
:20AE400002A8ADF808308DF8106005F02FFB044600BB304628F0A6FF0446D8B9B8F1000F8C
:20AE600008D0154B93F89E3023B1384616F0D6FB28F03CFE0A2017F0F9FB4FF48C710B4A0C
:20AE800095F8263501FB03239DF807201A7103225A7094E717F026FC91E77E248FE74F24CB
:20AEA0008DE773248BE700BF509A038040B40080A81E0010F88603805E520680F7B54FF479
:20AEC0008C771C4D1C4E95F8263507FB03635B78052B29D116F060FA014628B116F00AFAC5
:20AEE0000446204603B0F0BD0DF107002AF00CFAE0B116F0DFFB10B917F054FCF0E7AC7891
:20AF000014B117F051FCEBE72B780A2B10D1012028F058FF95F826359DF8072007FB0363F1
:20AF20001A7103225A70DCE77E24DAE74F24D8E77324D6E7509A038040B400804FF48C72C9
:20AF40002DE9F041674C684F94F82635CAB002FB03735B7805463C3B3C2BA04600F2B9805F
:20AF600016F01AFA014630B116F0C4F9044620464AB0BDE8F0810DF117002AF0C5F90028F7
:20AF800000F0A98016F096FB10B917F00BFCEDE7A37813B117F008FCE8E7102D237816D1DE
:20AFA000082B40F09A80514E33780BB10FF0ECFB737823B3102D03D0F378AB4240F08F80C0
:20AFC00032799DF817309A421FD05924CFE7092B00F2838001229A4012F4657F7DD0082B5C
:20AFE000E1D0434AD27F012A07D1042B05D128F0BFFC04460028D6D0B9E7022BD1E79DF8B5
:20B0000017300120337105F0FDF99DF8170018F0E5F817F03BFB022D3DD032D8002D36D0F2
:20B02000012D3AD04FF48C7298F8263508A802FB03735B782F4A542B9EBF00219B1883F812
:20B04000341000232C4982F88830802259F019FE06A805F02BFA044618BB2946264807F027
:20B0600043FD0446E8B901234FF48C7288F80A3098F8263502FB037733793B7103237B70BB
:20B0800075E7032D0BD0102DCCD1842300E08023ADF81830C6E78223FAE78123F8E78323FC
:20B0A000F6E7164E17F01EFB96F8F631002B3FF45EAF002501230095CDE901352A462B4664
:20B0C0002946062013F044F886F8F65115F00EFE4DE77E244BE74F2449E7732447E75E24D4
:20B0E00045E700BF509A038040B40080F886038016530680A81E0010B81E00106887038066
:20B100004FF48C71F0B5304C304E94F82625C9B001FB026252782746062A4ED116F03CF9DF
:20B12000014618B116F0E6F849B0F0BD0DF10F002AF0EAF8002842D016F0BCFA10B917F0A6
:20B1400031FBF1E7A37813B117F02EFBECE72378022B36D11E4C23780BB10FF015FB9DF8D5
:20B160000F3001201B4D237105F04CF99DF80F0018F034F817F08AFA2B7C04A88DF81830B6
:20B180008D23ADF8103005F091F988B905F1100009F0DCFC60B901234FF48C72BB7297F849
:20B1A000263502FB036322791A7103225A70BBE7019017F097FA0198B6E77E20B4E74F2013
:20B1C000B2E77320B0E700BF509A038040B40080F8860380A81E00102DE9F0414FF48C78A7
:20B1E000414C424D94F82635C8B008FB03535B782646473B3C2B6DD816F0CEF8014630B11A
:20B2000016F078F80446204648B0BDE8F0810DF107002AF079F800285ED016F04BFA10B900
:20B2200017F0C0FAEEE7A47814B117F0BDFAE9E73378082B52D12E4B1A799DF807309A4254
:20B240004ED118F023F800284CD09DF8070017F0C5FF17F01BFA96F82635264F08FB03532E
:20B260005B78F0223B4483F87940852307F1100106A8ADF8103059F004FD04A805F016F9F8
:20B28000044620BB02A907F1100008F087FA0446E8B9082218480DEB020159F0F2FC002393
:20B2A0009DF80720B372154B1A724FF48C7296F8263502FB035508236B70114B93F8A23083
:20B2C000012B04BF15236B7017F0C4FF9BE717F009FA98E77E2496E74F2494E7732492E77A
:20B2E000592490E7D5248EE7509A038040B40080F8860380A81E0010D01F0010C01F001046
:20B300005E5206802DE9F0414FF48C78404C414D94F82635C8B008FB03535B7826467D33A8
:20B32000DBB23C2B69D816F037F8014630B115F0E1FF0446204648B0BDE8F0810DF10700D3
:20B3400029F0E2FF00285AD016F0B4F910B917F029FAEEE7A47814B117F026FAE9E73378A3
:20B36000082B4ED12C4B1A799DF807309A424AD117F08CFF002848D017F088F996F826356B
:20B38000264F08FB03535B78F0223B4483F83D408E2307F1100106A8ADF8103059F071FC80
:20B3A00004A805F083F8044620BB02A907F110000AF0DCFA0446E8B9082219480DEB020158
:20B3C00059F05FFC00239DF80720B372154B1A724FF48C7296F8263502FB035508236B7054
:20B3E000114B93F8A230012B04BF15236B7017F031FF9FE717F076F99CE77E249AE74F2446
:20B4000098E7732496E7592494E7D52492E700BF509A038040B40080F8860380A81E0010B8
:20B42000D01F0010C01F00105E5206804FF48C72F0B5424C424E94F82635C9B002FB036321
:20B440005B782746252B70D115F0A6FF014618B115F050FF49B0F0BD0DF10F0029F054FFEE
:20B46000002864D016F026F910B917F09BF9F1E7A37813B117F098F9ECE742F20E72314C94
:20B48000E38D013B9BB2934253D83B78092B52D8012505FA03F313F4277F4CD00FF074F952
:20B4A00015F024FC9DF80F20274B10341A7117F0EDF8284604F0A6FF18230DEB0305ADF88F
:20B4C00010300FCC0FC594E80F0085E80F0004A804F0ECFF20BB9DF80F0017F07FFEA4F153
:20B4E00010000AF0E9F9D8B9012342F20F740021164ABB729DF80F30F9701372144BB3F87A
:20B50000303101339BB2A34294BF538151814FF48C7297F8263502FB03660523737099E74F
:20B52000019017F0DFF8019894E77E2092E74F2090E733208EE773208CE700BF509A038091
:20B5400040B40080A81E0010F8860380C01F0010E02506807FB54FF48C76204D204C95F847
:20B56000263506FB03435B78063B012B32D815F013FF014618B115F0BDFE04B070BD0DF119
:20B58000070029F0C1FE38B395F82635154A06FB03435B78118A062B18D1C9B202A8118213
:20B5A00027F0A4FE0028E8D10F499DF8073000200B72DDE90223C1E904234FF48C7295F8A6
:20B5C000263502FB034409236370D6E702A827F09DFEE7E77E20D0E74F20CEE7509A038000
:20B5E00040B40080A81E0010C01F001073B54FF48C75184E184C96F8263505FB03435B78DA
:20B60000062B22D115F0C8FE014618B115F072FE02B070BD0DF1050029F076FEB8B10F4B84
:20B620000DF10600197C27F027FE0028F0D10C4B9DF805201A72BDF806205A81052296F844
:20B64000263505FB03435A70E2E77E20E0E74F20DEE700BF509A038040B40080A81E0010A7
:20B66000C01F00102DE9F341054615F095FE18B115F040FE05460CE0E5B14FF48C71814BC9
:20B68000814A93F8263501FB03235B78092B04D07E25284602B0BDE8F0817C4B1E7C1C7D29
:20B6A0005F8A1E210DF1070029F02EFE002843D14F25EEE715F0FEFF10B917F073F8D9E796
:20B6C0004FF48C706F49704A91F8263500FB03235A78892ADCD86D4A167C147D0A2E578A88
:20B6E000DFD1D3F80C21D1F818359A42E0D1684B9A5D1AB3B21D03EB8203D3F80280B8F849
:20B700000130BB42C0F0B080002F00F0AD8098F80330A342C0F0A880002C00F0A580002DE1
:20B720006CD0172E49D1A4F10F03042B45D8DFE803F00720442633001A2ED8D95D25A8E7F3
:20B740000024544D544E554F301915F8012B394602345AF08FFE802CF6D14FF48C71494B89
:20B76000494A93F8263501FB032382225A7000258FE780222D21484859F087FAEDE7464879
:20B7800022F010FE4FF48C713E4B3F4A93F8263501FB03237A22E9E7414A424953683E486C
:20B7A00052785AF067FE4FF48C71364B364A93F8263501FB03230622D8E7013CE5B2013FCC
:20B7C0003A46294630462AF0BDF900233A46294630462AF067F90E2303FB04840146E27BD7
:20B7E0002D4859F04EFA4FF48C71264B264A93F8263501FB0323E27B0232B7E73A46214604
:20B8000030462AF061FE054600287FF442AF264B3A46214630462AF017FC054600287FF481
:20B8200038AF012E11D1304626F00AFF26F016FB0EF0AAFF4FF48C71124B134A93F82635CD
:20B8400001FB032302225A7023E7112EF0D1013CE4B2132C0AD8122CEAD2022CE8D0E9D33E
:20B86000083C052CE6D8E3E7332512E71A2CDFD004D8162CDCD0182CDCD1D9E7263C012C7B
:20B88000F0E700BF509A038040B40080A81E001050030010E81A0010C81F0010548906000C
:20B8A000209A038050890600BD1E0010F7B54FF48C771A4D1A4E95F8263507FB03635B789D
:20B8C000052B24D115F068FD044618B115F012FD03B0F0BD1E210DF1070029F015FDC0B172
:20B8E0002B78042B17D1012029F038FD204626F0A7FE204617F036F995F826359DF80720BE
:20B9000007FB03631A71022220465A70E0E77E20DEE74F20DCE77320DAE700BF509A038004
:20B9200040B400802DE9F7434FF48C71324C334D94F82625264601FB02525278072A53D153
:20B9400015F02AFD014630B115F0D4FC0446204603B0BDE8F0830DF1070029F0D5FC00282C
:20B9600044D023780E2B43D00B3B012B40D9244B1A7C984602F003021A749AB35B7C8BB377
:20B9800015F098FE10B916F00DFFDFE7A47814B116F00AFFDAE71B4B5B785BBB16F076FEF1
:20B9A0000027DFF8649098F81120FBB29A424FF000030CD84FF48C72B37296F8263502FBD9
:20B9C00003539DF807201A7103225A70BFE798F8102049460C4824F0E1FC01370028E2D18E
:20B9E00016F080FE3324B2E77E24B0E74F24AEE77324ACE74A24AAE7509A038040B4008088
:20BA0000A81E0010F88603809FD50600F7B54FF48C76164F164D97F8263506FB03535B7808
:20BA2000062B1DD1134B1C7CE4B915F0B5FC28B115F060FC0446204603B0F0BD21460DF1EF
:20BA4000070029F061FC78B126F0C6FC97F826359DF8072006FB03531A7103225A70EAE720
:20BA60007E24E8E73324E6E74F24E4E7509A038040B40080A81E00104FF48C712DE9F041B5
:20BA8000444C454E94F8262592B001FB026252782746052A74D115F07FFC014620B115F0C2
:20BAA00029FC12B0BDE8F0810DF1070029F02CFC002867D015F0FEFD10B916F073FEF0E7CD
:20BAC000A278052A06D80123934013F0340F5BD19B075BD13B78062B5AD0012B58D0002185
:20BAE00005222E4DBA7029726971E97911B96A7A02B9FA70082B31D10F2329490DF10900F0
:20BB00008DF808305BF038FC264900230222084624F044FC00230222224902A824F03EFCE7
:20BB20000624DFF880800023022241461D4824F035FC70B1013C14F0FF04F4D11A4B9B79E9
:20BB4000012B08D0022B09D10321184824F066FD20B94B20A5E703211548F7E70020154B30
:20BB60004FF48C7258800123AB7697F82635687002FB03639DF807201A7103225A7090E795
:20BB80007E208EE74F208CE750208AE7722088E7732086E7509A038040B40080F8860380EC
:20BBA000C2D906009FD50600C358068027E5060024E50600105803802DE9F3414FF48C762E
:20BBC0001F4F204D97F8263506FB03535B78062B30D115F0E1FB044620B115F08BFB02B00B
:20BBE000BDE8F0811E210DF1070029F08DFB18B3154B1B7C1A2B21D8144AD15CF1B10633E4
:20BC000002EB8303D3F802802822D8F8041010485BF024FCB8F801200E4B20461A8698F8B3
:20BC2000032083F832202D2297F8263506FB03535A70D4E77E20D2E74F20D0E75D20CEE750
:20BC4000509A038040B40080A81E001050030010C81F0010C01F00104FF48C722DE9F34753
:20BC6000344F354E97F8263502FB03635B78072B58D115F091FB804620B115F03BFB02B02E
:20BC8000BDE8F0871E210DF1070029F03DFB00284AD02A490B7C1A2B48D8294AD05C00288B
:20BCA00044D0063302EB8303D3F80290497C99F803300139C9B28B423AD94FF00E0A0AFBED
:20BCC00001FA09EB0A04D4F80A1028221D485BF0C5FB1D4DA37B323505F8023CE47B05F841
:20BCE000014CC3B90AF1100122464944284658F0C8FF0AF1140122464944281958F0C1FFAF
:20BD00004FF48C7297F82635163402FB0366640074700020B3E780224146284658F0B5FFB3
:20BD20000124EDE77E20AAE74F20A8E75D20A6E73320A4E7509A038040B40080A81E00103E
:20BD400050030010C81F0010C01F00102DE9FF414FF48C762E4C2F4D94F82635074606FBD4
:20BD600003535B78363B3C2B49D815F015FB014620B115F0BFFA04B0BDE8F0810DF10F00DF
:20BD800029F0C2FA00283CD015F094FC10B916F009FDF0E794F80280B8F1000F02D016F0BB
:20BDA00003FDE8E72378082B2DD11B4B1A799DF80F309A4229D116F069FCA7F10A03012B09
:20BDC00017D994F82635154806FB03535B7839460344103083F8108008F0BEFF50B994F8AA
:20BDE00026359DF80F2006FB03531A7103225A70C1E73720019016F075FC0198BBE77E2073
:20BE0000B9E74F20B7E77320B5E75920B3E700BF509A038040B40080F8860380A81E0010BC
:20BE20004FF48C7170B52E4D2E4E95F82625C8B001FB026252782C46052A47D115F0ACFAC8
:20BE4000014618B115F056FA48B070BD0DF10F0029F05AFA00283BD0234B93F84E3053B130
:20BE600015F028FC10B916F09DFCEDE7AB7813B116F09AFCE8E72278082A01D00D2A29D13D
:20BE80001A4A937A43BB12799DF80F309A4225D116F0FCFB882304A8ADF8103004F006FBD4
:20BEA00078B907F0EBFB60B94FF48C7294F82635A07202FB03639DF80F201A7103225A7080
:20BEC000C2E7019016F00EFC0198BDE77E20BBE74F20B9E77320B7E75020B5E75920B3E73C
:20BEE000509A038040B400805E520680F886038073B54FF48C711E4C1E4D94F826252646AA
:20BF000001FB02525278052A2AD115F045FA014618B115F0EFF902B070BD0DF1070029F09F
:20BF2000F3F9F8B12278082A01D00D2A1CD112499DF807300A799A4218D1082210310F487A
:20BF400058F09FFE9DF807200D4B00201A724FF48C7296F8263502FB035308225A70DAE70A
:20BF60007E20D8E74F20D6E77320D4E75920D2E7509A038040B40080F8860380D01F0010D7
:20BF8000C01F00104FF48C72F0B53A4E3A4C96F82635C9B002FB03435B7807460A2B354649
:20BFA00062D115F0F9F9014618B115F0A3F949B0F0BD0DF10F0029F0A7F9002856D015F0E7
:20BFC00079FB10B916F0EEFBF1E7B37813B116F0EBFBECE73378092B4AD8012606FA03F391
:20BFE00013F4277F44D00EF0CFFB14F07FFE234B9DF80F00187117F0F1F816F047FB3046EE
:20C0000004F000FA0C2F14BF512350231C4E04A8ADF81030D6E90423CDE9062304F046FA49
:20C02000E8B9394606F1100008F018FDB8B942F20F71144A9DF80F301372134BB3F8303186
:20C0400001339BB28B4294BF538150814FF48C7295F8263502FB034405236370A7E7019013
:20C0600016F040FB0198A2E77E20A0E74F209EE773209CE7509A038040B40080F88603804C
:20C08000A81E0010C01F0010E025068070B54FF48C76294C294D94F82635C8B006FB035345
:20C0A0005B78052B41D115F077F918B115F022F948B070BD1E210DF10F0029F025F9B0B302
:20C0C00015F0F8FA10B916F06DFBF1E7A37813B116F06AFBECE72378042B2AD10EF054FB2B
:20C0E00014F004FE164B9DF80F201A7116F0CEFA012004F087F9272304A8ADF8103004F058
:20C10000D5F968B99DF80F0017F068F808F06AFF30B9022294F8263506FB03535A70C7E701
:20C12000019016F0DFFA0198C2E77E20C0E74F20BEE77320BCE700BF509A038040B400801E
:20C14000F88603804FF48C7110B50C4B0C4A93F82635044601FB03235B78052B0BD115F0F6
:20C160001BF918B1BDE8104015F0C4B82046BDE81040FDF707BA7E2010BD00BF509A0380C5
:20C1800040B400802DE9F0414FF48C782F4D304C95F82625274608FB024253782E46062BA9
:20C1A0004ED115F0F9F818B1BDE8F04115F0A2B895F8263508FB0343D3F80C21D5F8183529
:20C1C0009A423FD116F08CFBAC781CB1BDE8F04116F0EABA29784B1EDBB20A2B06D80122A8
:20C1E00002FA03F340F2816213422DD1194B1A7C062A05D0072A1FD033242046BDE8F081F3
:20C200004FF47050144BD881134B14481A730022DD891A8273780581012086F8283586F80D
:20C22000271516F023FA4FF48C7296F8263502FB037304225A70E0E7074B4FF48040E2E72D
:20C240007E24DAE74F24D8E77324D6E7509A038040B40080A81E00106C1A0010C01F0010B9
:20C260002DE9F0434FF48C79464C474D94F82625D5B009FB025253782F46052BA0467BD1B1
:20C2800015F08AF8064620B115F034F855B0BDE8F08394F8263509FB0353D3F80C21D4F8A7
:20C2A00018359A426AD116F01BFB2578012D67D1364C237B218A062B4FEA411103D0072B6F
:20C2C00040D03320E2E706AE202201F50041304658F0D7FC94F82090B9F1000F17D0202355
:20C2E0002B4A314647F210000FF068FF294B227B00201A72228A511C5A814FF48C7298F821
:20C300002635218202FB037325225A70BEE70EA81DF035FC4FF480721F490EA81DF03EFC68
:20C320001022494602A858F0B0FC194BCDE9006302AB202229460EA81EF03FF80EA81DF005
:20C3400023FCD3E70DF11809202201F10041484658F097FC0EA81DF012FC4FF480720E49AA
:20C360000EA81DF01BFC1022314602A858F08DFC074BCDE90093DBE77E2087E74F2085E77B
:20C38000732083E7509A038040B400806C1A0010CC1F0010C01F0010598906002DE9F04110
:20C3A0004FF48C78224C234F94F826253E4608FB027253782546052B31D114F0EDFF18B163
:20C3C000BDE8F04114F096BF94F8263508FB0373D3F80C21D4F818359A4222D116F080FA6E
:20C3E0002378012B04D0052B1DD16378012B1AD1114B1B7B03F0FD03FC2B16D04FF48C725F
:20C4000095F8273500202B7095F828356B7095F8263502FB036302225A70BDE8F0817E20C6
:20C42000FBE74F20F9E77320F7E73320F5E700BF509A038040B400806C1A0010F0B54FF40D
:20C440008C762E4C2E4D94F82635C9B006FB03535B78052B4CD114F09FFF18B114F04AFF56
:20C4600049B0F0BD1D210DF10F0028F04DFF002840D015F01FF910B916F094F9F0E7A378C4
:20C4800013B116F091F9EBE72378092B34D8012707FA03F313F4277F2ED00EF075F914F061
:20C4A00025FC184B9DF80F201A7116F0EFF8384603F0A8FF2C2304A8ADF8103003F0F6FFDC
:20C4C0000028CDD19DF80F0016F088FE04F038FE20B1019016F006F90198C1E794F82635AD
:20C4E0009DF80F2006FB03531A7103225A70B7E77E20B5E74F20B3E77320B1E7509A03802E
:20C5000040B40080F8860380F7B54FF48C71294D294C95F826252E4601FB02425278052A4A
:20C520003DD114F039FF014618B114F0E3FE03B0F0BD0DF1070028F0E7FE90B31F4B1A781B
:20C540001F4682B31A799DF807309A422DD115F0B1F810B916F026F9E9E7A87810B116F0B5
:20C5600023F9E4E72A780F2A05D8012393404EF2020213421BD1052200210123B270104AB8
:20C58000BB7151804FF48C72BB7696F8263502FB03439DF807201A7103225A70C7E77E207E
:20C5A000C5E74F20C3E75620C1E75920BFE77320BDE700BF509A038040B40080F8860380A1
:20C5C0001058038070B54FF48C762B4C2B4D94F82635C8B006FB03535B78052B46D114F043
:20C5E000DBFE18B114F086FE48B070BD1D210DF10F0028F089FE00283AD015F05BF810B9AF
:20C6000016F0D0F8F0E7A37813B116F0CDF8EBE72378023B012B2DD80EF0B6F814F066FBDF
:20C62000174B9DF80F201A7116F030F8012003F0E9FE422304A8ADF8103003F037FF80B9C8
:20C640009DF80F0016F0CAFD08F0D0FD48B994F826359DF80F2006FB03531A7103225A7027
:20C66000C2E7019016F03EF80198BDE77E20BBE74F20B9E77320B7E7509A038040B40080A6
:20C68000F88603802DE9F74F38F074FC384B394DDA69394B002814BF4FF009084FF008083B
:20C6A000122A08BF1D464FF48C72344F344E97F8263502FB03635B78062B52D114F06CFEEC
:20C6C00020B114F017FE03B0BDE8F08F1D210DF1070028F019FE002845D0DFF8B49099F83E
:20C6E0001000404541D800283FD00928254CDFF8A4A017D1244A9AF81C30907801330344E1
:20C700001188E3721389A1724B434FF48C72238197F8263584F80C8002FB03660723002067
:20C720007370D0E76FF0004B00EB0B0315F81330A3720EF013FE99F810305B4405EB4305A0
:20C74000697832F0D7F99AF81C3099F81020013318440E4BE072134413F8013CA27A5343DB
:20C76000D3E77E20AFE74F20ADE73320ABE700BF6C1A0010BCD5060013410700509A03802F
:20C7800040B40080C01F0010D80E0780601E0010A81E0010C358068070B54FF48C762B4CE3
:20C7A0002B4D94F82635C8B006FB03535B78052B46D114F0F1FD18B114F09CFD48B070BDB4
:20C7C0001D210DF10F0028F09FFD00283AD014F071FF10B915F0E6FFF0E7A37813B115F046
:20C7E000E3FFEBE72378023B012B2DD80DF0CCFF14F07CFA174B9DF80F201A7115F046FF3F
:20C80000012003F0FFFD432304A8ADF8103003F04DFE80B99DF80F0016F0E0FC09F0A8F87B
:20C8200048B994F826359DF80F2006FB03531A7103225A70C2E7019015F054FF0198BDE7AC
:20C840007E20BBE74F20B9E77320B7E7509A038040B40080F88603804FF48C72F0B52C4C18
:20C860002C4D94F82635C7B002FB03535B7827460A2B48D114F090FD014628B114F03AFD14
:20C880000446204647B0F0BD0DF1070028F03CFD00283AD014F00EFF10B915F083FFEFE785
:20C8A000A37813B115F080FFEAE71B4E15F0EEFE304604F0A1FB044610BB184B9B7C6BB931
:20C8C0004FF48C7297F8263502FB03559DF807302B7103236B700123BB72D2E7104B5B7837
:20C8E000002BEDD096E80300C223049002A8ADF808308DF8141003F0D9FD0028E0D004463B
:20C9000015F0F0FEBDE77E24BBE74F24B9E700BF509A038040B40080B81E0010C358068002
:20C92000F8860380F7B54FF48C711C4E1C4D96F8262501FB025252782E2A2BD114F02CFDC3
:20C94000044618B114F0D6FC03B0F0BD01460DF1070028F0D9FCF8B12827124B1248197C11
:20C96000124A07FB010120461160113313F8014B11680C5401302828F8D14FF48C7296F8F3
:20C980002635002002FB03539DF807201A7103225A70D9E77E20D7E74F20D5E7509A0380DF
:20C9A00040B40080A81E00106CA003806809001070B54FF48C76124C124D94F8262506FB1E
:20C9C00002525378092B16D114F0E6FC18B1BDE8704014F08FBC0C4BD4F818259968914296
:20C9E0000BD10222DB68C4F8183594F8263506FB03535A7070BD7E20FCE74F20FAE700BF26
:20CA0000509A038040B40080A81E00104FF48C72F0B5474C474D94F82635C9B002FB03539F
:20CA20005B782646052B7AD114F0B6FC014628B114F060FC0446204649B0F0BD0DF10700AB
:20CA400028F062FC00286CD014F034FE10B915F0A9FEEFE72378042B01D0072B63D1B3784F
:20CA600013B115F0A1FEE5E716F010FC00285CD00DF08AFE15F00AFE012003F0C3FCE023B4
:20CA800004A8ADF8103003F011FD0446002843D19DF8070016F0A2FB9DF80720264B1A7187
:20CAA00004F0A2FB0446B8BB4FF48C77012396F826059DF807207843B3722B181A71032276
:20CAC0005A701E4B93F8A230012B22D1053004221B49284458F0D5F896F82605042207FB86
:20CAE00000501849093058F0CCF8174902A812F0C1FC96F82605052207FB005002A90D305D
:20CB000058F0BFF896F8263507FB03556B780D336B7016F09FFB8EE715F0E4FD8BE77E24C6
:20CB200089E74F2487E7732485E7D52483E700BF509A038040B40080F88603805E52068067
:20CB40009C890380A0890380888703802DE9F0414FF48C74464D474E95F82635C8B004FBDE
:20CB600003635B7880460A2B2F4604D97E24204648B0BDE8F08114F00FFC014618B114F0F6
:20CB8000B9FB0446F3E70DF1070028F0BDFB00286AD014F08FFD10B915F004FEF1E7AB782B
:20CBA00013B115F001FEECE715F070FD95F8263504FB03635B78B8F1000F23D1072BD5D1C4
:20CBC0002D4B1A7C5B7CADF80820ADF80A30022302AD28468DF80C3024F07CFC04460028C3
:20CBE00040D1264B9B7CFBB901234FF48C72BB7297F8263502FB03669DF807303371032370
:20CC00007370B4E71E4A92F89820012A0AD10A2BACD1194B5A8AB2F5BE6F27D81A691B7DFE
:20CC20000292D5E7092BF3E7164B5B78002BDBD095F90430002B4FF0C103ADF8103095E83A
:20CC400003000690ADF81C1004A808DB03F02EFC05460028C8D015F045FD2C4687E703F099
:20CC600063FEF5E70546F6E74F2480E733247EE7509A038040B40080A81E0010C358068061
:20CC80005E520680F8860380F7B54FF48C711F4E1F4D96F8262501FB025252782F2A2ED14D
:20CCA00014F07AFB044618B114F024FB03B0F0BD01460DF1070028F027FB10B3154B198A19
:20CCC000B1F5BE6F1FD228271348144A07FB010120461160123313F8014B11680C54013007
:20CCE0002828F8D14FF48C7296F82635002002FB03539DF807201A7103225A70D6E77E20ED
:20CD0000D4E74F20D2E73320D0E700BF509A038040B40080A81E00106CA0038068090010A0
:20CD2000F0B54FF48C743E4D3E4E95F82635DBB004FB03635A783C4B2F461B68DB080833AD
:20CD40009A4269D814F028FB014628B114F0D2FA044620465BB0F0BD0DF1030028F0D4FA50
:20CD600000285BD014F0A6FC10B915F01BFDEFE7AD7815B115F018FDEAE715F087FC54222A
:20CD8000294601A857F081FF28490DF107000B8A1331ADF8043011F8013C8DF8063097F8FC
:20CDA000263504FB03635A78083A57F06AFF502101A804F057F9044660BB1D4B9B7C43B9B1
:20CDC0004FF48C7297F8263502FB036603237370BFE7184B5B78002BF2D09DF906305422AE
:20CDE000002B4FF0C50301A9ADF8583018A80BDB57F047FF16A803F059FB05460028DFD0D0
:20CE000015F070FC2C46A4E757F03BFF16A803F08BFDF2E70546F3E77E249AE74F2498E7D7
:20CE2000509A038040B400803C1E0010A81E0010C3580680F8860380F7B54FF48C771B4DD5
:20CE40001B4E95F8263507FB03635B78052B26D114F0A2FA014628B114F04CFA0446204665
:20CE600003B0F0BD0DF1070028F04EFAC8B114F021FC10B915F096FCF0E7AC7814B115F02E
:20CE800093FCEBE70B4B5B786BB902200EF072FA032295F8263507FB03635A70DFE77E24B1
:20CEA000DDE74F24DBE74A24D9E700BF509A038040B40080F886038073B54FF48C71294CCD
:20CEC000294D94F82625264601FB02525278062A42D114F061FA014628B114F00BFA04466A
:20CEE000204602B070BD0DF1070028F00DFAA8B314F0E0FB10B915F055FCF0E7A47814B1B8
:20CF000015F052FCEBE7194B5B784BBB184A194B127C9B79AAB1012B0FD053B1022B0ED0D2
:20CF20004FF48C7296F8263502FB035303225A70D6E704200EF01EFAF2E72046FAE701204D
:20CF4000F8E7012B06D01BB1022BE9D10620F1E70220EFE70520EDE77E24C1E74F24BFE7EB
:20CF60004A24BDE7509A038040B40080F8860380A81E0010C3580680F7B54FF48C771A4DED
:20CF80001A4E95F8263507FB03635B78052B25D114F002FA014628B114F0ACF90446204667
:20CFA00003B0F0BD0DF1070028F0AEF9C0B114F081FB10B915F0F6FBF0E7AC7814B115F0D8
:20CFC000F3FBEBE70A4B5B7863B90EF029FC032295F8263507FB03635A70E0E77E24DEE7BD
:20CFE0004F24DCE74A24DAE7509A038040B40080F886038037B54FF48C72304D304C95F837
:20D00000263502FB03435B78083B3F2B52D814F0C3F9014618B114F06DF903B030BD0DF1F0
:20D02000070028F071F9002846D0264B1A7C012A20D01AB1FA2A2DD03320EEE7597C0A060E
:20D04000FAD4214A123302EB8112511E3F3213F8010B01F8010F9142F9D14FF48C7295F867
:20D060002635002002FB03449DF80730237103236370D2E7597C0F29DED8144A123302EB8C
:20D080008112511E3F3213F8010B01F8010F9142F9D1E2E7597C0329CED80D4A123302EB67
:20D0A0008112511E3F3213F8010B01F8010F9142F9D1D2E77E20B0E74F20AEE7509A0380E1
:20D0C00040B40080A81E0010D7EE068020960380680800104FF48C72F0B5464C464E94F86A
:20D0E0002635C7B002FB03635B7827460F2B7AD814F052F9014628B114F0FCF80446204618
:20D1000047B0F0BD0DF1070028F0FEF800286CD014F0D0FA10B915F045FBEFE7A37813B163
:20D1200015F042FBEAE715F0B1FA344BDB690A2B1FD0334B1A7C432A02D031D8032A56D195
:20D1400041F6B132598A914251D89A7E022A4ED893F91420002A4ADB5A7D282A47D89A7DFE
:20D16000082A44D85A7E032A41D8DB7D033B052B3DD8244D284603F0A5FF044688BB224BF8
:20D180009B7C8BB94FF48C7297F8263502FB03669DF807303371032373700123BB72AEE744
:20D1A000832ACDD0C32ACAE7184B5B78002BE9D0DE222B78ADF8082013F0400F04AB95E87F
:20D1C000070083E8070002A808D103F06FF905460028D7D015F086FA2C4690E703F0A4FBDE
:20D1E000F5E70546F6E77E2489E74F2487E7332485E700BF509A038040B400806C1A00103F
:20D20000A81E0010B81E0010C3580680F886038070B54FF48C762B4C2B4D94F82635C8B0F8
:20D2200006FB03535B78052B46D114F0B5F818B114F060F848B070BD1D210DF10F0028F01F
:20D2400063F800283AD014F035FA10B915F0AAFAF0E7A37813B115F0A7FAEBE72378023B96
:20D26000012B2DD80DF090FA13F040FD174B9DF80F201A7115F00AFA012003F0C3F84423C6
:20D2800004A8ADF8103003F011F980B99DF80F0015F0A4FF08F0C2FB48B994F826359DF849
:20D2A0000F2006FB03531A7103225A70C2E7019015F018FA0198BDE77E20BBE74F20B9E791
:20D2C0007320B7E7509A038040B40080F88603802DE9F0434FF48C78554E564F96F826357A
:20D2E0008BB008FB03735B78022B40F09C80524B1B7A012B40F0998028220021684657F027
:20D30000C4FC4E4B4E48DB699DF80320073B18BF012390F8981063F382024B1E594259413D
:20D320009DF804308DF8032061F345138DF80430444B4FF000095A789DF80530B2FA82F284
:20D34000520962F3041361F345138DF805303E4A009B6C461A403D4B3D4D13430093019BDA
:20D3600090F8A22023F47333511E23F400734A4243F498434A410193C3F3074362F3820316
:20D380008DF8063015F056FF9DF8063060F3C30396F826058DF806301BF0ACF89DF80630A6
:20D3A00060F3041396F826058DF806301BF0A2F89DF806308DF80E9060F345138DF8063096
:20D3C000BDF806301E206FF38F13ADF80630214BCDF8109002931023ADF80C301E4BCDE9AC
:20D3E000050324F0D3FE40238DF81D3040F2B633ADF81E3041F21233C008ADF820308DF843
:20D400001C000FCC0FC50FCC0FC594E8030096F8263585E8030008FB0377232348467B707E
:20D420000BB0BDE8F0837E20FAE73320F8E700BF509A038040B40080A81E00106C1A00105C
:20D440005E520680B6510680A547BFF45AA04003C81F00100C18010C0006FF002DE9F743B0
:20D460004FF48C77DFF8A880264E98F8263507FB036393F80190B9F1050F3DD100210DF199
:20D48000070027F041FFC8B31F4B93F82450BDBB284642F077F81D4C6072012042F072F8CB
:20D4A000A072022042F06EF8E072032042F06AF82073042042F066F86073484642F062F863
:20D4C000A073062042F05EF8E073072042F05AF8207422F0F5FAB0FA80F00C224009607493
:20D4E00028469DF80730237298F8263507FB03635A7003B0BDE8F0837E20FAE74F20F8E7A8
:20D50000C820F6E740B400806C1A0010C01F0010509A03804FF48C72F0B5694E694F96F8FD
:20D5200026359DB002FB03735B78052B40F0C18000210DF1070027F0E7FE002800F0BB80E7
:20D54000614B93F82430002B40F0B7805F4C02A802AD26F0B1FB0FCD0FC495E80F0084E841
:20D560000F003378103C022B1ED10AA902A826F0FBFB13A904F1600026F0F6FB0AA859F00D
:20D58000C3FF054613A859F0BFFF514B281ADA796FF03B03534303F5A83303F5C073984280
:20D5A00002D9032015F062F894F88020B4F884300AB1013B9BB2474D00202B82E369EB7234
:20D5C000A369AB72E3686B72A3682B7363686B732368AB73E36F85F82230A36F85F82130FE
:20D5E000E36E85F82030A36E85F82330636E85F82430236E85F82530374BD3F872216A617C
:20D60000D3F82021AA61D3F8242103F52963EA61D3E90023C5E90A2341F0B4FF85F83000C9
:20D62000012041F0AFFF85F83100022041F0AAFF85F83200032041F0A5FF85F833000420C5
:20D6400041F0A0FF85F83400052041F09BFF85F83500062041F096FF85F83600072041F0B0
:20D6600091FF94F880303278002B0CBF00230823032A94F8642185F8370008BF43F01003F1
:20D680000AB143F0060394F8B2200020FF2A4FF48C7218BF43F0010385F838309DF80730EC
:20D6A0002B7296F8263502FB03772C237B701DB0F0BD7E20FBE74F20F9E7C820F7E700BF65
:20D6C000509A038040B400806C1A0010688703805E520680C01F0010E02506802DE9F74361
:20D6E0004FF48C71344A354F92F82635904601FB03735B78FF2B59D013F04EFE064620B129
:20D7000013F0F8FD03B0BDE8F08301460DF1070027F0FAFD00284BD0294CA37D012B49D1CE
:20D72000237C013B3F2B45D8A28A531EFD2B41D8638A002B3ED0134440F2B632934239DC28
:20D74000204B35469946204A1A60608AD9F800302844013803EB80104022002157F095FAB9
:20D760000023217C9A199942D2B212D80135A38AEDB2AB421646E8D84FF48C7298F82635B6
:20D78000002002FB03779DF807303B7103237B70B8E72244D07D628AD9F800102A44013AA1
:20D7A00001EB8212D0540133DBB2DAE77E20A9E74F20A7E73320A5E7509A038040B4008058
:20D7C000A81E0010680900106CA003804FF48C72F0B5384C384E94F82635C7B002FB0363B2
:20D7E0005B7827460C2B5FD113F0D6FD014628B113F080FD0446204647B0F0BD0DF10700B3
:20D8000027F082FD002851D013F054FF10B914F0C9FFEFE7A37813B114F0C6FFEAE7274D7B
:20D8200014F034FF2B8A002B42D040F2B5326B8A013B9BB293423BD805F1100023F076FEB3
:20D8400005F11002044668BB1D4B9B7C6BB901234FF48C72BB7297F8263502FB03669DF839
:20D860000730337103237370C5E7164B5B78002BEDD04D2195F91630ADF80810002B04AB23
:20D8800092E8030083E8030002A808DB02F00EFE05460028DBD014F025FF2C46ABE703F0D5
:20D8A00043F8F5E70546F6E77E24A4E74F24A2E73324A0E7509A038040B40080A81E00106B
:20D8C000C3580680F886038070B54FF48C76254C254D94F82635C8B006FB03535B78052BA0
:20D8E0003AD113F059FD18B113F004FD48B070BD1D210DF10F0027F007FD78B3A37813B162
:20D9000014F052FFF2E72378023B022B28D80CF03BFF164B9DF80F201A7114F0B7FE012014
:20D9200002F070FDC72304A8ADF8103002F0BEFD68B925F0E1FE50B99DF80F200C4B1A729B
:20D94000032294F8263506FB03535A70CEE7019014F0C8FE0198C9E77E20C7E74F20C5E7DA
:20D960007320C3E7509A038040B40080F8860380C01F001010B520F06BFB431C02D17B248D
:20D98000204610BD632811DD25F07CFF0028F6D025F09AFE0322064B12209A71FEF7D2FB3B
:20D9A00004460028ECD025F0D1FEE9E74B24E7E75E520680F0B5E9B01E210DF1050027F07B
:20D9C000A3FC002874D013F075FE28B914F0EAFE0446204669B0F0BD384DAB7813B114F013
:20D9E000E3FEF5E72B78022B64D115F04FFC002862D04FF48C7795F82615314E7943083139
:20DA0000314430481AF068F90CF0BEFE14F03EFE9DF805202C4B01201A7102F0F3FC4FF4B5
:20DA20009B737022274926A8ADF8903057F029F924A802F03BFD04460028CAD10DF1060231
:20DA400004A920480BF07EFA04460028C1D195F82605BDF8062007FB006004A9053057F01C
:20DA600010F995F826359DF8062007FB036303325A70164B93F8A230012B16D1144902A8BB
:20DA800011F0F8FCBDF8063095F82605053307FB00300522304402A957F0F3F895F8263524
:20DAA00007FB036673780533737015F0D3FB90E74F248EE773248CE7D5248AE7509A0380E2
:20DAC00040B40080B81E0010F88603805E52068088870380802301210022F0B5CBB00DF11E
:20DAE0001607CDE9003102972AAB1146302010F02FFB0446002843D110AB2AAA39883020BD
:20DB000010F002F89DF84130002B5AD12E4D08A808AC26F0D1F80FCC0FC594E80F0005F1C1
:20DB200010060DF1200C85E80F00BCE80F000FC694E80F0086E80F00244E3378022B22D15C
:20DB400018A908A826F010F921A905F1500026F00BF918A859F0D8FC044621A859F0D4FC02
:20DB60001B4B201ADA796FF03B03534303F5A83303F5C073984206D9032014F077FD1624F3
:20DB800020464BB0F0BD08A906A811F073FC002301220297CDE9003206A90522172010F0D4
:20DBA000D7FA04460028EBD113F0A0F84FF48C71084A96F8263501FB03233A7803325A707D
:20DBC000DEE75E24DCE700BF68870380509A03805E52068040B40080F0B5E9B01E210DF178
:20DBE000050027F091FB002868D013F063FD28B914F0D8FD0446204669B0F0BD314DAB78E9
:20DC000013B114F0D1FDF5E72B78092B58D8012404FA03F313F4277F52D00CF0B5FD9DF860
:20DC20000520294B1A7114F031FD204602F0EAFB4FF49C7324A8ADF8903002F037FC04465F
:20DC4000002838D10DF1060104A807F09FFF044688BB4FF48C7795F826051C4E7843053068
:20DC6000BDF8062004A9304457F00BF895F826359DF8062007FB036303325A70144B93F86A
:20DC8000A230012BB7D1134902A811F0F3FBBDF8063095F82605053307FB0030052202A92A
:20DCA000304456F0EEFF95F8263507FB03635A7805325A709FE714F015FD9CE74F249AE787
:20DCC000732498E7509A0380F886038040B400805E52068088870380F0B50220E9B014F020
:20DCE00019F928B14B4E3278092A0AD9732428E00A224949494859F086FB0028F2D07A24A0
:20DD00001FE00123934013F4247FEFD015F0BEFA00287DD00CF038FD4FF48C7196F8263518
:20DD20003F4F594308313F48394419F0C7FF022014F0F0F840B93C4B93F836309B0703D5B4
:20DD40003324204669B0F0BD3849394A01F10C0015F008F80028F3D014F098FC012002F0A3
:20DD600051FB4FF483732F4D26ACADF890300FCD0FC40FCD0FC495E8030044F8040B24F826
:20DD8000021B24A8090C217002F090FB044600283BD10DF1060204A9A5F1200008F010FD8B
:20DDA000044690BB4FF48C7596F82605BDF8062005FB007004A9053056F063FF96F8263513
:20DDC0009DF8062005FB037303325A70194B93F8A230012B16D1184902A811F04BFBBDF838
:20DDE00006000522431D96F8260502A905FB0030384456F046FF96F8263505FB03777B78A5
:20DE000005337B7015F026FA9BE714F06BFC98E7D52496E7509A0380798906008555068003
:20DE200040B40080B81E0010A81E0010BD1E00101A8803805E52068088870380F0B5022013
:20DE4000E9B014F067F828B14A4E3278092A0AD9732528E00A224849484859F0D4FA002869
:20DE6000F2D07A251FE00123934013F4247FEFD015F00CFA00287AD00CF086FC4FF48C71A7
:20DE800096F826353E4F594308313E48394419F039FF022014F03EF840B93B4B93F8363027
:20DEA0009B0703D53325284669B0F0BD3749384A01F10C0014F056FF0028F3D014F0E6FB33
:20DEC000012002F09FFA4FF49A732E4C26ADADF890300FCC0FC50FCC0FC594E8030085E84A
:20DEE000030024A802F0E2FA054600283CD103460DF1060204A9A4F1200007F0E1FF054632
:20DF000090BB4FF48C7496F82605BDF8062004FB007004A9053056F0B4FE96F826359DF818
:20DF2000062004FB037303325A701A4B93F8A230012B16D1184902A811F09CFABDF8060015
:20DF40000522431D96F8260502A904FB0030384456F097FE96F8263504FB03777B780533C3
:20DF60007B7015F077F99EE714F0BCFB9BE7D52599E700BF509A0380798906008555068071
:20DF800040B40080B81E0010A81E0010BD1E00101A8803805E52068088870380F0B5CBB059
:20DFA00000210DF1170027F0AFF9002800F09B80504E357C13F07EFB28B914F0F3FB044651
:20DFC00020464BB0F0BD4C4B9A781F4612B114F0EBFBF4E7102D1B7815D1082B40F085807F
:20DFE000464C23780BB10CF0CFFB637813B3102D02D0E378AB427AD122799DF817309A42DC
:20E000001ED05924DCE7092B6FD801229A4012F4657F6AD0082BE3D0394AD27F012A07D179
:20E02000042B05D125F0A4FC04460028D8D0C7E7022BD3E79DF817300120237102F0E2F919
:20E040009DF8170015F0CAF814F020FB022D2CD021D835B3012D2AD000238022294908A813
:20E0600086F8883056F00DFE06A802F01FFA044608BB2946234804F037FD0446D8B9012352
:20E080004FF48C71204ABB7297F8263501FB032303225A7094E7032D0BD0102DDCD1842397
:20E0A00000E08023ADF81830D6E78223FAE78123F8E78323F6E7154E14F014FB96F8F6317C
:20E0C000002B3FF47DAF002501230095CDE901352A462B462946062010F03AF886F8F6517F
:20E0E00012F004FE6CE74F246AE7732468E75E2466E700BFA81E0010509A0380F88603804D
:20E1000016530680B81E001040B4008068870380F0B5E9B01E210DF1050027F0F5F8002898
:20E120006ED013F0C7FA28B914F03CFB0446204669B0F0BD354DAB7813B114F035FBF5E7D2
:20E140002B78092B5ED8012404FA03F313F4247F58D015F09BF8002856D00CF015FB14F0D1
:20E1600095FA9DF805202A4B20461A7102F04AF94FF49F7324A8ADF8903002F097F9044669
:20E1800000283AD10DF1060104A808F031FB044698BB4FF48C7795F826051E4E7843053080
:20E1A000BDF8062004A9304456F06BFD95F826359DF8062007FB036303325A70164B93F8BF
:20E1C000A230012B16D1154902A811F053F9BDF8063095F82605053307FB0030052202A926
:20E1E000304456F04EFD95F8263507FB03635A7805325A7015F02EF899E714F073FA96E75E
:20E200004F2494E7732492E7D52490E7509A0380F886038040B400805E52068088870380E6
:20E220002DE9F0411F4BC4B093F85040BCBB4FF48C77DFF8808014F029FA98F826151A4DB1
:20E2400079436B185A780831113AD2B22944174819F066FD40F24B13154E982206F11001B8
:20E2600002A8ADF8003086F8A04056F00AFD684602F01CF9044678B906F1100008F01EFC2B
:20E28000044648B9032298F8263507FB03535A70204644B0BDE8F08114F024FAF8E7372435
:20E2A000F6E700BF5E52068040B40080B81E0010A81E0010509A038070B5CAB000210DF131
:20E2C000170027F021F8002800F09B8013F0F2F928B914F067FA044620464AB070BD4B4D21
:20E2E000AB7813B114F060FAF5E72B78092B38D801229A4012F4657F33D0082B23D1444C75
:20E3000023780BB10CF040FA4FF48C7195F82635404E594373185A780831203AD2B2314435
:20E320003D4819F01EFD6378EBB13C4BE2781B7C23F01003934266D122799DF817309A42C0
:20E3400017D05924C8E7364AD27F012A07D1042B05D125F00DFB04460028D0D0BCE7022BD2
:20E36000CDD07324B8E79DF817300120237102F049F89DF8170014F031FF14F087F94FF45F
:20E38000A373B822244908A8ADF8183056F079FC06A802F08BF80446D8B91F4808F01CFD52
:20E3A0000446B0B9B8221C4908A856F06AFC1D4B06A91888013880B202F0A0FA01234FF4FA
:20E3C0008C72AB7295F8263502FB03660323737082E7154E14F086F996F8F631002B3FF469
:20E3E0007BAF002501230095CDE901352A462B46294606200FF0ACFE86F8F65112F076FCD1
:20E400006AE74F2468E75E2466E700BF509A0380F886038040B40080B81E0010A81E0010BD
:20E420001653068010580380688703802DE9F041CAB014F02BFF002876D04FF48C763B4D66
:20E4400014F024F995F82615394C714363185A780831763AD2B22144364819F0F7FC0023DE
:20E46000DFF8DC804FF4807288F8083140F2451308F1100108A8ADF8183056F002FC06A858
:20E4800002F014F8074600284BD101AB6A4604A908F1100009F0F2F90746002841D1052249
:20E4A000A87295F8260504A906FB0040104456F0E8FB95F82605042206FB004069460A3017
:20E4C00056F0DFFB042295F826050DEB020106FB00400E3056F0D5FB102295F8263506FB93
:20E4E00003435A70144B93F8A230012B13D1134902A810F0BFFF95F82605052206FB00405C
:20E5000002A9123056F0BDFB95F8263506FB034463780533637014F09DFE38464AB0BDE83E
:20E52000F08114F0DFF8F8E7D527F6E7509A038040B40080B81E00105E5206808887038048
:20E54000A81E0010F0B5E9B01E210DF1050026F0DBFE002876D013F0ADF828B914F022F960
:20E560000446204669B0F0BD394DAB7813B114F01BF9F5E72B78022B66D114F087FE00280C
:20E5800064D04FF48C7795F82615324E794308313144314819F095FC0CF0F6F814F076F8E0
:20E5A0009DF805202D4B01201A7101F02BFF4FF4A5737022284926A8ADF8903056F061FB2F
:20E5C00024A801F073FF0446002838D10DF1060204A921480AF0B6FC044680BB95F826058C
:20E5E000BDF8062007FB006004A9053056F049FB95F826359DF8062007FB036303325A7068
:20E60000174B93F8A230012B16D1164902A810F031FFBDF8063095F82605053307FB0030E2
:20E620000522304402A956F02CFB95F8263507FB036673780533737014F00CFE91E714F044
:20E6400051F88EE74F248CE773248AE7D52488E7509A038040B40080B81E0010F8860380DE
:20E660005E52068088870380F0B5C9B000210DF10F0026F049FE00284DD013F01BF818B9FD
:20E6800014F090F849B0F0BD264CA37813B114F08BF8F7E72378082B3FD14FF48C7694F8E3
:20E6A0002615214D71436B185A7808310A3AD2B229441E4819F03AFC94F826351C4F06FB42
:20E6C00003535B787A8A0A3B9A4228D113F0DEFF07F110000BF03AF8C0B940F24D134FF490
:20E6E000827207F1100106A8ADF8103056F0C9FA04A801F0DBFE48B994F826359DF80F205F
:20E7000006FB03531A7103225A70BBE7019013F0E9FF0198B6E74F20B4E77320B2E733204B
:20E72000B0E700BF509A038040B40080B81E0010A81E00102DE9F0434FF48C77DFF8A88058
:20E74000274C98F82615ADF21C4D794363181D7A0931022221440DF1120056F092FA294691
:20E76000BDF8122005A80FF0ABFE4FF48062002106A856F08AFA4FF001094FF4806304AE7E
:20E78000CDE90039029606AB032205A944200FF0DFFC0546F0B998F82605328807FB004085
:20E7A00006A9053056F06DFA4FF6FF73BDF812209A4206D1FC220B4B48461A731D8213F046
:20E7C00055FF4FF48C7298F8263502FB034433780333637028460DF21C4DBDE8F08300BF14
:20E7E00040B400806C1A0010509A0380F0B5CDB000210DF1010026F087FD002800F0998194
:20E8000012F058FF28B913F0CDFF044620464DB0F0BDC94DAB7813B113F0C6FFF5E72B7851
:20E82000082B40F0A181C54B0220D3E9162113F03BFE002800F09A81C14C22780AB10BF062
:20E84000A3FF4FF48C7195F82635BE4E594308313144BD4819F07EFB22799DF801309A42D4
:20E8600040F08681B94C13F011FFB74814F06CFE01AA217C04F1110018F0D2FE002858D066
:20E8800001AA217C04F1110018F067FF002850D0AF4B93F8A720002A3ED0247C02221E2CE2
:20E8A00028BF1E2440F2671300270DEB0201ADF820300DF12900A31C8DF82830ADF8027092
:20E8C00014F0AEFC2246A3490DF12B0056F0D9F9ADF81C7008A801F0E9FD044630BB0AA856
:20E8E0000AF07EFF044608BB4FF48C7344F24D4295F82605BDF81C1003FB00639142DC7173
:20E9000040F0FC80FF22DA719DF80920002A00F0F1800322DA71F1E01146FF2026F096FB38
:20E920008B4B93F8A730002BB7D1D32413F0DAFE6CE700221146104626F088FB40F26713B3
:20E94000ADF82030002344F60E128DF82830BDF81C30934271D02ED844F2085293424AD0CC
:20E9600044F20D5293425DD044F24D42934253D19DF80A20ADF80230002A00F08480152356
:20E980000DF12B0173488DF8283014F0C4FD0028C6D00B2270490DF1310056F072F942F238
:20E9A0002003ADF83C3002220DF129000DEB020114F036FC30E04CF21452934248D04CF2C8
:20E9C0001E52934254D045F24622934224D11623022207A90DF129008DF8283014F020FC34
:20E9E00006220DF12B015D4814F050FD002897D01422584937E00827022207A90DF1290028
:20EA00008DF8287014F00CFC3A460DF12B01514814F03CFD002883D09DF82830002B7FF447
:20EA200059AF7DE70823022207A90DF129008DF8283014F0F5FB0D22E7E70823022207A977
:20EA40000DF129008DF8283014F0EAFB0E22DCE71923022207A90DF129008DF8283014F0BE
:20EA6000DFFB17223E490DF12B0056F00AF9D3E71023022207A90DF129008DF8283014F0C1
:20EA8000CFFB0E22B5E79DF81630BDF81A200833DBB28DF8283012B113448DF828309DF8E5
:20EAA00028300DF12B01202B88BF20232D4888BF8DF8283014F02FFD00283FF431AFBDF846
:20EAC0001410BDF81620133121440DF1310056F0D8F8BDF81A20002A3FF465AFBDF81810FC
:20EAE000BDF8160008AB133111302144184456F0C8F858E79DF8082082B1DC714FF48C778A
:20EB000007FB0060022207A9053014F089FB95F8263507FB03660623737077E69DF807208A
:20EB20000AB10122F6E69DF80A20002AE6D00222F0E64F246AE600BF509A03806887038021
:20EB4000F886038040B40080B81E0010A81E00105E520680B91E0010C71E0010BC1E001088
:20EB6000C11E0010BB1E001073244FE677244DE659244BE62DE9F0474FF48C79614EDFF85A
:20EB800094A196F8263586B009FB03A35B785746062BB04640F0B0801D210DF1150026F019
:20EBA000B3FB002800F0AA803378012B40F0A880554D2B7BFD2B78D0FE2B02D0FC2B40F02C
:20EBC0009F80298A59B3EB8998F82605F92B9ABFADF816300023F93BEB814FF48C7388BF74
:20EBE000F92203FB0070494B88BFADF81620BDF816201944053056F044F8EB89BDF8162078
:20EC000013B12B8A13449BB24FF48C712B8298F82635033201FB03777A70002441E0FE2BFC
:20EC20004FF014030DF11602CDE901324FF480630A46009308BF4620344B18BF47200FF08D
:20EC400087FA044660B108282BD113F019FD4FF48C7298F8263502FB037703237B70DCE71C
:20EC6000BDF816302949F92B81BFF922F93B2A82EB8198BF28824FF48C7598F8260588BF15
:20EC8000ADF8162005FB0070BDF81620053055F0F8FF98F8263505FB03779DF81630033357
:20ECA0007B70204606B0BDE8F087194DE988AC88641A09D113F0E4FC96F8263509FB03A952
:20ECC000032389F80130ECE7F92C28BFF92496F826052B6809FB00A022461944053055F031
:20ECE000D0FFEB882344EB8096F82635033409FB03A989F8014090E77E24D2E74F24D0E772
:20ED00007324CEE7509A03806C1A00100C290180B89F038040B400802DE9F0474FF48C770D
:20ED2000404D414E95F8263586B007FB03635B78B1460A2BAA466FD11D210DF1110026F09F
:20ED4000E3FA00286AD02B78023B022B68D895F82615042207FB016105A8083155F091FF1A
:20ED6000324B93F89D308BB3059C7CBBDFF8C480B8F8043053B3B8F808303BB3FD222C4B37
:20ED800001201A7313F072FC95F82605022207FB0060D8F80010053055F073FF022295F899
:20EDA0002605D8F8001007FB00601144073055F068FF0423A8F8063095F8263507FB03665E
:20EDC00007237370204606B0BDE8F0874FF48C750DF112029AF826351E210292F92205FBBD
:20EDE0000393CDE900210533042205A945200FF0AFF904460028E5D1FE220D4B1882012033
:20EE00001A7313F033FC9AF826359DF8122005FB039303325A70D5E77E24D3E74F24D1E7A7
:20EE20007324CFE7509A038040B400805E5206806C1A0010B89F03804FF48C71064B074A1C
:20EE400093F8263501FB03235B780C2B01D1FEF7B1BD7E20704700BF509A038040B4008076
:20EE600013B54FF48C71134C134A94F8263501FB03235B78062B16D11E210DF1070026F080
:20EE800043FA90B1A3781BB113F08EFC02B010BD2278092A0BD80123934013F4257F06D0D9
:20EEA000FEF718FEF2E77E20F0E74F20EEE77320ECE700BF509A038040B400804FF48C716F
:20EEC000064B074A93F8263501FB03235B78062B01D1FEF781BE7E20704700BF509A0380FD
:20EEE00040B400802DE9F0474FF48C7A3B4FDFF8F49097F82635B8B00AFB03935B78062B32
:20EF000066D11E210DF1150026F0FEF9002861D0BA7832B113F048FC0546284638B0BDE860
:20EF2000F0873B78092B57D84FF0010808FA03F313F4277F50D080230DF116060093CDE931
:20EF4000018618AB114630200FF002F905460028E3D110AB18AABDF8161030200EF0D4FD28
:20EF60009DF8413093BB08A81D4C24F0A5FE0DF1200CBCE80F000FC49CE80F000DF1200EFE
:20EF800084E80F00BEE80F0010340FC49CE80F0084E80F0008A906A810F06CFA00952B4651
:20EFA000CDE90186052206A918200FF0D1F805460028B2D111F09AFE97F826350AFB039924
:20EFC0009DF81630033389F80130A6E75E25A4E77E25A2E74F25A0E773259EE7509A038022
:20EFE0006887038040B400802DE9F0474FF48C79394FDFF8EC8097F82635B8B009FB0383EF
:20F000005B78062B62D11E210DF1150026F07CF900285DD0BA7832B113F0C6FB05462846F5
:20F0200038B0BDE8F0873B78023B012B52D880234FF0010A0DF11606CDE9003A029618AB34
:20F04000114630200FF084F805460028E7D110AB18AABDF8161030200EF056FD9DF8413064
:20F0600093BB08A81D4C24F027FE0DF1200CBCE80F000FC49CE80F000DF1200E84E80F0006
:20F08000BEE80F0010340FC49CE80F0084E80F0008A906A810F0EEF900952B46CDE901A6ED
:20F0A000052206A913200FF053F805460028B6D111F01CFE97F8263509FB03889DF8163094
:20F0C000033388F80130AAE75E25A8E77E25A6E74F25A4E77325A2E7509A03806887038077
:20F0E00040B400802DE9F04F4FF48C7A424FDFF8109197F82635B9B00AFB03935B78062B03
:20F1000073D11E210DF1150026F0FEF800286ED0BA7832B113F048FB0546284639B0BDE845
:20F12000F08F3B78092B64D84FF0010808FA03F313F4257F5DD080230DF116060093CDE90F
:20F14000018618AB114630200FF002F805460028E3D110AB18AABDF8161030200EF0D4FC28
:20F160009DF84130002B3ED108A8244C24F0A4FD0DF1200CBCE80F000FC49CE80F0004F142
:20F18000100E0DF1200B84E80F00BBE80F00AEE80F009CE80F008EE80F0050340DF1200E8E
:20F1A000BEE80F000FC49CE80F0084E80F0008A906A810F05FF900952B46CDE90186052298
:20F1C00006A911200EF0C4FF05460028A5D111F08DFD97F826350AFB03999DF8163003337E
:20F1E00089F8013099E75E2597E77E2595E74F2593E7732591E700BF509A03806887038021
:20F2000040B40080F0B54FF48C75174E174C96F8263587B005FB03435F78062F20D11D2128
:20F220000DF1150026F070F8E0B10DF1160202920A22CDE90072002296F82635114605FB4C
:20F240000343102005330EF083FF38B996F826359DF8162005FB034303325A7007B0F0BD32
:20F260007E20FBE74F20F9E7509A038040B4008070B54FF48C75184E184C96F8263586B08C
:20F2800005FB03435B78062B21D11D210DF1150026F03AF8E8B10DF116020A210292022207
:20F2A000CDE90021002296F82635114605FB0343422005330EF04CFF38B996F826359DF87D
:20F2C000162005FB034303325A7006B070BD7E20FBE74F20F9E700BF509A038040B4008061
:20F2E00070B54FF48C751C4E1C4C96F8263586B005FB03435B780A2B2AD11D210DF111001E
:20F3000026F002F830B396F82615042205FB014105A8083155F0B5FC0DF112021E21029208
:20F32000F92296F82635CDE9002105FB03430422053305A941200EF00BFF38B996F826355D
:20F3400005FB03449DF812300333637006B070BD7E20FBE74F20F9E7509A038040B40080F3
:20F3600070B54FF48C75184E184C96F8263586B005FB03435B78062B21D11D210DF11500AE
:20F3800025F0C2FFE8B10DF11602012102921022CDE90021002296F82635114605FB034381
:20F3A000202005330EF0D4FE38B996F826359DF8162005FB034303325A7006B070BD7E209A
:20F3C000FBE74F20F9E700BF509A038040B4008070B54FF48C751C4E1C4C96F8263586B002
:20F3E00005FB03435B780A2B2AD11D210DF1110025F08AFF30B396F82615042205FB0141C5
:20F4000005A8083155F03DFC0DF112021E210292502296F82635CDE9002105FB0343042205
:20F42000053305A940200EF093FE38B996F8263505FB03449DF812300333637006B070BD13
:20F440007E20FBE74F20F9E7509A038040B4008070B54FF48C75174E174C96F8263586B0AC
:20F4600005FB03435B78062B1FD11D210DF1150025F04AFFD8B10DF116020121029220220C
:20F48000CDE90021002296F82635114605FB0343302005330EF05CFE28B9212296F8263500
:20F4A00005FB03435A7006B070BD7E20FBE74F20F9E700BF509A038040B4008070B54FF482
:20F4C0008C75174E174C96F8263586B005FB03435B78062B1FD11D210DF1150025F014FF91
:20F4E000D8B10DF11602012102921022CDE90021002296F82635114605FB0343312005337D
:20F500000EF026FE28B9132296F8263505FB03435A7006B070BD7E20FBE74F20F9E700BF49
:20F52000509A038040B4008070B54FF48C75174E174C96F8263586B005FB03435B78062B50
:20F540001FD11E210DF1150025F0DEFED8B10DF1160201210292FA22CDE90021002296F880
:20F560002635114605FB0343322005330EF0F0FD28B9082296F8263505FB03435A7006B064
:20F5800070BD7E20FBE74F20F9E700BF509A038040B4008070B54FF48C75174E174C96F810
:20F5A000263586B005FB03435B78062B1FD11E210DF1150025F0A8FED8B10DF116020121B2
:20F5C00002921122CDE90021002296F82635114605FB0343332005330EF0BAFD28B914228E
:20F5E00096F8263505FB03435A7006B070BD7E20FBE74F20F9E700BF509A038040B40080C0
:20F600002DE9F0414FF48C78224D234F95F8263586B008FB03735B78072B35D11E210DF19C
:20F62000170025F071FE88B3AE7836B113F0BCF80446204606B0BDE8F0812B78092B27D8DE
:20F64000012404FA03F313F4257F21D095F82615224608FB017105A8083155F012FBCDE962
:20F66000014622460096334605A902200EF070FD04460028DDD111F039FB032295F826352F
:20F6800008FB03735A70D4E77E24D2E74F24D0E77324CEE7509A038040B4008013B54FF4AF
:20F6A0008C71144C144A94F8263501FB03235B78282B18D11E210DF1070025F025FEA0B1AA
:20F6C00011F0F8FF18B913F06DF802B010BDA37813B113F069F8F8E7084813F039FA30B1F1
:20F6E000FEF7FAFAF1E77E20EFE74F20EDE75E20EBE700BF509A038040B400801A8803807D
:20F7000013B54FF48C71144C144A94F8263501FB03235B78292B18D11E210DF1070025F0B1
:20F72000F3FDA0B111F0C6FF18B913F03BF802B010BDA37813B113F037F8F8E7084813F0F9
:20F7400007FA30B1FEF77AFBF1E77E20EFE74F20EDE75E20EBE700BF509A038040B40080DE
:20F760001A8803802DE9F0414FF48C77DFF88C801F4E98F8263586B007FB03635B78072BF9
:20F7800031D11E210DF1170025F0BEFD68B300233C2298F82615CDE9012307FB016100930B
:20F7A0000122083160200EF0D3FC0446B8B9114D4FF496702B6823F480632B6012F09AFE8C
:20F7C0002B6843F480632B600B4B83F8644111F08DFA032298F8263507FB03635A7020464B
:20F7E00006B0BDE8F0817E24F9E74F24F7E700BF40B400806080092068870380509A03804F
:20F800002DE9F0434FF48C76DFF89880244D98F82635A7B006FB03535B78062B3BD11E2112
:20F8200005A825F071FDC0B30A2300224FF080090DF11607CDE90093029706AB11463220B7
:20F840000EF086FC044610BB9DF81C3002978DF815301E230122CDE900930DF1150106AB5D
:20F8600043200EF075FC044688B998F82605BDF8162006FB005006A9053055F002FA98F87F
:20F8800026359DF8162006FB035303325A70204627B0BDE8F0837E24F9E74F24F7E700BF05
:20F8A00040B40080509A0380F0B54FF48C76214F214D97F82635A7B006FB03535B78072B02
:20F8C00033D11E2105A825F01FFD80B397F8263506FB03531B7A8DF8153023B30DF1160347
:20F8E00002931E2280230DF11501CDE90032432006AB01220EF02CFC044688B997F82605F2
:20F90000BDF8162006FB005006A9053055F0B9F997F8263506FB03559DF8163003336B70A1
:20F92000204627B0F0BD3324FAE77E24F8E74F24F6E700BF509A038040B40080F0B54FF44C
:20F940008C76154F154D97F8263587B006FB03535C78062C1CD11E210DF1170025F0D4FC3B
:20F96000C0B1002301222046CDE9012300931A4619460EF0EDFB044638B911F0B7F9032247
:20F9800097F8263506FB03535A70204607B0F0BD7E24FAE74F24F8E7509A038040B40080DC
:20F9A00073B54FF48C75184E184C96F8263505FB03435B780B3BDBB2F22B1FD800210DF109
:20F9C000070025F0A1FCD8B196F8260504F10A036843C35A5A1EF42A14D8221852780A339F
:20F9E00093420FD10830204411F0B4FB96F8263505FB03440323637002B070BD7E20FBE77E
:20FA00004F20F9E73320F7E7509A038040B400804FF48C7108B50C4B0C4A93F8263501FBF9
:20FA200003235B78223BDBB2DC2B0AD811F0B4FC18B1BDE8084011F05DBCBDE80840FEF797
:20FA4000ADBA7E2008BD00BF509A038040B40080F0B54FF48C771E4D1E4E95F8263587B05B
:20FA600007FB03635B78062B2CD11E210DF1150025F04AFC40B3AB782BB112F095FE04469F
:20FA8000204607B0F0BD297809291FD801228A4012F4257F1AD00DF1160202920A2219461C
:20FAA000CDE9003204201A460EF052FB04460028E6D111F01BF9032295F8263507FB0363DC
:20FAC0005A70DDE77E24DBE74F24D9E77324D7E7509A038040B400804FF48C71064B074AE9
:20FAE00093F8263501FB03235B78062B01D1FEF70FBB7E20704700BF509A038040B4008074
:20FB0000F7B54FF48C771F4E1F4D96F8263507FB03535B78062B2FD11E210DF1070025F07C
:20FB2000F3FB58B3194B5C7854BB1948012322462146006841F03EF996F82635B8B107FB0D
:20FB4000035002221349053055F09BF896F8260507FB005080234FF48C72C37196F82635B9
:20FB600002FB035506236B70204603B0F0BD07FB035044718471EDE77E24F5E74F24F3E7C8
:20FB80003524F1E7509A038040B40080B6510680FC2B00101C2000802DE9F3414FF48C7743
:20FBA000DFF8BC80284E98F8263507FB03635B78092B3FD11E210DF1070025F0A5FB002831
:20FBC0003AD0224B5C78002C38D198F82615022207FB01611E48083155F053F898F8263538
:20FBE0001C4D07FB03632A8A9B7A1A44B2F5004FAB7425DC802B23D81748012322462146FF
:20FC0000006841F0D7F8E8B198F826052B8A07FB00601249AA7C1944053055F032F898F8FF
:20FC2000263507FB0366AB7C03337370204602B0BDE8F0817E24F9E74F24F7E73524F5E788
:20FC40003324F3E70524F1E740B40080B6510680B81E0010A81E0010FC2B001020200080BE
:20FC6000509A03802DE9F3414FF48C76264F274D97F8263506FB03535B78082B3ED11E210A
:20FC80000DF1070025F040FB002839D0204B5C78002C37D197F82615DFF8888006FB01516F
:20FCA000022208311B4854F0ECFFB8F81030B3F5805F04D93324204602B0BDE8F08116481E
:20FCC000012322462146006841F074F80028F1D1B8F81020114B12481A802146012322461F
:20FCE000006841F067F80028E4D0802297F8263506FB03535A7104225A70DCE77E24DAE76C
:20FD00004F24D8E73524D6E7509A038040B40080B6510680B81E0010002C00106C09001086
:20FD2000FC2B0010A81E00102DE9F74F4FF48C7B464E474D96F826350BFB03535B78892B1C
:20FD400004D97E24204603B0BDE8F08F1E210DF1070025F0D9FA002874D03E4B5C78002CC6
:20FD600072D196F8261502220BFB01513A48083154F087FF96F82635384F0BFB03533A8AE6
:20FD80009B7A1A44B2F5805FBB7401DD3324D9E7802BFBD8DFF8D090012322462146D9F8CD
:20FDA000000041F007F80028F0D12D4B1A889846002AEBD096F826350BFB03535A78BB7CFF
:20FDC00009339A42BDD1DFF8A4A0012322462146DAF8000040F0EEFF0028D7D096F82615E8
:20FDE0003B8A0BFB01511F48BA7C18440B3154F048FFBA7C3B8A1344B8F80020934218DB3C
:20FE00000027DFF86CB03B463A463946DAF80000ABF8047040F0CEFFB8F800303A46ABF85F
:20FE2000063039463B46D9F80000A8F8007040F0D6FE4FF48C7296F8263502FB0355032302
:20FE40006B707FE74F247DE735247BE7509A038040B40080B6510680B81E0010A81E0010A5
:20FE60006C09001040A40080002C0010FC2B00101820008013B54FF48C711A4C1A4A94F810
:20FE8000263501FB03235B78912B23D811F084FA014618B111F02EFA02B010BD0DF107001F
:20FEA00025F032FAC0B111F005FC10B912F07AFCF2E7A37813B112F077FCEDE72378082B7E
:20FEC0000CD10A4B1A799DF807309A4208D1FEF7A7F9E1E77E20DFE74F20DDE77320DBE793
:20FEE0005920D9E7509A038040B40080F88603804FF48C7108B50C4B0C4A93F8263501FB5B
:20FF000003235B78203BDBB2802B0AD811F044FA18B1BDE8084011F0EDB9BDE80840FEF7F5
:20FF2000CBB97E2008BD00BF509A038040B4008013B54FF48C711B4C1B4A94F8263501FB83
:20FF400003235B78763B402B23D811F025FA014618B111F0CFF902B010BD0DF1070025F0FF
:20FF6000D3F9C0B111F0A6FB10B912F01BFCF2E7A37813B112F018FCEDE72378082B0CD173
:20FF80000A4B1A799DF807309A4208D1FEF74EFAE1E77E20DFE74F20DDE77320DBE759208E
:20FFA000D9E700BF509A038040B40080F88603804FF48C71064B074A93F8263501FB0323F6
:20FFC0005B78452B01D1FEF7BDBA7E20704700BF509A038040B4008070B5174B5B7803B39B
:20FFE0004FF48C76154D164C95F82605704323185B78022B17D12B78082B16D801229A40A9
:020000040001F9
:2000000012F48E7F11D0053020441BF08BFC00280DDC0ED10D2295F8263506FB03435A70A9
:2000200070BD3520FCE77E20FAE77320F8E73620F6E7D220F4E700BFAC5B0680509A0380B1
:2000400040B4008008B511F0A7F918B1BDE8084011F050B94FF48C71084B094A93F8263542
:2000600001FB03235B780A3BDBB2F32B03D8BDE80840FEF7F9BA7E2008BD00BF509A03809C
:2000800040B400804FF48C7273B5224E224C96F82635354602FB03435B78892B32D11E2135
:2000A0000DF1070025F030F970B33278082A2DD80123934013F48E7F28D0184B1A781AB136
:2000C000DA799B79134323D14FF48C7295F826355A43A318187A124BD15A124B0B32DB69F6
:2000E0002244112B0BD11CF097FA4FF48C7295F8263502FB03440323637002B070BD1CF094
:2001000037F9F2E77E20F8E74F20F6E77320F4E73520F2E7509A038040B40080AC5B068003
:2001200049B400806C1A001073B54FF48C750F4E0F4C96F8263505FB03435B78062B10D174
:2001400000210DF1070025F0DFF860B1094811F001F8032296F8263505FB03435A7002B061
:2001600070BD7E20FBE74F20F9E700BF509A038040B400802096038013B54FF48C710E4C48
:200180000E4A94F8263501FB03235B78092B0DD11D210DF1070025F0B7F848B12378023B41
:2001A000022B07D8FEF7C6FA02B010BD7E20FBE74F20F9E77320F7E7509A038040B40080DE
:2001C00073B54FF48C75134E134C96F8263505FB03435B78062B19D100210DF1070025F09B
:2001E00093F8A8B113F036F896F82605102205FB00400A49053054F044FD1322002096F8CF
:20020000263505FB03435A7002B070BD7E20FBE74F20F9E7509A038040B40080E0900380F1
:2002200073B54FF48C75164E164C96F8263505FB03435B78162B1ED100210DF1070025F01F
:2002400063F8D0B196F8260505FB0040083013F013F896F82605102205FB00400A490530D0
:2002600054F00FFD96F82635002005FB03440323637002B070BD7E20FBE74F20F9E700BF78
:20028000509A038040B40080E09003804FF48C7108B50B4B0B4A93F8263501FB03235B7807
:2002A000012B0AD911F078F818B1BDE8084011F021B8BDE80840FEF799BA7E2008BD00BFD7
:2002C000509A038040B400804FF48C734C4A03FB002090F81031013B662B00F28E80DFE8EA
:2002E00003F03436383A3C3E4248444C8C4A4E848C8C8C8C8C8C8C8C8C8C8C8C8C8C8C8C33
:200300008C8C8C8C8C8C8C8C8C8C8C8C8C8C8C8C8C5456585A406C6E686A5C70725E50520B
:20032000606264668C8C78768C8C8C7A74467E808C8C8C8C7C8C8C8C8C8C8C8C8C8C8C8CA5
:200340008C8C8C8C8C8286888A00FFF781B8FFF7B5B8FFF7E9B8FFF71DB9FFF751B9FFF7DC
:200360009DB9FFF7CDB9FFF7FDB9FFF749BAFFF79BBAFFF7E3BAFFF713BBFFF729B8FFF797
:2003800047BBFFF765BBFFF7A7BBFFF7B9BBFFF703BCFFF767BCFFF7C7BCFEF7E1BFFEF7B2
:2003A0009FBFFEF765BFFEF72DBFFEF79BBEFEF71BBEFEF797BDFEF781BDFEF751BDFEF755
:2003C0003BBDFEF7A9BCFEF7D5BBFFF753BDFFF78FBDFFF7ADBDFFF7EBBDFFF7FDBDFFF75A
:2003E00031BEFFF74FBEFFF79FBEFFF7C5BEFFF7E7BEFFF715BFFFF749BF3720704700BF0F
:2004000040B4008008B5D0B142F6E46200210C4854F03BFC0B4B002193F89D300A48002B70
:2004200014BF4FF4C0324FF4003254F02EFCBDE8084042F604320021044854F026BC08BD1E
:20044000105803805E5206800C2D01800C2D03800023084A32F82310814204D102EB830328
:20046000B3F90200704701332A2BF3D14FF0FF30704700BF84890600F8B500242646094D40
:2004800035F8047BA3B29F4202D807483044F8BD35F8020BFFF7DCFF0028C8BF36180134EB
:2004A000F0E700BF105803800C2D01802DE9F843074610F00FFF08B110F0C2FEFFF7DCFF0B
:2004C0002E4B064693F89D30002B2D4B14BF4FF4004E4FF0000E83424CD803F50033A3EB09
:2004E0000E09814546D3B7F80080264CA8F1850189B20929258833D9234A681CB2F800C0C5
:20050000CCF5F9610631884236D09A1B542303FB0CF3A2EB0E0203F580639A422CD34046B7
:20052000FFF796FF83B2B3F5805F024622D8831999451FD304EB4503A3F8048004EB8503F9
:20054000C3F8A46F20B107F10801304654F099FB0020238801339BB223806380BDE8F883BB
:2005600040F2092222FA01F1CA07C5D540F2CF739D42D4D13920F1E74B20EFE75E52068005
:200580000C2D0180105803800C2D0380F8B50F46104D114C4FF4887200210646284654F0E2
:2005A00074FB04EB470398882880FFF751FF021E07DD04EB8704D4F8A41F05F1080054F036
:2005C00060FB4FF488720349304654F05AFB3046F8BD00BF700900101058038030B5ADF543
:2005E0002D7D10F077FE08B110F02AFE1FF068FA80B9BE4D95F8602062B1BD4C2288638888
:200600009A420AD1BB4A9378052B03D1BA4B9070D88098760DF52D7D30BD61886846FFF77E
:20062000B5FF4FF48872694668A854F02AFBBDF8A031852B00F0DC805DD8422B00F0068106
:2006400031D8272B00F0F3801CD8172B00F0FC800FD8122B00F0F3806388013363801FF0A2
:200660002FFAB0F5E77FD5D8228863889A42D4D1D0E7182B00F0D580192BEDD1012023F00E
:20068000A1FBE9E72F2B00F0E88004D82C2BE3D100F056FDB6E0402B00F0CC80412BDBD1BD
:2006A00044A91220C8E0512B00F0BF800ED8442B00F0DE80C0F0D9804D2B00F0D280502BE7
:2006C000CAD10C216AA804F0C9F99BE0822B00F0A48006D8802B00F09E80812BBCD101215C
:2006E00005E0832B00F09B80842BB5D110216AA802F0FAF986E0B3F59A7F00F0D9802DD88A
:20070000C22B00F0B88010D88D2B00F0A28004D8882BA1D102F0B2FF74E08E2B76D0C12B2F
:200720009AD16AA820F0D6FE6CE0DE2B00F0B68007D8C52B00F0A380C72B8DD122F0DCFFBE
:2007400060E0E02B00F0C680B3F5837F84D10DF5897248A96AA806F033F853E0B3F5A37FFB
:2007600000F0B48025D8B3F59C7F00F09B800AD8B3F59B7F7FF470AF0DF5897248A96AA854
:2007800008F0E0FB3EE0B3F59F7F00F0998040F2451293427FF460AF1FF092F9B0F5E77F14
:2007A0003FF638AF45AB1A4646A96AA807F066F828E040F24D12934200F08F80B3F5A77F3C
:2007C0000BD2B3F5A57FD7D040F24B1293427FF443AF6AA806F072F914E040F26712934219
:2007E0007FD0B3F5007F7FF437AF08F0A3FF09E01FF066F9B0F5E77F3FF60CAF46A96AA83D
:2008000002F0CCFF00283FF427AF03E746A96AA805F0ACF8F6E7002169E7022167E7032183
:2008200065E76AA805F048F8ECE70E214AE704F0D9FBE7E7112044A900F098FFE2E70121CC
:200840006AA804F067F8DDE70021F9E704F0CEFCD8E76AA804F07AF9D4E76AA804F0BCF803
:20086000D0E76AA820F062FECCE705F081F8C9E705F0D4F8C6E76AA800F0BEFBC2E71FF08D
:200880001FF900287FF4C6AE95F86030002B3FF4C1AE50216AA800F0E5FBB3E76AA800F058
:2008A00011FCAFE70DF5897148A805F06FF9A9E700230DF5897248A96AA805F001FBA1E720
:2008C0000DF5897148A805F093FF9BE76AA806F083FA97E700F088FC94E76AA808F036FFF2
:2008E00090E76AA808F07CFF8CE700BF548F058010580380509A0380F886038038B50546D1
:2009000008880C46FFF7A4FD021E0ADD054B04F1080103EB8503D3F8A40FBDE8384054F0B4
:20092000B0B938BD1058038070B52C4D01462E887E2E51D8562404FB06540388C12BA38091
:2009400027D00AD82F2B1AD04D2B2FD0562303FB065500233920AB8070BDC52B32D0DE2B62
:20096000F4D100F1080303CBC4F80600C4F80A101868A379C4F80E0023F0400307E041224A
:200980000831A01D54F07DF9A37903F07F03A37108E08068C4F806008B896381A37A03F068
:2009A0007F03A37201362E800020D5E700F1080303CBC4F80A10237BC4F8060003F07F036A
:2009C0002373EFE754220831A01D54F05AF9237A03F07F032372E5E74B20BDE70C2D03806A
:2009E00080B582B000AF78607B681B68124A13607B685B68104A53607B689B680E4A9360F0
:200A00007B68DB680C4AD3607B681B690A4A13617B685B69084A53617B689B69064A936120
:200A20007B68DB69044AD361034B044A1A62024B024A1A6200F004F8E85207806473829149
:200A4000BFF34F8F0449054BCA6802F4E0621343CB60BFF34F8FFEE700ED00E00400FA0539
:200A600008B5012040F02AF9014B186008BD00BF800A0010F8B50F4C054620680E461746D7
:200A800098B100230A22194640F094F901280ED13946304643F060FC002328601A461946AC
:200AA000206840F09CF80020F8BD0120FCE70220FAE700BF800A0010F8B50F4C05462068DA
:200AC0000E46174698B100230A22194640F072F901280ED13946304643F02CFC00232880B0
:200AE0001A461946206840F07AF80020F8BD0120FCE70220FAE700BF800A00102DE9F04191
:200B0000174D074628680E461446984618B300230A22194640F04EF901281ED1002043F0AD
:200B2000F3FB104BE2B21A72220A1A7283F80880012C0AD89B6828683B8000231A46194652
:200B400040F04DF80020BDE8F08116F8012B013C1A72A4B2ECE70120F5E70220F3E700BF06
:200B6000800A0010000009200023012213B50446CDE90023C11D431E13F8012FD2438B4225
:200B80001A70F9D1694622460E23084618F0EDFEDDE90023C4E9002302B010BD00238AB2E1
:200BA000C0E90023704730B400240025C0E90045052230BC54F065B838B504460D46102267
:200BC000002154F062F829462046BDE83840082254F057B8D0E9002313430CBF01200020A9
:200BE000704707B5FF234FF0FF32CDE900236A460146104618F0CCFE003018BF012003B01D
:200C00005DF804FB07B54FF6FF734FF0FF32CDE900236A460146104618F0BAFE003018BFB0
:200C2000012003B05DF804FB2DE9F041044608460E4656F0C2FB012805461BD0A0B102287C
:200C400023D0335C871E302B00F1FF383A463146204622D116F80830302B1ED154F011F8BD
:200C60000023E355BDE8F0812046BDE8F041124956F082BB1049204656F07EFB2A46314684
:200C8000E01CBDE8F04153F0FCBF0B49204656F073FB2A463146A01CF3E753F0F2FF2E2314
:200CA00004EB0800E3550222F11953F0EAFF00232C446370D6E700BF46D706002DE9F0415F
:200CC000044608460E4656F078FB0546032824D8DFE800F00208131B2046BDE8F041214968
:200CE00056F04ABB1F49204656F046FB01223146201DBDE8F04153F0C4BF1A49204656F0D2
:200D00003BFB02223146E01CF3E71649204656F033FB03223146A01CEBE7C71E3A463146ED
:200D2000204653F0AEFF2E23A5F10208E3550322F11904EB080053F0A4FF002362190A4937
:200D40005370C97959B114F80810302907D112F8012C302A03D1625D302A08BFE355BDE80D
:200D6000F08100BFDDD60600C3580680F8B5044608460D4656F021FB06461C49204656F092
:200D8000FBFA062E20D8DFE806F030040B0F13171B0001222946E01DBDE8F84053F071BF03
:200DA00002222946A01DF7E703222946601DF3E704222946A018EFE705222946E01CEBE793
:200DC00006222946A01CE7E7B71F3A462946204653F057FF2E23701FE35520440622E91988
:200DE00053F04FFF002334446370F8BDB6D7060030B50024130602D50023035530BD8D5C62
:200E000015B97CB9013AF5E72B095CB913B13033037001238D5C5C1C05F00F053035E4B24C
:200E2000C554EFE72D09631C3035DBB20555F1E730B50D4604468DB00A22002103A853F0F0
:200E400024FF2946082203A853F01BFF03A96846092218F04BFD0822694606A8FFF7C8FFB5
:200E600020461F2306A900F8013BFFF7DDFE0DB030BD30B50D4604468BB00822002103A8B9
:200E800053F003FF2946082203A853F0FAFE03A901A8072218F02AFD062201A905A8FFF76C
:200EA000A7FF05A92046FFF7BFFE0BB030BDFFFF30B50D468BB008220021044603A853F029
:200EC000E4FE0822294603A853F0DBFE072203A901A818F00BFD062201A905A8FFF788FF46
:200EE0000A4B1B7A2BB105A92046FFF79DFE0BB030BD05A856F061FA20B105A9204656F066
:200F00003BFAF4E7302360702370F0E7509A038070B50E46154604468AB00822002103A879
:200F200053F0B3FE0822002101A853F0AEFE0822314603A853F0A5FE072203A901A818F022
:200F4000D5FC01A905A80722FFF752FF032D05A9204603D1FFF7B2FE0AB070BDFFF706FF59
:200F6000204656F02AFA0138C0B2235C302B07D02E2B01D10138C0B2002320444370EBE763
:200F8000013810F0FF00F0D1F6E7002330B5150600EB030402D50023237030BD8C5C5D1C8B
:200FA00024093034C4548C5CEDB204F00F0402333034DBB24455013AE9E7082230B585B0EC
:200FC00004460D460DEB0200002153F05EFE082229460DEB020053F054FE02A96846072210
:200FE00018F084FC062269462046FFF7CEFF05B030BDFFFFFFFFFFFF10B5AAB001466846B9
:20100000FFF7D1FD15A3D3E90023CDE9022302AA6946104618F0BCFC0446D8B9694617A8E0
:20102000FFF7CBFF0A230C220DF15E010DF111008DF8103053F025FE23460222064904A876
:201040008DF81D401FF0AAF9002808BF4B2420462AB010BD3324FAE7A2D50600FF0FA5D455
:20106000E8000000F0B590F9023093B0002B0F4602DA002013B0F0BD044642F21B030F4E00
:2010800000253046ADF8043034F8033B502220F8033B29468DF8065053F0F7FD3A46214642
:2010A000F01C53F0EEFD2B460222054901A81FF075F90028DDD14B20DCE700BF18A00380EF
:2010C000A2D506001A232DE9F041044694B001460C220DF105008DF8043053F0D2FD00231B
:2010E00024788DF8113014F0400404D00024204614B0BDE8F08142260F4D0D22D5E90078E5
:201100007E4306F1080001A9284453F0BAFD02232E4486F849302B680133B3F5007F08BFBC
:20112000234643452B6005D0044B5B7A002BDDD02F60DCE74B24DAE7E88F0580F8860380E3
:201140002DE9F041234B8CB0DA789846002A37D0214C04A804AD22F0AFFD0FCD0FC495E889
:201160000F0004F1300604AF84E80F000FCF0FC695E80F0086E80F00103404AE0FCE0FC4A5
:2011800095E80F0084E80F000023CDE90133134900931A46B1F83011114814F0B9FA0446A8
:2011A000A0B908F055FF044680B902210D481FF035FA50B1052088F8020009F0D7FE05E0F6
:2011C00002200AF0D7F80028C2D14B2420460CB0BDE8F081509A038068870380E025068058
:2011E000ACD906002DE506002DE9F047DEB02DAA9046C54B03F110051446186859680833D5
:2012000003C4AB422246F7D119889B782180A3702E2200210DF1C70053F037FD11F0F6F8E6
:20122000032010F077FE002800F07E82042010F071FE002800F07A8221F096FF10F04AF86F
:201240000446002840F07482B04811F081FC002855D00DF043F9802301200DF11206CDE96A
:20126000003002963EAB2246214630200CF070FF054600284BD1A64FFB78002B41D014AB41
:201280003EAA318830200CF03FFCA24B9A7E002A40F0E78180230A210296CDE900311020E2
:2012A0003EAB11460CF054FF002840F018813EAA07AB318810200CF027FC9DF81C2032B950
:2012C000BDF81E30ADF820200133ADF81E30BDF81E00914CBDF82010A4F8F201A4F8F4113A
:2012E00012F008FF9DF85330002B40F05E819DF85190B9F1000F0ED0B9F1020F45D05E2533
:2013000005E002200AF036F80028B8D14B2528465EB0BDE8F0870CA822F0CEFC0DF1300C1B
:20132000BCE80F000FC49CE80F0004F1100E0DF1300A84E80F00BAE80F00AEE80F009CE8F4
:201340000F008EE80F0050340DF1300EBEE80F000FC49CE80F0084E80F000CA905A80EF043
:2013600089F80123CDF80890CDE9009305224B4605A911200CF0ECFE002840F0B0800FF01E
:20138000B5FC644B187911F029FF634991F8F7315B0740F1B58040F2FD300FF04BF8002845
:2013A00040F097805D4B93F85030002B00F091805A4C94F85020002A40F0C28000224FF068
:2013C000800A4FF001090296CDE900A93EAB114630200CF0BDFE0446002840F0AB8114AB6F
:2013E0003EAA318830200CF08FFB9DF85130224687F82D351B9B2146C7F830351E230296FD
:20140000CDE900A312203EAB0CF0A2FE0446002840F0908109AB3EAA318812200CF074FB17
:20142000DDE90A123E4812F069FACDE901443D49CDF8009023462246B1F83011404614F0C4
:2014400067F900284BD19DF8540008B112F0E6FD354B93F88D31002B40F098802F4C94F81E
:201460005030EBB1314B987D0AF0B2F98DF870000DF1710012F010FA002303222C491CA829
:201480001EF08CFF94F85030012B09D90DF1710012F00AFA0023032225491CA81EF07EFF1F
:2014A0000023032222491E481EF078FF21491CA855F062FF002302221D491CA81EF06EFFCE
:2014C00000283FF423AF144BD3E91E1011F026FFA1E0194940F2FD300DF0ECFE08B1054643
:2014E00015E70E4B93F85030002B7FF461AF13494FF483600DF0DEFE00283FF459AFEEE74B
:2015000001F58E71E6E700BF2C8A06001A880380509A0380F8860380688703805E52068053
:2015200044880380E0250680AC5B068036590680A2D50600E98A060084880380855306804C
:20154000022A11D094F85030012B16D87A497B4A1CA854F08FFF1CA940F2A4400DF0AAFEBA
:2015600000283FF42BAFBAE70222002340F2B9400DF08BFF0028E5D0B1E70222002340F2AE
:20158000A5400DF082FF0028E0D0A8E710F0F6FC00283FF463AF00230222694969481EF06A
:2015A000FDFE00287FF45AAFB0E60CA820340CAE22F082FB0FCE0FC496E80F0084E80F00ED
:2015C0002022002104F1300053F05FFB00230122CDE901335C490092B1F830111A464046AF
:2015E00014F096F800287FF47AAF9DF8540008B112F014FD554B93F88D312BBB54491CA8B0
:2016000055F0BAFE002302224D491CA81EF0C6FE00283FF47BAE0FF05DFE08B10FF010FEB6
:20162000002302214B4887F82D351EF0F7FF2A2009F09CFC05230220BB7011F017F8012269
:20164000454B83F8802062E610F098FC0028D5D0002302223A493B481EF0A0FE0028CDD177
:2016600054E600230122CDE9013337490092B1F830111A46404614F04BF800287FF42FAF5E
:201680009DF8540008B112F0C9FC304B93F88D31002B3CD1304C94F8DC60002EAED02F4E78
:2016A00096F85030EBB12E4B987D0AF091F88DF870000DF1710012F0EFF800230322204971
:2016C0001CA81EF06BFE96F85030012B09D90DF1710012F0E9F80023032219491CA81EF0E5
:2016E0005DFE0023032216491E481EF057FE1E491CA855F041FE0023022211491CA81EF0FD
:201700004DFE00283FF402AED4E91E10DEE610F035FC0028BED000230222094909481EF0E5
:201720003DFE0028B6D1F1E57725F0E57C25EEE57525ECE52546EAE544400700AF0E070010
:20174000A2D50600CD8A0600E0250680AC5B0680F78A06002DE50600688703805E52068050
:201760003659068044880380E98A0600002200232DE9F04FADF5777DCDE91623CDE918237C
:20178000CDE91A23CDE91C23CDE91E23CDE92023CDE92223CDE92423CDE926232D4B2E4A8A
:2017A0009B792E4E002B2E4B054618BF1E462D4B08BF13462C4A0A932C4B08BF13462C4AB7
:2017C000099308BF91462B4B2B4A18BF99462B4B08BF13460021082226A8089353F055FA52
:2017E000274BDB7873B34FF400734FF0010B00220DF13607CDE9003B029776AB114630204E
:201800000CF0A6FC002840F0C282DFF878A04CAB76AA398830200CF077F99AF81A30002B04
:2018200060D1112D00F065819DF83181B8F1000F2AD0B8F1080F55D05E2738460DF5777D8C
:20184000BDE8F08F022009F095FD0028CBD14B27F3E700BF0953068039DD06006ADC06009E
:2018600053DC06002DDD060067DD060059DD060042DE06002CDE0600FBDD0600DADD0600CC
:20188000509A0380F886038044A8C24C22F014FA0DF5887CBCE80F000FC49CE80F000DF59F
:2018A000887E84E80F00BEE80F0010340FC49CE80F0084E80F0044A90EA80DF0DBFDCDE99F
:2018C00001B7CDF80080434605220EA913200CF03FFC07460028B0D10FF008FA9AF80400AD
:2018E00011F07CFCAC4B9A7E002A3DD14FF400730A210DF13604CDE90031029476AB11461A
:2019000010200CF025FC0746002896D110AB76AA218810200CF0F8F89DF840300BB9ADF890
:201920004430BDF84200BDF84410DFF86882A8F8F201A8F8F41112F0DDFB4FF400730A227E
:20194000CDE900320022029476AB114620200CF0FFFB074600287FF470AF08F5087376AA9A
:20196000218820200CF0D0F88C4B112DB3F8301140F0DB808A4B30461B78042B18BF012227
:201980004FF0000318BF00921A46CDE9013308BF009313F0BDFE074600287FF44EAF9DF8C0
:2019A000340108B112F03AFB7A4C7E4E2946B4F8F40112F0ABFAB07D09F00AFF8DF85001B4
:2019C000B07D09F005FF784B94F8F7619B798DF89401022B02BF13238DF850318DF8943194
:2019E00016F002063AD171490DF2511055F0C4FCB4F822226E490DF2951054F03BFD33466F
:201A0000022265A954A81EF0C9FC6A490DF2511055F0B2FC94F828326749009394F82932AF
:201A200094F82A220DF2951054F024FD3346022265A954A81EF0B2FC60490DF2511055F014
:201A40009BFCD4F824225A490DF2951054F012FD3346022265A954A81EF0A0FC122D09D1D9
:201A60004D4CA37E002B67D0554B93F8A030002B40F0E78021F078FB0FF02CFC002840F08A
:201A80000D810FF027FC002840F0088109F0B6F8074600287FF4D1AE3F4E33782BB941F258
:201AA000E8123E49474853F0ECF80FF013FC002840F0F480444A537F9046012B00F02F8113
:201AC00098F81D30022B40F05A81102200213CA8334C53F0DAF8082216A93CA853F0D1F84D
:201AE000237A002B00F0558114A940A8FFF764F858E10FF0FBF8274C9AF8040011F06EFBC3
:201B000044AF44A822F0D8F80FCF0FC497E80F000DF5887C84E80F00BCE80F0010340FC47A
:201B200097E80F0084E80F00DCE600230122CDE90133009225482CE70FF09AFB022849D1C0
:201B4000082216A91EA853F09CF8082218A920A853F097F808221AA922A853F092F80822CC
:201B60001CA924A853F08DF80B4B1B78002B40F08D87122009F0FAF9032115481EF04EFDBC
:201B800000283FF464AE05220027054B9A7083F82D7552E668870380F8860380E0250680DD
:201BA000509A038036590680095306807C9B0600889E06008D9B06008C9E0600769C060002
:201BC0005E520680F8130680C358068048DD06002DE506009A4991F8F7315B072ED540F22F
:201BE000FD300EF027FC00BB964B93F85030012B1BD9944E96F8502042B993494FF48360F3
:201C00000DF058FB074600287FF417AE96F85020012A7FF629AF002340F2B9400DF035FCD5
:201C2000074600283FF420AF07E6884940F2FD300DF040FB07460028DBD0FEE501F58E71E0
:201C4000F4E7A67E002E60D10FF012FB02283FF477AF4FF4007A4FF001080DF136040294C4
:201C6000CDE900A876AB3246314630200CF070FA074600287FF4E1AD4CAB76AA21883020BA
:201C80000BF042FF724B9DF8312183F82D25539AC3F830250FF01EFB024608B17527CCE534
:201CA0003C230146CDE900A3029476AB14200CF04FFA0646074600287FF4BFAD604F39ABC2
:201CC00087F8800076AA218814200BF01DFFDDE93A1207F1DC0011F011FE334603225D49B7
:201CE00007F1DC001EF05AFB00283FF4B0ADCDE90184CDF800A076AB42460DF13501212037
:201D00008DF835600CF024FAB4E600230322514951481EF043FB00287FF4ACAE97E52D226E
:201D200054AC1A5501333F2BFBD100230222494920461EF033FB00283FF489AD47490DF22F
:201D4000511055F019FB00230222424920461EF025FB00283FF47BAD1FF0A8FAB8B901239A
:201D60002D22E25401333F2BFBD100230222394920461EF013FB00287FF4A2AE67E50022D0
:201D800014A928461EF008FE00283FF49EAE074653E56422002312A9CDE9122340A814AAE3
:201DA00017F095FE3CA940AA084617F037FE08223CA91AA852F065FF102200213CA852F040
:201DC00064FF082218A93CA852F05BFF237A002B30D16422002312A9CDE9122340A8204ACB
:201DE00017F075FE3CA940AA084617F017FE08223CA91CA852F045FF122D40F05086002270
:201E0000002330A9CDE92823CDE92A23CDE92C23CDE92E23CDE93023CDE93223CDE9342395
:201E2000CDE9362308460E230E4A17F09EFDD8B1482702E50A4940A8FEF7BEFED2E700BFD7
:201E4000688703805E5206808553068084880380509A0380A2D506004488038062D8060074
:201E6000A83006807830068034A90E23514A084617F07BFD0028DBD132AA0E2311461046D2
:201E800017F073FD0028D3D136AA0E231146104617F06BFD0028CBD10546474C04F50966C8
:201EA00028A90E237219084617F05FFD0028BFD12035802DF4D1054604F6984628A900234E
:201EC0007219084617F051FD0028B1D12035B5F5C07FF3D1054604F698062CA90E237219B4
:201EE000084617F042FD0028A2D12035802DF4D1054604F54A662CA900237219084617F020
:201F000034FD002894D12035B5F5C07FF3D1054604F50A662AA90E237219084617F025FD47
:201F2000002885D12035802DF4D1054604F6A8462AA900237219084617F017FD00287FF4A4
:201F400077AF2035B5F5C07FF2D1054604F6A8062EA90E237219084617F007FD00287FF4E0
:201F600067AF2035802DF3D1054604F54B642EA900236219084617F0F8FC00287FF458AF32
:201F80002035B5F5C07FF2D10C4B1B79F3B90C4B9D7E0C4B93F8A030002B00F0FF84002DBA
:201FA00040F062850BF046FD0122074B83F87A2000F05ABD80300680E0250680C3580680D9
:201FC000F88603805E5206806C1A0010BC4DBD4CA87D09F0FDFBA2798DF85001022A08BF28
:201FE000132349460DF2511008BF8DF8503155F0C3F900230322B44954A81EF0CFF90028AF
:202000003FF425ACA87D09F0E3FBA3798DF85001022B04BF13238DF85031AC4B1B78002BED
:2020200000F08C830025DFF8CCA2102453462E462F46A846AB46CDE905550795F3E8020118
:2020400018EB000805984BEB010BD3E91E2182180592069A04F1FF3441EB02020692D3E91E
:202060003E21BF18079A41EB02020792D3E95E21AD1841EB060614F0FF04DFD1944B93F867
:202080000490B9F1010F00F0AA83B9F1000F00F0DC80B9F1030F00F2D8800BD13F222D213F
:2020A0000DF2511052F0F1FD23464A46864954A81EF074F987490DF2511055F05DF914A9C9
:2020C00065A8CDE9148BFEF7B3FE0023032265A954A81EF063F900283FF4B9AB7C4C237919
:2020E000032B1BD14FF00008FAE802235FFA88F008F101081DF0F2FCB8F1100FF4D1247980
:20210000032C0BD13F222D210DF2511052F0BDFD002322466C4954A81EF040F96E490DF270
:20212000511055F029F9079B14A965A815931497FEF77EFE0023032265A954A81EF02EF920
:2021400000283FF484AB624C2379032B19D10027DFF8A481F8B2F8E8022301371DF0BEFCC2
:20216000102FF7D12479032C0BD13F222D210DF2511052F08AFD00232246534954A81EF0A7
:202180000DF956490DF2511055F0F6F8059B14A91493069B65A81593FEF74AFE0023032228
:2021A00065A954A81EF0FAF800283FF450AB484C2379032B19D10027DFF84081F8B2F8E82E
:2021C000022301371DF08AFC102FF7D12779032F0BD13F222D210DF2511052F056FD002393
:2021E0003A46394954A81EF0D9F83D490DF2511055F0C2F814A965A8CDE91456FEF718FE28
:202200000023032265A954A81EF0C8F800283FF41EAB2379032B18D10025324EE8B2F6E8AA
:20222000022301351DF05AFC102DF7D12479032C0BD13F222D210DF2511052F026FD00239C
:202240002246214954A81EF0A9F827490DF25110264E55F091F8D6E9002314A965A8CDE98D
:202260001423FEF7E5FD0023032265A954A81EF095F800283FF4EBAA1D490DF2511055F068
:202280007BF8D6E9042314A965A8CDE91423FEF7CFFD0023032265A954A81EF07FF800286E
:2022A0003FF4D5AA0024A6F58466334610222746A3462546A146CDE90544079420E000BF17
:2022C0003659068009530680A2D50600F8860380C358068080DD06009CDD0600B8DD06006B
:2022E000C9DD06001090038089DD0600B0900380A5DD0600908E0380908F0380108F0380F3
:20230000F3E802012D1849EB0109996F013A0846D96F0B910599091805910B98069940EB25
:2023200001010691D3E93E101BEB010B079940EB01010791D3E95E10641840EB070712F0A2
:20234000FF02DDD1DFF81C8398F8160009F040FAB84B8DF850019B790A99022B08BF1323C5
:2023600054A808BF8DF8503155F006F800230322B14954A81EF012F800283FF468AA98F8FE
:20238000160009F025FAAB4B8DF850019B79022B04BF13238DF85031A84B93F80480B8F158
:2023A000030F0BD13F222D210DF2511052F06DFC00234246A04954A81DF0F0FFDFF87C8214
:2023C00098F80430012B00F06582002B00F07D81032B00F27A819A490DF2511054F0CCFFB0
:2023E000DDE928325D1942EB090214A965A8CDE91452FEF71DFD0023032265A954A81DF0BB
:20240000CDFF00283FF423AA98F80430032B33D10025DFF854A2FAE808894B46F6E80201FB
:2024200010EB080241EB0303E8B201351DF056FB042DF0D1DFF834A2824EF6E808894B46C8
:20244000FAE8020110EB080241EB0303E8B201351DF044FB102DF0D1784B1D79032D0BD1E1
:202460003F222D210DF2511052F00FFC00232A46714954A81DF092FF73490DF2511054F0B9
:202480007BFFDDE92C32079913EB0B0342EB0101CDE9143165A814A9FEF7CAFC00230322FB
:2024A00065A954A81DF07AFF00283FF4D0A9634B1B79032B34D10025DFF8B4A1634EF6E863
:2024C00008894B46FAE8020110EB080241EB0303E8B201351DF002FB042DF0D1DFF894A1E6
:2024E0005B4EF6E808894B46FAE8020110EB080241EB0303E8B201351DF0F0FA102DF0D152
:202500004E4B1D79032D0BD13F222D210DF2511052F0BBFB00232A46474954A81DF03EFF10
:202520004C490DF2511054F027FFDDE92A32059965A85B18069942EB0101CDE9143114A976
:20254000FEF776FC0023032265A954A81DF026FF00283FF47CA9394B1B79032B34D10025A0
:20256000DFF814A13C4EF6E808894B46FAE8020110EB080241EB0303E8B201351DF0AEFAA4
:20258000042DF0D1DFF8F4A0344EF6E808894B46FAE8020110EB080241EB0303E8B2013570
:2025A0001DF09CFA102DF0D1244B1D79032D0BD13F222D210DF2511052F067FB00232A4623
:2025C0001D4954A81DF0EAFE25490DF2511054F0D3FEDDE92E321C1942EB070714A965A861
:2025E000CDE91447FEF724FC0023032265A954A81DF0D4FE00283FF42AA9104D2B79032B27
:2026000063D10024DFF87890DFF87880F8E808673B46F9E80201821941EB0303E0B201346C
:202620001DF05CFA042CF1D1DFF85C90DFF85C802EE000BF09530680A2D50600C358068002
:2026400080DD0600783206809CDD0600782E068080320680B8DD0600802E068088320680F5
:20266000C9DD060036590680702E0680B08C0380908D0380B08D0380108D0380308D0380F6
:20268000108E0380882E0680308E038090320680F8E808673B46F9E80201821941EB0303D3
:2026A000E0B201341DF01AFA102CF1D12C79032C0BD13F222D210DF2511052F0E6FA002330
:2026C0002246AC4954A81DF069FEAB4CAB490DF2511054F051FEDDE93010D4E900325B18E7
:2026E00040EB020214A965A8CDE91432FEF7A0FB0023032265A954A81DF050FE00283FF44D
:20270000A6A89F490DF2511054F036FEDDE93410D4E904325B1840EB020214A965A8CDE98C
:202720001432FEF785FB0023032265A954A81DF035FE00287FF42BACFFF789B8914901F6D2
:20274000481001F62813D3E90023C0E9002301F5156001F51363D3E90023C0E9002301F6CB
:20276000581001F63813D3E90023C0E9002301F5166001F51463D3E90023C0E90023D1E9C6
:20278000802301F59F60C0E90023D1E9822301F5A060C0E90023D1E9842301F5A160C0E9B3
:2027A0000023D1E9862301F5A260C0E90023102001F5A561F1E80223C1E97E23D1E91E235F
:2027C000C1E99E23D1E93E23C1E9BE23D1E95E23C1E9DE23431E13F0FF00EBD122E46A492A
:2027E0000DF25110694D54F0C7FDD5E9002314A965A8CDE91423FEF71BFB2346032265A97C
:2028000054A81DF0CBFD00283FF421A860490DF2511054F0B1FDD5E9042314A965A8CDE963
:202820001423FEF705FB2346032265A954A81DF0B5FD00283FF40BA856490DF2511054F0C4
:202840009BFDD5E9022314A965A8CDE91423FEF7EFFA2346032265A954A81DF09FFD0028FF
:202860003EF4F5AF4C490DF2511054F085FDD5E9062314A965A8CDE91423FEF7D9FA2346F8
:20288000032265A954A81DF089FD00287FF4DDACFEF7DDBF3B4C3C490DF2511054F06CFDA8
:2028A000DDE92810D4E980325B1840EB020214A965A8CDE91432FEF7BBFA0023032265A943
:2028C00054A81DF06BFD00283EF4C1AF30490DF2511054F051FDDDE92C10D4E984325B186A
:2028E00040EB020214A965A8CDE91432FEF7A0FA0023032265A954A81DF050FD00283EF44E
:20290000A6AF24490DF2511054F036FDDDE92A10D4E982325B1840EB020214A965A8CDE98B
:202920001432FEF785FA0023032265A954A81DF035FD00283EF48BAF17490DF2511054F0B4
:202940001BFDDDE92E10D4E986325B1840EB020214A965A8CDE91432FEF76AFA00230322DD
:2029600065A954A81DF01AFD00287FF4AEAEFEF76EBF00BFA2D506009090038089DD0600C5
:20298000A5DD06006887038080DD0600608C03809CDD0600B8DD0600C9DD0600002D6CD13B
:2029A0000EF066FC02283FF4CBA84FF4007801260DF136040294CDE9008676AB2A462946FB
:2029C00030200BF0C5FB074600287EF436AF4CAB76AA218830200BF097F83D4B9DF8312117
:2029E00083F82D25539AC3F830250EF073FC024600287FF453A93C230146CDE9008302944C
:202A000076AB14200BF0A4FB0546074600287EF414AF304F39AB87F8800076AA2188142073
:202A20000BF072F8DDE93A1207F1DC0010F066FF2B460322284907F1DC001DF0AFFC00282B
:202A40003EF405AF76AB32460DF13501CDE90164CDF8008021208DF835500BF079FB0AF0AF
:202A6000E9FF1E4B83F87A60022109981DF0D6FD00287FF465A8FEF7EABE032216491848E3
:202A80001DF08CFC0028EFD1FEF7E1BE032108981DF0C4FD00287FF46CA8FEF7D8BE3378AE
:202AA0006BB903210F481DF0B9FD00283EF4CFAE05232846A37008F059FAFEF7BEBE032154
:202AC00008981DF0ABFD0028EBD1FEF7C0BE00BF509A038068870380A2D506006C1A001099
:202AE000448803802DE506002DE9F04FB94BBA4A93F84D30ADF5757D03F01003002BB74B43
:202B000008BF13460593B64BB64A18BF9846B64B0CBF90469946B54AB54B0CBF91469A4645
:202B2000B44AB54B08BF924693F8502005460E4632B19B78012B40F27485102900F06E85F5
:202B4000AE4B5A7B012A00F26C8595F82920062A00F26A850021AA4A102E82F8F61100F0EE
:202B6000AA80A84C6278002A40F0A580627A002A4BD1A27A002A48D1DB7C002B45D00123A2
:202B80006372A37E002B40F090809D4F21A821AC21F092F80FCC0FC794E80F0007F1300C47
:202BA0000DF1840E87E80F00BEE80F00ACE80F0094E80F008CE80F00934B1B78022B2FD103
:202BC00029A921A821F0D0F832A907F1500021F0CBF829A854F098FC044632A854F094FCE9
:202BE000854B201ADA796FF03B03534303F5A83303F5C073984213D903200FF037FD1624F1
:202C000020460DF5757DBDE8F08F7F4BDB78002BB7D1022008F0AEFB0028B2D14B24EFE7B3
:202C200021A90EA80CF026FC4FF0800B01230DF13607CDE900B3029770AB05220EA915209D
:202C40000BF086FA04460028DAD10EF04FF86D4B187910F0C3FA0A232246CDE900B321462C
:202C6000029770AB10200BF073FA04460028C7D170AA10AB398810200AF046FF9DF8402004
:202C800032B9BDF84230ADF844200133ADF84230BDF84410BDF8420011F02CFA304613F02E
:202CA00049FA0122564B83F8F621544B1B7C002B57D020F059FA0EF00DFB0746002840F0E5
:202CC000198295F838302F2B05D195F83970A7F12F02574257414B4C617829B90C2204F18F
:202CE0005C00218351F0D1FF434B93F89430012B00F09A80002B00F08F80022B00F09F804A
:202D00003E4B1B7E0593002B00F0BF804FF482722021B3A851F0B9FF402290A95DA851F0F2
:202D2000B0FF00235DA88DF8B43154F046FBDFF8E4A081469AF8023083420593C0F29182C5
:202D40009AF80080314B9AF801404344987808F005FB0FF067FD04EB0903834276DD912458
:202D60004EE7032E00F26384DFE806F002121D280123CDE901330093002350461A462449D7
:202D8000B1F8301112F0C4FC0446002891D037E70123CDE90133009300231D491A46B1F863
:202DA00030114846EEE70123CDE901330093002317491A46B1F830114046E3E70123CDE9D7
:202DC00001330093002312491A46B1F830110598D8E700BF3753068045D8060073D80600C5
:202DE00028D806000BD80600F7D70600E3D7060097DF060083DF06005E520680C358068095
:202E000068870380F8860380509A038036590680E02506806A59068005F13803B64A8B210C
:202E200090A853F05DFB6BE7238B05F1380200920133B24A8B2190A853F052FB60E795F885
:202E4000293004EB4304B4F85A30EEE79AF9033008F1FF3801345FFA89F208EB88187BB11A
:202E6000059B5DA91C44A4EB090909EB0800B3AB184407F0A5FC0446002800F09E80BFE638
:202E80004444B3AB5DA91819F3E7002F40F09580DFF86C820DF5107998F8030008F05EFA94
:202EA0000FF0C0FC8346484654F087FA09909DF824309B45089309D398F8030008F04EFA8F
:202EC0003A460146484607F07DF8D4E73C46DA46CDF8288019F80A30202B05D009EB0A03FB
:202EE00013F8013C202B3DD14A2200215DA851F0CCFE09EB04015A465DA851F0C2FE0AEB00
:202F00000B03DBB20B930A9BD87808F027FA002201465DA807F056F8044600287FF470AEB4
:202F2000089B9A4549D2D0460B9B089A934216D34A2200215DA851F0A8FE9DF8242090AB4B
:202F400003EB0801A2EB08025DA851F09AFE6C4BD87808F003FA002201465DA8B3E7444677
:202F60009A46B7E7D04608F1FF33DBB219F80320202A03D09C429846F5D1D0464A2200218F
:202F80005DA851F082FEA8EB040209EB04015DA851F077FE0A9BD87808F0E0F900220146EF
:202FA0005DA807F00FF8044600287FF429AE089A08EB0B039045DBB2B7D312A8D5E9022326
:202FC000CDE91223FDF70DFE002840F03383D5E9042314A8CDE91423FDF703FE002840F01E
:202FE0002C83032212A94CA8FDF792FF14A95DA8FDF75EFF5DAB4CAA42493BA853F03AFAD3
:20300000414B1A7E002A00F08580102E36D03E4B5B7C002B63D03BA854F0CFF9DFF8F09025
:20302000804699F824408442C0F21B8199F822A0334B99F823B05344987808F08FF90FF066
:20304000F1FB0BEB080383423FF789AE99F925100AF1FF330BF101005FFA88F203EB831309
:2030600011B12044A0EB08001844B3AB3BA9184407F0A6FB0446002838D0C1E523495DA874
:2030800054F07AF95DA854F098F9DFF884801C4B98F8889004464B44987898F889A008F01B
:2030A0005DF90FF0BFFB0AEB040383423FF757AE98F98B1009F1FF330AF10100E2B203EB2F
:2030C000831311B105990144081B1844B3AB5DA9184407F075FB0446002898D090E5DDE9FA
:2030E0001223002B08BFB2F57A7F94D10EF0F2F800283CD0752483E5444007000DCE06001B
:203100003659068018D70600C35806804CDC06006A5906805B7C8BB9DDE91223002B08BF85
:20312000B2F57A7F0AD1102EE0D1002FDED1032172481DF073FA0028D8D16FE5102E0CD1AF
:203140006E495DA854F018F9002FCFD13B4603223BA95DA81DF022F9EDE7694B187908F0C7
:20316000FDF800238DF874018DF87531ECE712AA14A91CA816F0ABFC1EA8FDF72BFD08B9B2
:2031800060243DE54FF47A7200231CA9CDE9182316A818AA16F00DFC16A8FDF722FD0028F9
:2031A000EED1584B9B78C3B9D5E90830DDE916219B18069340EB01030793D5E90601DDE98B
:2031C00006348C4208BF8342C0F03A82069B1A1A079B63EB0103CDE9162316A8FDF701FD87
:2031E000002840F03082D5E9082313433BD1D5E90623134355D116A94CA8FDF759FE05F123
:2032000029015DA81FF0C8F9044600287FF4F8AC5DAB4CAA3C493BA853F02CF995F8288023
:20322000B8F1100F00F21282384B1B7E002B00F0A081B8F1000F5DD0354B08F1FF314022F8
:2032400003EB81115DA851F01CFD8DF8B4415DA854F0B3F8DFF8C8A081469AF846B08345CB
:2032600060DA9024CCE405F1200421464CA8FDF71FFE6FB1274B06F1830103EBC101224605
:203280000E23084616F071FB0028B0D08A24B7E43B4603224CA920481DF080F80028E9D1E2
:2032A000BCE405F1180421464CA8FDF701FE144B587908F053F819498DF874010DF27510BB
:2032C00054F05AF86FB1134B06F17F0103EBC10122460E23084616F048FB00288BD08B2451
:2032E0008EE43B4603224CA95DA81DF057F80028E9D193E48DF87481A9E700BF4CDC060010
:20330000365906805E52068020D70600C358068002660680E0250680F5DB0600EDDB0600A7
:203320006A5906809AF84440CA4A9AF8453022449078059308F012F80FF074FA059B03EB10
:20334000090282423FF70BAD581C9AF94730013C5FFA89F204EB841413B15844A0EB0900A6
:203360002044B3AB5DA9184407F02AFA044600287FF446AC3BA854F020F8DFF8E0A28146D8
:203380009AF868408442FFF66CAF9AF866B0B14A9AF867305A449078059307F0DFFF0FF03F
:2033A00041FA059B03EB090282423FF7D8AC9AF969100BF1FF3001335FFA89F200EB801001
:2033C000002900F0C1801C44A4EB09042044B3AB3BA9184407F0F4F9044600287FF410AC10
:2033E0004FF00009DFF884B2DFF884A2B3AC41220DF28F31204652F02FFA002840F0A680AB
:2034000009F10109B9F1030F04F14104EFD10DF061FF00287FF46EAED5E90623134306D0CB
:203420008D4B06F1400003EB40001FF0E0FED5E90823134306D0884B06F1440003EB400011
:203440001FF0D5FE16AA3146404607F05FFD044600287FF4D5AB324616A9284607F0D4FDA8
:20346000044600287FF4CCAB95F82930002B00F0A480013B5FFA83F8784B422493F8662081
:20348000744B04FB08F41344987807F067FFDFF8E491A11C8DF87401492249440DF275102F
:2034A00053F0DCFF00238DF8B43139F8042016A91AA807F063FD1AA93BA8FDF7F9FC684BF2
:2034C000B3F80B30DB057BD5102E40F09680654BD97816A807F01AF9044600287FF490AB69
:2034E000604FBB7A1BB9DDE91623C7E904237B78DFF88481002B40F08280304607F036FD72
:20350000012295F829303A83082007EB4307A7F85A200FF0ABF8D8E90E100FF0FFFF0023C7
:2035200088F8F63195F8292098F8F134002A72D00121013A01FA02F21343DBB288F8F13419
:203540000DF0CCFBFFF75CBB184440E71BF8090007F004FF2070002F7FF452AF3B46032228
:20356000514620461CF01AFF00287FF449AFFFF755BB384B587907F0F1FE8DF87401B8F1B3
:20358000000F17D0384B08F1FF31402203EB81110DF2751051F075FB002F7FF438AF3B4668
:2035A00003223BA95DA81CF0F9FE00287FF42FAFFFF734BB8DF87581EEE74FF003085BE7C0
:2035C000002F81D1264B93F84F30032B3FF47CAFB8F1030F0DD1012B7FF476AF00230322BE
:2035E0003BA95DA81CF0DAFE00287FF46DAFFFF715BB022B3FF468AFF0E7314669E73B8BA6
:2036000001333B8395F829302B3307EB4307BB880133BB8083E743F008038FE73724FFF717
:20362000EFBA3524FFF7ECBA3324FFF7E9BA3924FFF7E6BA6224FFF7E3BA6124FFF7E0BADB
:203640005F24FFF7DDBA4824FFF7DABA6324FFF7D7BA00BF36590680E02506806A590680AE
:203660005E520680F88603800266068039590680A2D506006A6B06806887038000230A2274
:20368000F0B53A4F85B0CDE9012300931A46194606200AF05DFD0DF029FB3B78082B08D042
:2036A000022133481CF0BAFF50B94B24204605B0F0BD03212F481CF0B1FF0028F0D1F4E74C
:2036C0002D4EB37E5BB9F17806F1100201F5AE732A4901EBC30108460E2316F046F9284C46
:2036E00004F120050FCD0FC495E80F0084E80F00244B5B782BB1244B5B7E13B9012017F0A0
:203700003BFE224D95F89D3013B1012013F0AAFB747A44B395F84E30012B07D1AC792CB91C
:203720001B4BC3E98D4408F065F8BFE7002419481FF05DFD18481FF05AFDF3780F48B3334F
:2037400000EB43001FF053FD0EF09AFF70220021094851F09AFA1FF007FDAB79BC70012BDD
:20376000A4D1AC71A2E70523BB709FE7509A03802AE50600FFDB0600F8860380E025068067
:2037800088870380AC5B06806C1A00105E520680688703801A2706802C27068000232DE9F3
:2037A000F04FADF24C7D00220C930023A54ECDE97C2396F84D30A44A03F01003002BA34B1E
:2037C00008BF1346A24A1293A24B08BF1346A24A1193A24B08BF1346A14A1093A14B08BF4D
:2037E00013460F93A04B0E91A04A9979A04B0546002918BF1A469F4B13925B7B002B41F0F1
:203800006E809D4B9B7E83BB0EF000FE0DF062FD08B175249EE00423984F012487F82D353F
:2038200080230C9A0DF5B378CDE90034CDF808800DF59563114630200AF08AFC0446002848
:2038400040F088808AAB0DF59562B8F8001030200AF05AF90DF03EFD0028DAD19DF82932AA
:2038600087F82D35919BC7F8303596F84C30824F0D9366ABAB9368ABAC936AABAD936CAB8F
:20388000AE930DF58963AF930DF58A63B0930DF58B63B1930DF58C63B2930DF58D63B393E3
:2038A0000DF58E63B4930DF58F63B5930DF59063B6930DF59163B7930DF59263B8930DF5D0
:2038C0009363B99308220DF5946300217AA8BA9351F0DBF93B8B002B00F0F48040F22140F6
:2038E0000CF0A8FD48BB664EB07B07F037FD0022014605F1880006F065FB044650BB12F086
:2039000069FF05F18201EEA81EF046FE044608BBF9785CA806F0FAFE0446D8B9002200234E
:20392000CDE96023CDE96223564BB5F980209B78022B14D0BAB133240CE0524B93F8963064
:20394000002BD0D0504B93F8F20410F0CBF804460028C8D020460DF24C7DBDE8F08F93B21C
:20396000632B00F2BF8712B2D3175EA8CDE95E23FDF730F90446B8B10DF0ACFC00287FF486
:2039800048AFB5F98030002B53DD5CAA60A964A815F0FEFF002840F0A88764A8FDF721F9B9
:2039A000002879D04824D5E75CA9DDA8FDF761FADDAA3649BBA852F05DFD307C07F0CEFC23
:2039C00033498DF8FC030DF2FD3053F0D5FC9DF8FC332BBBF07B07F0C1FC2E498DF8FC03E3
:2039E0000DF2FD3052F046FDB5F9802060A9D317BBA8CDE96023FDF75BFA60A9CCA8FDF77F
:203A000057FACCAA2149BBA852F034FD00230322BBA9FFA81CF0C2FC0028ADD14B2499E7ED
:203A200023460322BBA9FFA81CF0B8FC0028D1D1F4E70E235CAA62A964A815F096FF002878
:203A4000ABD0AFE73753068045D8060073D806000BD8060028D80600E3D70600F7D706004E
:203A600083DF060097DF060009530680FBDD0600DADD0600C3580680F8860380509A0380D6
:203A8000365906805E5206806887038026D7060090D80600848A0600294CA37D6BB95EA825
:203AA000FDF798F880B1D5E9002366A8CDE96623FDF797F8C8B141244CE764A8FDF78AF80D
:203AC0000028ECD08E2445E7637B002BEBD1B5F980305EA9002BCCBF08222622284607F06D
:203AE00093FA04460028DED034E768A8D5E90223CDE96823FDF775F8002840F0F986D5E9D4
:203B000004236AA8CDE96A23FDF76BF8002840F0F286D5E906236CA8CDE96C23FDF761F875
:203B2000002840F0EB86D5E908230DF589642046C4E90023FDF755F820B149240AE700BF7F
:203B4000C35806800DF58A60D5E90A23C4E90223FDF747F80028F0D1D5E90C230DF58B6025
:203B6000C4E90423FDF73DF80028E6D1D5E90E230DF58C60C4E90623FDF733F80028DCD1C2
:203B8000D5E910230DF58D60C4E90823FDF729F80028D2D1D5E912230DF58E60C4E90A23D0
:203BA000FDF71FF80028C8D1D5E914230DF58F60C4E90C23FDF715F80028BED1D5E91623C8
:203BC0000DF59060C4E90E23FDF70BF80028B4D1D5E918230DF59160C4E91023FDF701F8B8
:203BE0000028AAD1D5E91A230DF59260C4E91223FCF7F7FF0028A0D1D5E91C230DF59360DD
:203C0000C4E91423FCF7EDFF002896D1D5E91E230DF59460C4E91623FCF7E3FF00288CD11D
:203C20000646A64B0DF5926293F8A370DDE97C34F1B28F4200F2AD8008B1CDE97C34A04BA0
:203C4000587C07F08BFB64A902469E4806F09CF9044600287FF47EAE6EAC0E236AAA68A9CC
:203C6000204615F082FE00287FF49CAE0E236CAA2146204615F079FE00287FF493AED4E94B
:203C800000230646CDE970230DF5896700233A462146204615F069FE00287FF483AE01369B
:203CA0000C2E07F10807F1D164AA214672A815F06FFE002840F025860E23224666A972A83B
:203CC00015F053FE00287FF46DAE72AA64A974A815F05EFE002840F017860446774E96F8A0
:203CE000A33062B2C3F10A039A425ADBDDE96601DDE97434A14208BF984216D0C21A61EBDE
:203D00000403CDE97223704B0021DA7DDDA8003218BF012207F0C2FA694B987C07F01EFBE2
:203D200072A90246DDA806F088F8644B93F85030002B6CD0DDE97023134311D0624B102196
:203D4000DA7DDDA8003218BF012207F0A7FA5C4B987C07F003FB70A90246DDA806F06DF8D2
:203D60007CA8FCF737FF48B34FF00E09564F544E0DF52B7858F829402046FCF72BFF5FFA24
:203D800089F1002830D0B9F10F0F56D04FF00F09F0E772E802011B1841EB04040136012049
:203DA00046E70DF5896101EBC20270A90023084615F0DBFD0134002891D0F3E5424B0D2182
:203DC000DA7DDDA8003218BF012207F067FA3C4B987C07F0C3FA7CA90246DDA806F02DF827
:203DE00004460028C0D0B5E5FA7DDDA8003218BF012207F053FAB07C07F0B0FA214602463F
:203E0000DDA806F01AF804460028BCD0A2E5DDE96E23134311D02C4B1021DA7DDDA800324C
:203E200018BF012207F03AFA254B987C07F096FA6EA90246DDA806F000F8234B93F8223035
:203E4000012B49D074A8FCF7C5FE002800F09A800DF040FA00287FF4DCAC1B4BDB7B032BD5
:203E600000F0C1804FF00009184F194EDFF86480F97876A801EB890101F19703AF3106EBDE
:203E8000C30306EBC101D3E90023CDE97623D1E90023CDE97823FCF79DFE002800F06281C4
:203EA00098F8F13423FA09F3D80700F15B8109F10109B9F1060FDBD19AE000BF5E520680AA
:203EC000365906808CD90600C3580680F8860380E025068068870380AD4B0024987C07F09C
:203EE0003DFAAC4B8DF8FC0393F850300DF52B78002B0CBF10260D2663B2B34215DA58F8B8
:203F00002300FCF767FE013407460028F4D1A2490DF2FD3053F030FA3B4603229F49FFA8FE
:203F20001CF03CFA00283FF479AD4FF0000AABAFDFF86C82DFF8589207E057F82340204696
:203F4000FCF748FE40B10AF1010A4FFA8AF39E425FFA8AFBF1DC75E798F8172059460032EC
:203F600018BF0122DDA807F099F999F8120007F0F5F921460246DDA805F05FFF04460028B8
:203F8000E1D0E7E4864E96F82220012A1ED096F82230022B7FF45CAF7D4EF07C07F0DEF958
:203FA00066A902467F4805F0EFFF044600287FF4D1ACF07C07F0D2F974A902467A4805F054
:203FC000E3FF044600283FF443AFC3E4704BD87C07F0C4F974A90246734805F0D5FF0446CB
:203FE0000028D4D0B6E405F0D1FC00287FF43AAF0DF070F900287FF40CAC06F077FC6B4E3A
:20400000044618B13378002B3FF4A4AC60A806F089FC044618B13378002B3FF49BAC62A844
:2040200006F0A2FC044618B13378002B3FF492AC66AA74A972A815F0ABFC0DF5896300931E
:204040006AAA6CAB68A972A806F0FAFC574E044618B13378002B3FF47DACF17872A806F0BB
:20406000CFFB044618B13378002B3FF473AC0DF512790DF51E7B5C464F460022CA46F3783F
:204080004B4E973306EBC3030132062AD3E93001E7E80201F3E80801E4E80201F4D106F076
:2040A000FBFB044620B1414B1B78002B3FF452AC0DF010F900287FF4ACAB06F079FC06F01B
:2040C00093FC06F0A7FC364B1B7C012B56D011F017FA044600287FF43DAC344B9A7E1F4672
:2040E000002A40F0FF820DF0F5F800287FF491AB284B9A789846022A40F08D800BF070FBF2
:20410000044600287FF426AC2A4D0DF5A5600DF5A5641FF0D1FD0FCC0FC594E80F0005F152
:2041200010060DF5A56C85E80F00BCE80F000FC694E80F005AAC86E80F000DF5A5612046D6
:204140000BF098F994E80300FB787E908DF8FC11103D032B00F2A780DFE813F0A2006901D7
:2041600067016B0178AA76A95FFA89F005F084FE044600283FF49BAEFFF7ECBB0B4BDB78AD
:20418000032B00F2C483DFE803F01728323C00BF365906805E5206802FDB0600A2D50600BA
:2041A000C358068089DB0600A6D90600F8860380E0250680688703800123CDE901330093D0
:2041C00000231A46B6F830110F9811F0A1FA044600283FF47CAFFFF7BDBB0123CDE90133DE
:2041E00000930023B6F830111A461098EDE70123CDE9013300930023B6F830111A46119882
:20420000E3E70123CDE9013300930023B6F830111A461298D9E7B5F9800000281FDCB5F958
:2042200080000028BFF66AAFDDE9622312F020F9044600287FF48EABF87811F07BFF04464F
:2042400000287FF487ABFB78AF3306EBC3060134062CF6E80823E9E80223F8D14EE7DDE958
:20426000602312F005F9044600287FF473ABF87811F060FF044600287FF46CAB5A46CC463A
:20428000FB78973306EBC3030134062CD3E93001ECE80201F3E80801E2E80201F4D1BEE7E4
:2042A00001238DF8FD3164A905220DF5FF7050F0E8FC95F8F731590707D540F2FD300CF012
:2042C000B9F80446002800F0B68040F2FD30AE490AF0F0FF044600287FF43CABDDE972232F
:2042E00040F207400BF0D1F8044600287FF432ABDDE96410DDE9722398F85040002C40F0AE
:20430000A5808A1A60EB030340F239400BF0BDF8044600287FF41EAB0026FBE8020150EA34
:204320000102F3B240F0A68095F8F124F240D20700F1A0800136062EEFD1B8F89930DC073A
:2043400040F1C58098F85030002B00F0C080B8F89930580740F1C6800D980EF07BFD0122EF
:204360000023824040F21F400BF08FF8044600287FF4F0AA98F85030002B40F0BE800CF021
:20438000A9FF00287FF445AA80230A220DF5B376CDE9003202960DF595630B227EA91620ED
:2043A00009F0D6FE04460CF095FF08B10CF048FF002C7FF4CFAA81AB0DF59562318816202E
:2043C00009F0A2FBDDE9821270480FF097FA01210D980FF021FD06F077FD044600287FF472
:2043E000B9AADDE964230E99C7E90423DDE97423C1E900230CF03CFF02283FF40AAA0122FA
:20440000634B83F824250CF065FF08B10CF018FF0CF02EFF022840F0C7807B7A002B3FF4E1
:2044200099AA07F0E7F9FFF795BA022339E7032337E7042335E75749142284A853F00EF806
:204440008DF8244284A940F20C4041E7DDE97C64921944EB0303891ADDF8982460EB030096
:20446000DDF89C34891A60EB0300DDF8A024DDF8A43446E7013B042B04D8DFE803F00F140F
:20448000191E230040F24E40DAE900230AF0FDFF044600283FF44EAFFFF75CBADAE9022390
:2044A00040F24F40F2E702460B464FF48A60EDE702460B4640F25140E8E7DAE9082340F27D
:2044C0005240E3E7DAE90A2340F25340DEE732494FF483600AF0EEFE044600283FF437AFF4
:2044E000FFF738BA2D4940F2F1300AF0E3FE044600283FF431AFFFF72DBADDE97C2340F237
:20450000BF400AF0C2FF044600287FF423AA0DF58966D6E914234FF498600AF0B6FF044614
:2045200000287FF417AAD6E9162340F2C1400AF0ACFF044600287FF40DAA194940F22440BB
:204540000AF0B8FE044600287FF404AAB8F8993019070FD598F85020012A7FF610AF002319
:2045600040F2B9400AF091FF044600283FF407AFFFF7F0B90B4940F2A3400AF09BFE044646
:204580000028E7D0FFF7E6B98488038044880380509A0380165306808553068045540680F0
:2045A00096550680D655068040222021B44850F06CFB40222021B34850F067FBDDE96489A0
:2045C000FB78EE6B032B98BFAF4A404698BFD35C494698BF0C930C9B64220B93839B06F51C
:2045E000FA660A93829B0993A84B0893002353F009FC4046CDE9062349466422002353F02C
:2046000001FCCDE904016B6A32460293AB6AA0490193EB6A9A480093AB6B51F02BFF0CF027
:2046200059FE08B10CF00CFE002564A807F01EF9984E7B7A86F82D55002B4FD1B378F3B928
:204640000523B3701BE0A9B208FB01718B88C12BADF838362DD017D82F2B23D04D2B34D07D
:2046600001353A88ABB29A42EDD84FF400730DF5C760ADF83836FBF719FF07F0BBF800237B
:2046800086F82435FFF766B9C52B25D0DE2BE7D10B4653F8060F0DF5C862596803C2986825
:2046A00010600DE0412206310DF5C86050F0E9FA06E051F8060F8B88CDF84006ADF8443635
:2046C0000DF5C760FBF7F2FECAE751F8060F0DF5C863496803C3F3E75422E4E76E4F4FF005
:2046E0005608BEE71B7801210D98002B6BD00FF093FB032113981BF091FF00283FF48EA96E
:204700000121664A664C82F8FD10E378617902F5A056B1FBF3F1202982F8FC3086F800313E
:204720009EBF03F1FF33DBB282F8FC305D4A98BF86F80031927994F85130002A46D1002B92
:204740004AD0594C218811B3013989B214A8FBF71DFF4FF4887214A90DF5A56050F091FA22
:20476000BDF82835B3F5007F11D00025B4F80280494E3288ABB29A425AD84FF400730DF558
:20478000A560ADF82835FBF791FEA4F8028006F09BFB044600287FF4DDA8DDE964230E9989
:2047A000C7E90423DDE97423C1E900237B7A002B7FF437AE374B9A78002A7FF4CBA80522B5
:2047C0009A70FFF7C7B80FF027FB99E794F89520002AB6D1062BB4D00525DFF8A480DFF816
:2047E000D090404694F804A052F0E7FD4346CDE9000900222946504623F06AFE4FF6FF73DC
:2048000080B29842A6F8FE0005D096F8003162794343934207DA0135EDB2082DE1D14FF644
:20482000FF7398428DD0022120481BF0F7FE88E75623A9B203FB01618B88C12BADF838368F
:2048400038D008D82F2B14D04D2B3FD00023ADF8383601358DE7C52B3FD0DE2BF6D10B46AB
:2048600053F8060F0DF5C862596803C29868106027E0412206310DF5C86050F002FA20E0AF
:20488000D70C0780170D0780808A0600098803808F8A0600509A03800C2D03806CC40480E3
:2048A0005E520680095306801058038036E506006AC5048051F8060F8B88CDF84006ADF800
:2048C00044360DF5C760FBF7F1FDC2E751F8060F0DF5C863496803C3F3E75422CAE7352450
:2048E000FFF738B84024FFF735B85F24FFF732B84224FFF72FB84324FFF72CB84424FFF746
:2049000029B84D24FFF726B84524FFF723B83924FFF720B8F0B590F9003093B0002B0546F5
:2049200051DB21B3294B01211A7810238DF804302E4600244FF0200C01AB5818E7B2BA42AF
:2049400018D812AB1A4400230A44042002F8443C0DF0E0FAA0B32A78002302F003021C49F2
:2049600001A81BF01BFD70BB4B2013B0F0BD194B1A78DDE716F8013F037077B11B2B10D09C
:204980001F2B0ED816F8017C1B2F0AD00B2B08D01F2B18BF80F800C003E01B2B01D01F2B8D
:2049A000F4D901340130C9E712AB2344023403F8446CE4B201A852F000FD8442F4D3CAE753
:2049C00001247826F6E70020CFE700BF441E0010A2D50600401E001070B590F9003092B025
:2049E000002B044629DB407806F0B8FC012300228DF8040001AD5A550133412BFBD12A46D4
:204A00002026611C04F1410011F8013F1F2B17D95370884202F10102F6D1002604208DF801
:204A200045600DF077FA98B12278334602F00302094928461BF0B2FC60B1002012B070BD77
:204A4000002BE5D00B2BE3D01F2BE1D05670E0E77720F3E74B20F1E7A2D506002DE9F0438B
:204A6000334F8FB0FB7881468846002B53D0314C06A806AD1FF020F90FCD0FC495E80F00DE
:204A800004F130060DF1180C84E80F00BCE80F000FC695E80F0086E80F00103406AE0FCEE8
:204AA0000FC495E80F0084E80F000023CDE90133214900930122B1F83011204810F028FE77
:204AC000044670BB1EF050FBD9E9002304A8CDE90423FCF786F840BBB8F10C0F04A90CBFF2
:204AE0001748184805F08EF90446D0B9414604A805F086FE0446A0B906F0E6F9044680B901
:204B0000022111481BF08AFD50B1404606F02EFA0523BB7005E0022006F02CFC0028A6D1CB
:204B20004B2420460FB0BDE8F0834124F9E700BF509A038068870380E0250680A2D50600DE
:204B400010DC060019DC06002DE506002DE9F0418046C8B0734B0AAC0FCB84E80F0098F872
:204B60000030042B00F2DB806F4B93F84D30D90607D56E4B0A936E4B0B936E4B0C936E4B4E
:204B80000D936E4E737A002B47D1B37A002B44D16B4BDB7C002B40D001237372B37E002B6F
:204BA00040F08980674D0EA80EAC1FF085F80FCC0FC594E80F0005F130070DF1380C85E8F6
:204BC0000F00BCE80F000FC794E80F0087E80F005D4B1B78022B2ED116A90EA81FF0C4F88D
:204BE0001FA905F150001FF0BFF816A852F08CFC04461FA852F088FC544B201ADA796FF0F7
:204C00003B03534303F5A83303F5C073984212D903200DF02BFD162409E04B4BDB78002B7E
:204C2000BCD1022006F0A6FB0028B7D14B24204648B0BDE8F0810EA906A80AF01BFC002302
:204C400001220093CDE9012306A90522152009F07FFA04460028EAD10CF048F830790EF037
:204C6000BDFA80230A220DF11605CDE9003221462246029528AB102009F06AFA0446002875
:204C8000D5D128AA08AB2988102008F03DFF9DF8202032B9BDF82230ADF824200133ADF84B
:204CA0002230BDF82200BDF824100FF023FA98F8000011F03FFA224B1B7CB3B11EF054FA38
:204CC00074783CBB98F8000006F050F921460C221F4834834FF0D9FF08200DF0C7FC194B0C
:204CE000D3E90E100EF01AFCA1E798F8000048AA02EB80000122CDE9012216490092B1F8B9
:204D000030111A4650F8F80C10F002FD04460028D4D08CE7338B00240133338387E733248D
:204D200085E700BF708A06003753068097DF0600F7D7060028D8060073D80600F886038090
:204D4000C358068068870380509A03805E52068054870380E02506802DE9F04FA9B0D0E94D
:204D60000023CDE90423CDE906239A4B074693F8502088461AB19B78012B40F2148104A8DC
:204D8000FBF72FFF78B1A8F10703042B0BD8DFE813F0CE000A0005000500CE005B242046B6
:204DA00029B0BDE8F08F0CF095FA002840F0FD80894DA8F10703E8780193042B3ED8DFE81D
:204DC00003F0033D15273200844C403004EB40001EF00DFAE9780E237F3104EBC10104AA0D
:204DE000084614F0C2FD48B38B24D8E77B4C443004EB40001EF0FBF9E9780E23833104EB98
:204E0000C10104AA084614F0B0FDB8B18A24C6E7724A833002EBC00204A9104614F0B8FD85
:204E200060B18C24BBE76D4A7F3002EBC00204A9104614F0ADFD002840F0B980E97804A8AB
:204E400005F064FC04460028A9D1424606A9384606F0DAF804460028A1D1AB7E3BB1AB7A76
:204E6000002B9CD1DDE90423C5E9042397E75C490B88002B5BD0013B9BB29A1CA8F10A00EA
:204E800001EB420201EB8303C0B232F80269802E49D3832E43D9842E45D1B8F1070F40D03B
:204EA000B8F1090F3DD0D3F8A46F8B423DD0043B002EEAD08022314608A84FF0E2FE0A98BB
:204EC0000D9B0C9900FB03F20B9BA0FB018901FB032399444FF47A7200234046494652F022
:204EE00091FF4FF47A7282468B4600234046494652F088FF002B08BFB2F5FA7F03D31AF166
:204F0000010A4BF1000B334B9B78002B51D1019B042B2CD8DFE803F00D2B3D3D0D000128F0
:204F2000C1D833243BE70026BFE7002EC2D1402435E70E9A109B0F999B1A119A62EB0102A7
:204F400013EB0A03029342EB0B030393DDE90201D7E90023994208BF9042E8D3D7E9001035
:204F60000E9B0F9A5B1840EB0202CDE90E32802208A930464FF085FEE87811F0DBF830B99F
:204F8000E97804A805F0C2FB00283FF468AF044605E7109B119AD7E900105B1840EB0202E2
:204FA000CDE91032E3E73524F9E67524F7E68D24F5E6019B042BDAD801A252F823F000BFB9
:204FC0005D4F01006F4F0100934F0100934F01005D4F01005E520680F8860380E025068030
:204FE000105803802DE9F0416E4D8CB004A804AC1EF062FE0FCC0FC594E80F0005F1300658
:2050000004AF85E80F000FCF0FC694E80F0086E80F0005F1100704AE0FCE0FC794E80F00A9
:2050200087E80F00604F103DFB78002B00F0AE800023CDE901335D4C00931A46B4F83011A4
:205040005B4810F065FB0646002840F0A680012004F0FEFF0646002840F09F8004F529612B
:20506000544804F08FFF0646002840F09680524B5B695B057FD40CF02DF908B10CF0E0F895
:205080004FF0000C4D4B60461C466146E4E80401C4E900CC1024C5E980CCC5E984CCC5E95A
:2050A00082CCC5E986CCC3E902CCC3E906CCA3F58063E3E80201013C14F0FF04C3E91E0152
:2050C000C3E93E01C3E95E01F3D120254FF001082A46CDE900853A4B21463A483FF0EBF95D
:2050E000CDE9008504254FF04008344B2D22214634483FF0E0F9344B24222146CDE90058D2
:2051000030483FF0D8F9314B25222146CDE900582C483FF0D0F92E4B26222146CDE900583D
:2051200028483FF0C8F92B4B27222146CDE9005824483FF0C0F9284B28222146CDE9005855
:2051400020483FF0B8F9254B29222146CDE900581C483FF0B0F9224B2A222146CDE900586D
:2051600018483FF0A8F9CDE900581E4B2B22214614483FF0A0F902211B481BF04FFA58B1CD
:2051800005230F20BB7005F0F1FE06E0022006F0F1F800287FF44CAF4B2630460CB0BDE8E4
:2051A000F08100BF68870380509A0380E025068021DC06003FDC06004080092090900380A5
:2051C0006889038080002000908C0380D08C0380108D0380508D0380908D0380D08D03803D
:2051E000108E0380508E03802DE506002DE9F04FB84BB94A9B79D3B0002BB84B08BF1346D5
:20520000B74A059308BF9246B64BB74A14BF9A469346B64BB64A18BF9B46B64B08BF1346EE
:205220000493B54BDB78002B00F09881B34C28A828AD1EF041FD0FCD0FC495E80F0004F130
:20524000300628AF84E80F000FCF0FC695E80F0086E80F00103428AE0FCE0FC495E80F00B4
:2052600084E80F000023CDE90133A54D00931A46B5F83011A34810F04BFA2E4604460028BD
:2052800040F0B6810146102218A84FF0FEFC102221461CA84FF0F9FC1022214620A84FF004
:2052A000F4FC1022214624A84FF0EFFC2F46A046B7F890305FFA88F9002B40F05781B7F8E9
:2052C0009230002B40F05281B7F89430002B40F04D81B7F89630002B40F0488108F10108A7
:2052E000B8F1100F07F10807E2D1032158461BF095F9002800F03881834930A852F03CF8E6
:20530000082218A916A84FF0BCFC16A941A8FBF78FFD0023032241A930A81BF03FF8002853
:2053200000F02281794930A852F026F808221CA916A84FF0A6FC16A941A8FBF779FD00231F
:20534000032241A930A81BF029F8002800F00C816F4930A852F010F8082220A916A84FF0CB
:2053600090FC16A941A8FBF763FD0023032241A930A81BF013F8002800F0F680654930A873
:2053800051F0FAFF082224A916A84FF07AFC16A941A8FBF74DFD0023032241A930A81AF071
:2053A000FDFF002800F0E080032150461BF036F9002800F0D980B6F81021574930A851F07C
:2053C00059F8564930A804F01DFD0446002840F00F81B6F81221524930A851F04BF8514953
:2053E00030A804F00FFD0446002840F00181B6F814214D4930A851F03DF84C4930A804F089
:2054000001FD0446002840F0F380B6F81621484930A851F02FF8474930A804F0F3FC04462E
:20542000002840F0E580032105981BF0F7F8002800F09A80B6F81821374930A851F01AF830
:205440003D4930A804F0DEFC0446002840F0D080B6F81A21324930A851F00CF8374930A855
:2054600004F0D0FC0446002840F0C280B6F81C212D4930A850F0FEFF314930A804F0C2FC0E
:205480000446002840F0B480B6F81E21284930A850F0F0FF2B4930A804F0B4FC044600286F
:2054A00040F0A680032104981BF0B8F800285BD0154930A851F060FF00220023CDE90623CE
:2054C000CDE90823CDE90A23CDE90C2305F509663AE000BF0953068028DF060013DF0600FA
:2054E000FADE0600E6DE0600C8DE0600B0DE060056DF060042DF0600509A03806887038083
:20550000E02506805DDE060080DD06009CDD0600B8DD0600C9DD060051D70600302E068084
:205520005ED70600382E06806BD70600402E06807ED70600482E0680502E0680582E0680A1
:20554000602E0680682E068006A90E233219084614F00BFA00284FD0482449E0022005F0A6
:2055600009FF00287FF462AE4B2441E0BC4930A851F002FFBB4B402203EB881141A84FF0B2
:2055800080FB41A851F019FFB74B41A91B6883423EBF52AA9B18002230A838BF03F8442C12
:2055A000002303221AF0FAFE0028DDD018AB00224946AE481AF0A2FA0446C8B91CAB012207
:2055C0004946AB481AF09AFA044688B920AB02224946A8481AF092FA044648B924AB0322DD
:2055E0004946A5481AF08AFA044600283FF476AE204653B0BDE8F08F2034802CA4D104468C
:2056000005F6984606A900233219084614F0ADF90028A1D12034B4F5C07FF3D1044605F6BD
:20562000980608A90E233219084614F09EF9002892D12034802CF4D1044605F54A6608A9C1
:2056400000233219084614F090F9002884D12034B4F5C07FF3D1044605F6A8060CA90E23AB
:205660003219084614F081F900287FF475AF2034802CF3D1044605F54B660CA90023321978
:20568000084614F072F900287FF466AF2034B4F5C07FF2D1044605F50A660AA90E233219BB
:2056A000084614F062F900287FF456AF2034802CF3D1064605F6A8450AA90023AA190846BE
:2056C00014F053F9044600287FF446AF2036B6F5C07FF1D106A9694804F054FC08A9684899
:2056E00004F050FC0AA9674804F04CFC0CA9664804F048FC654B93F89730012B1BD0022BEB
:2057000000F0A08006A90E230CAA084614F02DF908A90AAA08460E2314F027F906AA08A902
:205720000CA814F035F9002800F0C1800CA8FBF71BFA0CA983E0002200232746CDE90E23BE
:20574000CDE91023CDE91223CDE91423504E0EA90E233246084614F008F900287FF4FCAEF2
:2057600010A90E2306F11002084614F0FEF800287FF4F2AE12A90E2306F10802084614F074
:20578000F4F800287FF4E8AE14AD0E2306F118022946284614F0E9F800287FF4DDAE0137C9
:2057A000042F06F12006D2D106463A4F0EA900233A46084614F0D9F8034600287FF4CCAE46
:2057C00010A907F11002084614F0CFF8034600287FF4C2AE12A907F10802084614F0C5F8CD
:2057E000034600287FF4B8AE07F118022946284614F0BBF800287FF4AFAE0136092E07F15B
:205800002007D3D10EA90E232A46084614F0ADF800287FF4A1AE10A90E2312AA084614F08C
:20582000A4F800287FF498AE0EAA10A912A814F0AFF8002836D012A8FBF796F912A9164893
:2058400004F0A4FB022115481AF0E8FE00283FF48BAE0522124B17209A7005F087FBC7E6C8
